:020000040000FA
:040000006FD00400B9
:101000006F00907D00000000000000009020002094
:10101000AA220020A9BDF9F56C23002000000000E1
:10102000000000006C230020902000200000000041
:101030000000000090200020000000009020002010
:101040000000000090200020902000209020002030
:101050009020002090200020482F00208224002093
:101060000000000090200020902000200C24002090
:1010700090200020D22300209020002090200020EB
:101080009020002090200020902000209020002020
:101090009020002001A04111B7170040985F3AC688
:1010A000945F3247E39CE6FE3245410182800111A4
:1010B00013078008F337078093F787083EC20100C3
:1010C0000100B7170040930570052380B70413068D
:1010D00080FA2380C7040100010083C6B70493F699
:1010E000F60DA385D704238007049246F3A6068055
:1010F0000100010093760502D5CEF336078093F602
:10110000860836C4010001002380B7042380C70489
:1011100001000100B70614007D89558D88C70100C4
:1011200001000100010023800704A246F3A6068007
:101130000100010073370780137787083AC6010062
:1011400001002380B7042380C704010001000100CF
:1011500001003727004093061005A303D7802380A2
:101160000704B247F3A70780010001009307800836
:10117000F3B7078093F787083ECE01000100B71749
:101180000040130770052380E704130780FA2380CB
:10119000E7040100010003C7B70413670708A3852C
:1011A000E70423800704F247F3A70780010001004A
:1011B0000561828093760504BDC6F336078093F6F9
:1011C000860836C8010001002380B7042380C704C5
:1011D00001000100B7061400938606047D89558D31
:1011E00088C7010001000100010023800704C246F6
:1011F000F3A6068001000100733707801377870884
:101200003ACA010001002380B7042380C70401000B
:1012100001003727004093062005A303D7802380D1
:101220000704D24781B773370780137787083ACC12
:10123000010001002380B7042380C70401000100DE
:1012400098471367070C98C723800704E24719BF24
:101250000111814601468145114506CE97000000E7
:10126000E780405793078008F3B7078093F7870814
:101270003EC601000100B717004013077005238028
:10128000E704130780FA2380E7040100010003C785
:101290006704136717002383E70423800704B2471A
:1012A000F3A7078001000100F2400561828041112F
:1012B000814601468145114597000000E780805135
:1012C00013078008F337078093F787083EC40100AF
:1012D0000100B7170040130670052380C70493066A
:1012E00080FA2380D70401000100FD552396B70240
:1012F00023800704A245F3A5058001000100733790
:101300000780137787083AC6010001002380C704CD
:101310002380D7040100010003C767041367170087
:101320002383E70423800704B247F3A70780010063
:10133000010001A0B1473305F50201007D1575FDDF
:101340008280411122C426C206C6AA8401446317C2
:101350009400B24022449244410182800504130566
:10136000803E420497000000E78000FD4180C5B741
:101370009305000273A04580824573901534924016
:101380002242B2424243D2436244F2440255925551
:101390002256B2564257D2576258F25806499649D9
:1013A000264AB64A464BD64B664CF64C065D965DD1
:1013B000265EB65E465FD65F09617300203041113C
:1013C000B7170040985F3AC6945F3247E39CE6FE49
:1013D000324541018280B71700401307000323887C
:1013E000E702854717170000232AF75C73002030B7
:1013F000411122C406C637040020977000E0E78040
:10140000E08B975000E0E780E0BA1C408297F5B788
:1014100037370040834747009146BD8B639ED70214
:10142000B73600401306F00F973500009385053658
:101430009737000083D7874503C7A6001377F70FB8
:101440001DE3B7E70400BC4F0946894517150000A6
:10145000034585F7829731A099466394D700834767
:1014600057007300203003C786001377F70FE3653A
:10147000F6FC13851700AE97173800002318A84014
:101480002380E70075B7B787004003C76700098B63
:101490006309071003C77700930600031377070358
:1014A000630DD708174800000348D8951746000079
:1014B000130686940547B30606012380E60083C51C
:1014C0007700174700001307A793429793F5F50F8E
:1014D0002300B70003C58700974500009385059258
:1014E000C2951375F50F2380A500034707008945B2
:1014F0001377F703630CB70C63E7E50A6306071A73
:101500008545630CB7129747000083C7B78F330731
:10151000F600034707001377F70F19CB850793F7FA
:10152000F70F0D476363F71A17470000A30CF78CFA
:10153000B787004009472383E700B787004083C788
:101540007700E207E18763DE07049747000083C75F
:10155000778B174700001307278A3E97854623009D
:10156000D700174700001307A7893E97930600038B
:101570002300D70017470000130747883E97A1466E
:1015800085072300D70093F7F70F0D476364F7141F
:1015900017470000A308F786B78700400947238351
:1015A000E70073002030930610026300D70E930605
:1015B00020026305D70693060002E316D7F403C79B
:1015C00027021377C70F13672700D5A803C7670043
:1015D0001377070465CB03C7A70217380000130869
:1015E0002863173500001305655A1347070823853C
:1015F000E70203C7A7021377370F13678700238516
:10160000E702814713070004B305F5008C41B306D8
:10161000F80091078CC2E399E7FEF5B503C7A7026E
:10162000134707042385E70203C7A7021377C70FF1
:10163000136727002385E702F9B503C7670013770F
:10164000070449C303C7670217380000130808508E
:101650001735000013054547134707082383E702A2
:1016600003C767021377370F136787002383E702E7
:10167000814713070004B305F5008C41B306F80059
:1016800091078CC2E399E7FEBDBD03C7670213470C
:1016900007042383E70203C767021377C70F1367A3
:1016A00027002383E70285B503C767001377070484
:1016B00011CB03C727021377370F136787002381E6
:1016C000E70291B5238006003DBD97370000A38B4C
:1016D0000772B9BD97370000A386077275BD230353
:1016E000048015472303E48001002302A480828044
:1016F00083076480E3CE07FE230304808280830790
:101700006480E3CE07FE03454480828083076480C3
:10171000E3CE07FE2302A4808280411126C44AC280
:101720004EC006C61377F50BAD47AA892E8995449E
:10173000630CF700194597000000E78080FA9700D6
:101740000000E78020FB8D444E8597000000E78075
:1017500040F9FD59FD1463983401B240A244124986
:10176000824941018280135509011375F50F9700D5
:101770000000E780E0F92209F1BF011126CC06CE76
:10178000B704080097000000E780C0F615459700F1
:101790000000E78000F597000000E78080F69700E2
:1017A0000000E78000F62AC697000000E78080F47A
:1017B00032459377150089EB136515001375F50F06
:1017C000F240E24405618280FD14E9F00145CDBF9D
:1017D000397126DC4ADA4ED852D656D45AD25ED067
:1017E00006DE62CE66CCB7E700E07D5783AA07002D
:1017F00022C603AA470023A0E71823A2E718B717B9
:101800000040130770052380E704130780FA238044
:10181000E70483C74704930B75FFB684E20793FB85
:10182000FB0F8546AA892E8B328937240040E18739
:10183000015763FA76016308D50089461307000251
:101840006313D5000157D98F93F7F70FB71C0040EA
:101850002382FC0411472303E4801305F00F970053
:101860000000E78000E8094C97000000E78080E86E
:1018700063657C15B7050700DA953787070079554A
:1018800063FEE504B3879500636AF704370B08002D
:10189000A94733EB65016395F90881E88144970016
:1018A0000000E78020E5268515A8DA850945970020
:1018B0000000E780C0E605090345F9FFFD14050BAC
:1018C00097000000E780C0E481C49377FB0FE5F741
:1018D00097000000E780A0EA69F17D55B717004046
:1018E000130770052380E704130780FA2380E704B9
:1018F00003C74704418B2382E704F250B7E700E0B7
:1019000023A0571123A24711E25432445259C2591D
:10191000325AA25A125B825B724CE24C2161828085
:10192000A547639BF90685691309F00FB306990073
:10193000B3742B01B6941349F9FFB3749900856B06
:1019400033796901416B9387F9FFB3F7270199E375
:1019500063FC340193D94900C147E3E637FF3DBF3B
:101960000569C1697D19D9B71305800D63886901BF
:10197000130500026384790113051008CA859700D6
:101980000000E780C0D997000000E78040DF31D534
:101990004E99B38434416DBFDA852D459700000020
:1019A000E780E0D7CA94E30B99EE050997000000A1
:1019B000E78020D5A30FA9FEFDB79387F9FF93F722
:1019C000F70F636DFC0C83C71C0413073008631505
:1019D000F706370708006361EB06B3079B00B706FD
:1019E000100063FBD704334BEB0089476399F9067A
:1019F0008980D549E38404EADA8509459700000027
:101A0000E780E0D111090327C9FF91472320E48033
:101A100003076480E34E07FE23033481FD17EDFBCB
:101A2000FD14110B81C49377FB0FE9FF97000000B1
:101A3000E780E0D461F155B5B717004003C75704FC
:101A4000B70708001377070219E3B787070079552E
:101A5000E376FBE833079B00E3F9E7F841B58547F8
:101A6000E380F9F0DA852D4597000000E78020CB70
:101A70009389F4FFE38404E297000000E78060C8E4
:101A800093F7390091EB832604800327090093071D
:101A90004900E396E6E03E89CE84D9BFB547639915
:101AA000F9001305900B97000000E78080C3FDB399
:101AB000B1471305B00AE388F9FE99476397F90423
:101AC000B7050800B365BB002D4597000000E7800F
:101AD00000C581448D4BA14997000000E78060C29A
:101AE00063967401832704802320F9008504E3951D
:101AF00034FF8327048013172B016355070023123B
:101B0000F90069BB2322F90051BB9D47639FF9028D
:101B100081451305B00497000000E78040C0BD4434
:101B20002320090023220900FD5997000000E780C7
:101B300040BD93F77400CA9703C70700FD14398DA1
:101B40002380A700E39334FF91BBA1476397F90675
:101B500097000000E780A0C28144630D0B008D4711
:101B60009304C0036308FB009304000563048B0126
:101B7000930440041375C507E30295D219459700F5
:101B80000000E78000B697000000E780A0B605459A
:101B900097000000E780E0B4268597000000E7800A
:101BA00020B7094597000000E78080B69700000045
:101BB000E780E0BCE31405CE0DB39147639FF900C5
:101BC0001305600697000000E780A0B197000000B1
:101BD000E78040B213059009F9B5E38109CCF154CF
:101BE0007DB9BD660147173600001306263F938670
:101BF00006A685458347060093F7F70F91C38280B9
:101C00000507E3F9E6FE973700002389B73CDDB707
:101C10007D166206618693178601E18763D407000B
:101C200001458280931726003307F500AE971843CD
:101C30009C4363E7E7007D16E37FF7FC7D558280D8
:101C400005458280FD15E205E185139785016187D1
:101C500093F7F50F63480700FD15139725002A97A2
:101C6000584365D713851700620561858280330864
:101C7000B5021C4283A80600B335B502C29733B53E
:101C80000701AE98469585486367B5006394A50043
:101C900063E3070181480C43C6950CC388C21CC28C
:101CA000828081471397870161876343B7008280F1
:101CB000139727002A97232007008507E5B7814758
:101CC000014793968701E18663C5B6001335170077
:101CD000828093962700AA9694428507558FD5B7A0
:101CE00093D755408A07AA979C4305453315B500FD
:101CF0007D8D828017F3FFDFE702A33D2A849700E2
:101D00000000E78060F405C5931725003E94032783
:101D1000C4FF814711EB7D1516053E9542054185AF
:101D200017F3FFDF6700233D05838507E5B701450E
:101D3000C5BF81471397870161876343C7008280CE
:101D400013972700B386E50094422A97850714C3AA
:101D5000D5B77D1662066186014793178601E18734
:101D600063D5070013351700828093172600B3064A
:101D7000F500AE9794429C437D16B58F5D8FF1BF01
:101D80008A05AA9501476363B500828083A6C5FFD3
:101D9000F11593D71600D98F9CC11397F601E5B7BB
:101DA0002A830148014701456343D7008280B387F6
:101DB000050183A80700B30706019C43C697AA97AD
:101DC0006384F80033B517010507B3080301620700
:101DD00023A0F80061871108C1BF2A83014781470A
:101DE000014563C3D70082803388E500832808005B
:101DF000330EE600032E0E003388A8403308C84196
:101E00006384080133B508018507B308E300E207DE
:101E100023A00801E1871107E9B717F3FFDFE70205
:101E2000432B0111B286B2842E86AA850A859700BB
:101E30000000E780C0FA2A84A6850A859700000082
:101E4000E78020E833348000060413351500018D47
:101E5000056117F3FFDF6700032A17F3FFDFE702CF
:101E6000C3244111AA89AE8A328BB68402C202C44D
:101E700002C60144131C8401135C8C4163499C021B
:101E8000939B1400FD1B0549138CF4FFF15C330494
:101E90008901620461846340740792478E04CE9482
:101EA00023AEF4FE410117F3FFDF6700832313190C
:101EB0002400B30B2B01014A93172A00D69783A560
:101EC0000B00884378003400500097000000E78042
:101ED00040DA050A93178A01E187F11BE35EFCFCF7
:101EE00092474E9905042320F900A2473EC2B2470B
:101EF00002C63EC441B7131A8901135A8A41131D01
:101F0000240093178A01E18763CF970092470A0460
:101F10004E941CC0A24705091379F90F3EC2B2477F
:101F200002C63EC4ADB7B3079A0313152A005695EF
:101F30000841780034005000050AEA97DA978C438C
:101F400097000000E780E0D26DBF0000197106C263
:101F500012C416C61AC81ECA22CC26CE2AD02ED229
:101F600032D436D63AD83EDA42DC46DECAC0CEC2D9
:101F7000D2C4D6C6DAC8DECAE2CCE6CEEAD0EED209
:101F8000F2D4F6D6FAD8FEDA97150000938585A22A
:101F90008841E700050092402242B2424243D243C8
:101FA0006244F244025592552256B2564257D257D5
:101FB0006258F25806499649264AB64A464BD64BCD
:101FC000664CF64C065D965D265EB65E465FD65F55
:101FD0000961730020300000972100209381810265
:101FE000175100201301018217F5FFFF1305C501EA
:101FF0009705002093850501171600201306C6FDDE
:1020000063FAC5008322050023A055001105910540
:10201000E3EAC5FE171502001305C5EF971500206A
:102020009385C5FB171600201306467C63FAC5008E
:102030008322050023A0550011059105E3EAC5FEA2
:10204000171500201305857A9745002093850545CF
:102050006377B500232005001105E36DB5FEFD4251
:10206000739002BC8D4273904280B722000093822D
:10207000828873900230970200209382A2F893E244
:1020800032007390523097520000938242AF7390A7
:1020900012346FB0F47673002030397101436EC68C
:1020A00019A0397141536AC866CA62CC5ECE19A0C4
:1020B000397101535AD056D252D44ED64AD826DA64
:1020C00022DC06DE33016140828241114AC026C211
:1020D00022C406C68282B24D4101024D924C224C6E
:1020E000B24B4101024B924A224AB2494101024994
:1020F00092442244B240410182803D432A87637367
:10210000C3029377F700BDEFADE5937606FF3D8AF6
:10211000BA960CC34CC30CC74CC74107E36BD7FE40
:1021200011E28280B306C3408A06970200009696A9
:102130006780A6002307B700A306B7002306B700F1
:10214000A305B7002305B700A304B7002304B70015
:10215000A303B7002303B700A302B7002302B7000D
:10216000A301B7002301B700A300B7002300B70005
:10217000828093F5F50F93968500D58D9396050192
:10218000D58D61B7939627009702000096968682B8
:10219000E78086FA9680C1171D8F3E96E374C3F8D8
:1021A000A5B73367B500FD530D8B79E7B7877F7F00
:1021B0009387F7F710419441B372F6003363F6004A
:1021C000BE92B3E262006397720C6318D606504168
:1021D000D441B372F6003363F600BE92B3E26200FC
:1021E0006398720A631BD60410459445B372F600D7
:1021F0003363F600BE92B3E262006391720A631E1B
:10220000D6025045D445B372F6003363F600BE9251
:10221000B3E26200639A72086311D60210499449CE
:10222000B372F6003363F600BE92B3E262006393CA
:1022300072085105D105E30FD6F6131706019397DF
:102240000601631CF7001357060193D706013305F7
:10225000F7409375F50F91E982804183C18333057F
:10226000F7409375F50F91E182801377F70F93F79D
:10227000F70F3305F74082800346050083C605004B
:10228000050585056313D60065FA3305D6408280BF
:1022900011059105E312D6FE014582802105A105B5
:1022A000E31CD6FC014582803105B105E316D6FC5E
:1022B000014582804105C105E310D6FC01458280BD
:1022C000B717004003C777051377E70FA38BE70421
:1022D000130700F8A38DE7043D47238CE704130799
:1022E0005003A38CE70403C7A7051377D70F238DEB
:1022F000E7048280B717004003C7E7020D89411148
:102300001377C70F498F93068008F3B6068093F6BC
:10231000860836C601000100930670052380D704A5
:10232000930680FA2380D704010001002387E70287
:1023300023800704B247F3A7078001000100410191
:10234000828041112A83014E930E407E130F0019A3
:10235000930F400663E56E129308001913034006BD
:10236000B3781503854E0D4FA14F337365020D8968
:102370001335150063EFBE121308F6FF7946729805
:102380004208135808013307C70213D61700BE07C7
:1023900032976146B3F6C60213068070B386C60252
:1023A0003697A166F58F42075D8FB716004083C749
:1023B000F60293F70708A303F1000346710083C7F1
:1023C000F60293F70708E394C7FE83477100B71638
:1023D000004093F7F70F6388071293078008F3B75D
:1023E000078093F787083EC401000100B71700403B
:1023F000930670052380D704930680FA2380D704C0
:102400000100010023AA070383C6170393E6060809
:10241000A388D70223800704A247F3A707800100FF
:1024200001001166B71700407D16D45BC85F938525
:102430004703A98EF18EF5FA93068008F3B606805D
:1024400093F6860836C601000100930670052380C6
:10245000D704930680FA2380D7040100010098C1B5
:1024600003C7170313670704A388E7022380070441
:10247000B247F3A7078001000100410182807D136C
:102480003368E3039308E016630E08003368F30330
:102490009308D016630808009378330093B81800A7
:1024A0009388D81633081E01131E0801135E0E010F
:1024B00055B56393E5030548638608000148630347
:1024C00003002A8871087298FD15131E0801C205C1
:1024D000135E0E01C18179BD13F8150063F4BF00CE
:1024E0007908D5B713381800E5BF83C7F60293F70C
:1024F0000708A303F1000346710083C7F60293F7B0
:102500000708E394C7FE8347710093F7F70FF1DFE5
:10251000E9B531714AD966CB06DF22DD26DB4ED71D
:1025200052D556D35AD15ECF62CD6AC96EC7AA8C36
:1025300002D897100000E78020B12A89930780080D
:10254000F3B7078093F787083EDA01000100B71759
:102550000040130770052380E704130780FA2380E7
:10256000E7040100010003C7F7021377770FA38781
:10257000E70203C7F70213678700A387E7022380F8
:102580000704D257F3A70780010001000545970013
:102590000000E78060D6130780C13347E902116A63
:1025A00093070AE893065002BD69930BA004814A81
:1025B000014B13048008930470057D1AB347F90298
:1025C0003307D7023EC0FD873ECC938709A6930907
:1025D000803E3347F7023AC27D873AC43347390316
:1025E0008549B399990193D93940B306D702B30B02
:1025F0007703B3C6F602B3CBFB0236C6FD8636C8F8
:1026000093D6FB4136CEB7460F0093860624334956
:10261000D9028566938606FAB3969601B389E902D4
:10262000130760553309D90293060010B389E902F4
:102630003349D902B3C9F9029316390036CA37199A
:102640000040FD8636D0930D090493D7F9413ED260
:10265000F336048093F6860836DC01000100930708
:1026600070052380FD00930680FA2380DD000100C1
:1026700001008346390593F6860FA309D9048346E2
:10268000390593E61600A309D90423800D00E2560C
:10269000F3A6068001000100130C80FA116DF336D9
:1026A000048093F6860836DE01000100930770056A
:1026B0002380FD0023808D01010001008346390540
:1026C000216693E60602A309D90483560905B3E6F9
:1026D000A6012318D90483560905D18E2318D904DD
:1026E00023800D00F256F3A6068001000100834608
:1026F000390593F606026381061A03463905218AD5
:102700006DDE081897100000E7800098733604808B
:1027100013768608B2C20100010023809D00238049
:102720008D0101000100B717004003C6370513767D
:10273000F60DA389C70403C6370513660602A389ED
:10274000C704835609052166B3E6A6012318D904F8
:1027500083560905D18E2318D90423800D0096468F
:10276000F3A60680010001008346390593F60602B0
:10277000638B061483463905A18AEDFE970000207D
:10278000E7806091AA8636D497000020E780A09069
:10279000A256E30AD5FE835609054255B3E6A601C3
:1027A0002318D90497100000E780C08F83463905AD
:1027B000A18AEDDE03560905834629058247337653
:1027C000CA00B306DA0293D5F641B296B388F64052
:1027D000E24733B8C6002E983308F840A247B3B694
:1027E00016013308D84063C70701631DF8009247FC
:1027F00063FA1701C247634FF80E63950701B247AA
:1028000063EAF80E894663E9660FF24693151800ED
:1028100013D3F8015E8613951800B365B30042D652
:1028200046D497C00100E78020313258050B137B56
:10283000FB0F63470001631A0838A2586387083802
:1028400013081500B336A800B69513D6F5013298D3
:10285000B336C800AE9613581800FE06B3E606015C
:102860007336048013768608B2C601000100238007
:102870009D0023808D01010001000356C902B2961C
:10288000C206C1822316D90223800D00B646F3A6E4
:1028900006800100010021B5F336048093F6860816
:1028A000B6C00100010023809D0023808D0101003E
:1028B00001008346390593E60602A309D904238063
:1028C0000D0086460DB5F336048093F68608B6C42F
:1028D0000100010023809D0023808D010100010083
:1028E0008346390593E60602A309D90423800D0027
:1028F000A646BDB5E30B0BF0F336048093F68608CD
:10290000B6C801000100930680FA23809D00238051
:10291000DD00010001008346390593F5FC0F93F6B5
:10292000860FA309D90483463905CD8EA309D9049E
:1029300023800D00C646F3A60680010001001305A2
:1029400080FA03463905930639051D8A631C9629CA
:102950007336048013768608B2CC0100010013069A
:1029600080FA23809D002380CD000100010003C672
:1029700006001376F60D2380C60003C60600136614
:1029800006022380C600835609051166D18E2318DE
:10299000D904835609052166D18E2318D9042380D2
:1029A0000D00E646F3A6068001000100130680FA3A
:1029B0008346390593F60602638006268346390569
:1029C000130C3905A18AFDDA081897000000E7808A
:1029D000A06BF336048093F68608B6D001000100A0
:1029E000930680FA23809D002380DD000100010012
:1029F00083460C00116693F6F60D2300DC00834637
:102A00000C0093E606022300DC0083560905D18EF4
:102A10002318D904835609052166D18E2318D904B9
:102A200023800D008656F3A60680010001001306E0
:102A300080FA8346390593F60602638A06208346A8
:102A40003905A18AEDFE97F0FF1FE780C0642A8C4C
:102A500097F0FF1FE7802064E30C85FF835609058C
:102A600011664255D18E2318D90497000000E780E3
:102A700060638346390513063905A18AFDDAF3360A
:102A8000048093F68608B6D401000100930680FA0C
:102A900023809D002380DD000100010083460600A5
:102AA00093F6F60D2300D60023800D00A656F3A65C
:102AB0000680010001008356090503462905D24717
:102AC000B376DA003306CA021305800C9355F6413B
:102AD0003696330DF6408257333CD6002E9C333663
:102AE000A601330CFC40330CCC40330885039256CE
:102AF0004E86B335A5033305A503C29597C00100E3
:102B0000E780800363468001631E0C16630C0D167C
:102B1000130615003335A6002E959356F50136960B
:102B2000B335D600AA959396F50105828585D18E99
:102B30006346B000639D051A638B061A0356C902EB
:102B400015823305D6003336C500B2956348B00010
:102B5000639105241306F00F637DA622894663F373
:102B6000561593078008F3B7078093F78708BED6FA
:102B70000100010037170040930770052300F70498
:102B8000930780FA2300F704010001008356C7026F
:102B900089678117D58FC207C1832316F7022300E7
:102BA0000704B657F3A7078001000100FA506A54E2
:102BB000DA544A59BA592A5A9A5A0A5BFA4B6A4C59
:102BC000DA4C4A4DBA4D296182801308F5FF33353E
:102BD000A800FD152E951356F5013298B336C8009E
:102BE000AA9695B9F336048093F68608B6CA010012
:102BF000010023809D002380AD0001000100834679
:102C00003905CD8EA309D90423800D00D646F3A63D
:102C100006800100010035B3F336048093F6860880
:102C2000B6CE0100010023809D002380CD0001006D
:102C300001008346390593E60602A309D9042380DF
:102C40000D00F646F3A606800100010095B3F336A9
:102C5000048093F68608B6D20100010023809D000F
:102C60002380CD00010001008346390593E606026A
:102C7000A309D90423800D009656F3A6068001000F
:102C8000010045BB9306F5FF33B5A600FD152E9553
:102C90009355F501AE96B3B5B600AA951396F50116
:102CA000858269B5F336048093F68608B6D80100AC
:102CB0000100930680FA23809D002380DD0001003F
:102CC00001008356C9020566011693F6F60FD18EF0
:102CD000C206C1822316D90223800D00C656F3A670
:102CE000068001000100850A93FAFA0F95B233E6D7
:102CF000B60045C20356C9023305D0403338A000A0
:102D0000B305B040B385054115826345B000D1E1FC
:102D10006371A608894663F0560593078008F3B7E8
:102D2000078093F78708BEDA01000100B71700405B
:102D3000130770052380E704130780FA2380E70454
:102D40000100010003D7C7027D8B2396E702238091
:102D50000704D65781BDF336048093F68608B6DCA7
:102D600001000100930680FA23809D002380DD008E
:102D7000010001008356C9020566011693F6F60F9D
:102D8000D18EC206C1822316D90223800D00E656D9
:102D9000B9B793078008F3B7078093F78708BEDEBB
:102DA0000100010037170040930770052300F70466
:102DB000930780FA2300F704010001000356C702BD
:102DC00093975600B297C207C1832316F7022300D8
:102DD0000704F657C1BB914763EEB70217E701003E
:102DE000130707E58A05BA959C41BA978287B717FA
:102DF000004003A7470B1345F5FF698F23AAE70A95
:102E000003A7070B698F23A8E70A03A7070A798D91
:102E100023A0A70A8280B717004083A6470B134759
:102E2000F5FFF98E23AAD70A83A6070B558D23A891
:102E3000A70A83A6070A758F23A0E70A8280B7171F
:102E4000004003A7470B498F23AAE70A03A7070BF4
:102E50001345F5FF45BFB717004083A6470B13473F
:102E6000F5FF758F23AAE70A03A7070A598D4DB707
:102E7000B717004003A7470B498FEDB7914763EEA3
:102E8000B70217E701001307E7DB8A05BA959C41F3
:102E9000BA978287B717004003A7470D1345F5FF80
:102EA000698F23AAE70C03A7070D698F23A8E70CF6
:102EB00003A7070C798D23A0A70C8280B7170040C9
:102EC00083A6470D1347F5FFF98E23AAD70C83A6D7
:102ED000070D558D23A8A70C83A6070C758F23A07B
:102EE000E70C8280B717004003A7470D498F23AA3C
:102EF000E70C03A7070D1345F5FF45BFB7170040C3
:102F000083A6470D1347F5FF758F23AAE70C03A788
:102F1000070C598D4DB7B717004003A7470D498FD0
:102F2000EDB7797122D43714004026D24AD0035924
:102F300024028354040206D64209C2044ECE52CC67
:102F400056CA13590901C1802DE11379F9F793F499
:102F5000F49F4209C20413590901C18093078008F4
:102F6000F3B7078093F787083EC401000100930779
:102F700070052300F404930780FA2300F404010091
:102F80000100231124032310940223000404A24708
:102F9000F3A7078001000100B25022549254025955
:102FA000F249624AD24A45618280B7F507008146FC
:102FB0003000B105194597000020E7806081A247E5
:102FC00013972701E34A07FC1369090893E40440B7
:102FD00093098008F3B7098093F787083EC0010082
:102FE0000100930A700523005405130A80FA230098
:102FF000440501000100231124032310940223003F
:1030000004048247F3A7078001000100294597F0D7
:10301000FF1FE7802032F3B9098093F989084EC277
:1030200001000100230054052300440501000100B4
:103030008357040293E707202310F40223000404BB
:103040009247B9B7B7170040884742054181937747
:10305000050491EB9377F5013755E80113050580D9
:103060003345F50282809377050C130700046397BC
:10307000E7009377F50137459C1CCDB72165130513
:1030800005D0828037E700E01C435443A183E20669
:10309000D58F1CC1FD572320F7182322F7188280F3
:1030A00013178500B7E700E023A0E710618123A292
:1030B000A7108280B7F700E08847CC47828081471D
:1030C00037370040A14663C4C7003285828003457C
:1030D000B740E38EA6FE3385F5000345050085075E
:1030E0002304A740CDB797070020938727EF9C4381
:1030F000173700201307873A3E95636EE5001737B0
:103100000020130727506368A70017070020232714
:10311000A7EC3E858280FD57EDBF8280411122C41D
:1031200006C62A8497000000E78000F22947B3070B
:10313000E502B2408D83B3D7870222449507B3D707
:10314000E70237370040C207C1832316F700410169
:103150008280411137150E0006C697000000E780F7
:1031600020FCB7370040130770F82381E7000D47B4
:10317000A381E70013070004A380E7000547238726
:10318000E700B24041018280373700408347270083
:103190001A0593F7F703C98F93F7F70F2301F70089
:1031A0008280B737004003C7170019C9D98DA380A3
:1031B000B70003C70700136787002380E7008280FA
:1031C00093C5F5FFF98DA380B7008280AE872A876B
:1031D000B736004021463738004089E71703000022
:1031E0006700E3F383C8B600E30916FF05078348C9
:1031F000F7FFFD17C20723041801C183F9BF41116E
:1032000022C406C62A8497000000E780E0E329472D
:10321000B307E502B2408D83B3D7870222449507F6
:10322000B3D7E70237370040C207C1832316F74000
:1032300041018280716541111305052006C6970082
:103240000000E78000FCB7370040130770F82381C7
:10325000E7400D47A381E74013070004A380E74040
:1032600005472387E740B24041018280CC414111AC
:1032700006C6328503C6150083C5050022064D8E9D
:1032800042068D654186138875A2630C0611634B57
:10329000C804138845A26300060D634AC8009385DD
:1032A00035A26301B6082390060029464DA0138875
:1032B00055A26305060D938565A2E316B6FE8D45FE
:1032C0001D4663E6E5081146198E63F3C7003E8686
:1032D000B7E704002390C600FC4797E501009385FB
:1032E000A5989DA0138895A263030611634E060D51
:1032F0001388A5A263000613938505A5E315B6FA06
:1033000099451D4663E5E504198E63F3C7003E86C3
:10331000B7E704002390C600FC479705002093857B
:1033200025D61DA09D451D4663E3E5022146198E65
:1033300063F3C7003E86B7E70400FC472390C6004E
:10334000970500209385054BBA9582970146B240B8
:10335000328541018280AD451D46E3EAE5FE3146F6
:10336000198E63F3C7003E86B7E704002390C600BA
:10337000FC4797E501009385A591F9B7B1451D4636
:10338000E3E7E5FC3546198E63F3C7003E86B7E7F1
:1033900004002390C600FC4797E501009385459003
:1033A00065B78D451D46E3E4E5FA1146198E63F3D2
:1033B000C7003E86B7E704002390C600FC4797E5A8
:1033C00001009385258B49B78D451D46E3E1E5F85E
:1033D0001146198E63F3C7003E86B7E704002390B9
:1033E000C600FC4797E501009385458DB1BFA54513
:1033F0001D46E3EEE5F42946198E63F3C7003E86C9
:10340000B7E704002390C600FC4797E501009385C9
:1034100025871DBFB5451D46E3EBE5F23946198EFC
:1034200063F3C7003E86B7E704002390C600FC475D
:1034300097E501009385458201BFB7E7040003A328
:103440000713970600209386A6C24146A545170597
:1034500000201305E5B802832D455DE703C505008F
:103460000947631FE50803A84500411106C6034745
:10347000180032850346080022074168518F9308DF
:1034800028FE6307170563E9E800051863030703CF
:1034900023900600294591A8130648FE630AC70435
:1034A0001518E31707FF15463E87637BF60015479F
:1034B00001A8130600023E876374F600130700029A
:1034C000B7E704002390E600FC471316070111A894
:1034D0003E8691C30546B7E70400FC472390C6002B
:1034E0004206CC45418282970145B240410182802B
:1034F000130600083E87E375F6FC13070008C9B7FA
:103500002390060005458280828041677917630415
:10351000E504411122C406C685472A84639FF5004D
:10352000B7E7040022852244B24003A3871397051E
:103530000020938565464101028389476399F50020
:10354000B7E7040083A7070B8545829771D9B2407E
:103550002244410182808280797126D252CCAE848D
:103560002A8A97D501009385657717D50100130541
:10357000657906D63AC622D44AD0368432894ECEF0
:1035800097C00100E78080A6A28517D5010013052A
:10359000657897C00100E78060A5294597C00100C4
:1035A000E780A0A983C7840093F70702F9E383C9E2
:1035B00004008947054532476396F908D44083C71C
:1035C000160083C60600A207D58FC166138616FEB5
:1035D000638CC7028D16638FD7068D6693862690FF
:1035E00029456391D706B7E70400A286225403A3B6
:1035F0004714B250F2494A86A68502599254528520
:10360000624A8547456102832D450DEF930700020D
:10361000354563E98702B7E70400FC47C844130651
:103620000002CA85829781499707002093878737D0
:103630009C43014581CB9C4391C74E852286CA8518
:1036400082970145B250225492540259F249624A7B
:10365000456182802D457DF79307700F3545E3E383
:1036600087FEB7E70400FC47C8442286CA858297D4
:1036700065BF2145C1BF411122C437E4040083273F
:10368000841326C2AA84416506C697050020938547
:10369000A5307D1582978327C40A170500001305FE
:1036A00005E78588829795C0032304132244B2401E
:1036B000924497060020938626AE4146C5451705DD
:1036C00000201305659C41010283B24022449244CC
:1036D00001454101828019C59707002023A4A72C2A
:1036E00001458280454582801147636AA70A97D6C3
:1036F00001009386665D0A0536951841411106C69C
:103700003697AE87B2850287130700026145639D35
:10371000E700B7E70400FC47130600021705002086
:103720001305C50D82970145B240410182800547CE
:103730006145E39BE7FEB7E70400FC470546170534
:1037400000201305A50DF9BF1307700F6145E39D18
:10375000E7FCB7E70400FC471306700F17050020CD
:103760001305050CC1B7130700086145E39EE7FA8E
:10377000B7E70400FC4713060008170500201305EF
:10378000A5194DB715476145E390E7FAB7E704007F
:10379000FC471546170500201305452061B709456C
:1037A0008280411126C2B7E4040083A7C41322C457
:1037B0004AC006C62E84970500209385E51D2A89F8
:1037C0008297058905C5970700209387E78B83D7E4
:1037D000A70BA28503A3440D2310F4002244B2409A
:1037E00092444A850249014641010283B240224483
:1037F0009244024949454101828097070020238570
:10380000071A9707002023A3071AB717004003A73A
:10381000070CB706C0FFFD16758F23A0E70C03A7A2
:10382000070DB7064000558F23A8E70C03A7070C28
:103830003D9B23A0E70C03A7070D1367070123A8EF
:10384000E70C8280B717004003A5470C83A7470CFD
:10385000598113451500C18B058999E3136525002E
:103860009707002083C747146380A70297070020AB
:10387000238CA71211C9970700209387271303A34E
:1038800007006303030002838280114517F3FFFFE3
:10389000670063C8411193962500AA852D4506C689
:1038A00097F0FF1FE780C0F2B240014541018280DE
:1038B000011122CC06CE3714004026CA4AC84EC693
:1038C00052C483447405034AB405834984050349FB
:1038D000940597F0FFFFE780E09E8347A40593F4EB
:1038E000F40F137AFA0F93E71700230DF40493F9FA
:1038F000F90F1379F90FB717004003C7A705058B18
:103900006DFF03D5C705A38D4705238C3705A38C11
:103910002705A38B9704F2406244D2444249B2493E
:10392000224A0561828041119397050122C406C68F
:1039300026C2C1872E8463DC0700B7E40400FC5470
:10394000829719C1BC5482972165218D15A893F7E0
:10395000150013C515008DE793F725009DC7970047
:103960000000E78060EEB7E70400BC4F1306000AD2
:103970008945170500200345E50382971345240078
:10398000B24022449244410182809397250163D83A
:103990000702B7E4040083A7C41E829797000000C3
:1039A000E780E0EEBC4C3756070013060630896509
:1039B00017050020034505008297096579B793979D
:1039C00015010145E3DE07FA17D501001305853C13
:1039D00097B00100E7806079B7E70400BC4F130699
:1039E00000649165170500200345C5FC82971165A9
:1039F000A9BF2D71232A9110FD74E98C232C81100D
:103A000023282111232631112A84AE893289930675
:103A100000100A86A6852D45232E111097F0FF1F52
:103A2000E78000DB13154401B7E70400FC47518130
:103A30000A0513962900CA850A958297A685856688
:103A40000146254597F0FF1FE78080D80A86A685A6
:103A500093060010294597F0FF1FE78060D7832069
:103A6000C1110324811183244111032901118329E8
:103A7000C11015618280B7F7070003C70701411124
:103A800006C622C426C24AC0A547631DF700970098
:103A90000000E78040F6B2402244924402490145CA
:103AA0004101828013942500AA843289A286AA85C6
:103AB0000146254597F0FF1FE78080D1A2864A8600
:103AC000A685294597F0FF1FE78080D0E9B71D71D3
:103AD000A2CC37E404005C5C485886CE494697D5B2
:103AE00001009385A526829711E917D501001305DA
:103AF000252797B00100E780406701A0B7F600E0F6
:103B0000795798CAFD57DCCA0567B7E700E023A0DC
:103B1000E7101306F00290C223A0E718010001008D
:103B20003707002018471306000481459706002038
:103B300023A0E6E84157A38AE7403C44080882975F
:103B400097170020938707843EC88567138707402F
:103B5000231AE1001D673ACC370701051307071048
:103B60003ACE938757D11307B00F2310E1022312E7
:103B7000F102054797F7FFFF938707542301E102FE
:103B80003ED817070000130727D197070000938737
:103B900067D2B7F50700BAC23EDC1707000013076B
:103BA000C7ED97070000938787CE81463000E10577
:103BB0001945BAC43EDE97F0FF1FE78060C11808C0
:103BC0008147994630003E96034606008507050763
:103BD000A30BC700E398D7FEC24791C70357410123
:103BE00085676373F70001A0B7E7040083A7470A5E
:103BF00008088297AA8511C917D5010013058517F2
:103C000097B00100E780803E01A0F6406644256140
:103C10008280411126C2B7E4040083A7040806C6C7
:103C200022C417050000130545D082971704002011
:103C3000130444D82300A40097000000E78080020A
:103C400097000000E780A0BB03450400224403A3C3
:103C50008405B24092441306003289654101028313
:103C6000797106D622D413078008F337078093F7BB
:103C700087083EC201000100B71700409305700598
:103C80002380B704130680FA2380C70401000100D3
:103C900083C6F70293F6A60FA387D70223800704F3
:103CA0009246F3A606800100010073370780137760
:103CB00087083AC4010001002380B7042380C704A9
:103CC0000100010003C7F70213672700A387E7027B
:103CD00023800704A247F3A70780010001000545E0
:103CE00097E0FFFFE780406197000000E78020BA7F
:103CF000014781468147054685451305407E97E08B
:103D0000FFFFE780406437E404003C44680051460C
:103D100081458297B707C0A83EC8B787E803938755
:103D200007D03ECA97E7FF1F938767693EC67C5856
:103D300068008297B250225445618280411197D524
:103D400001009385256D17D501001305A5FB06C657
:103D500097B00100E780802917E50100130545862B
:103D600097B00100E7808028B2402945410117B390
:103D700001006700832C411197D501009385C56A26
:103D800017D50100130505F806C697B00100E780B6
:103D9000E02517E501001305658197B00100E78074
:103DA000E024B2402945410117B301006700E32830
:103DB000411122C406C6834705002A849DC797D5B2
:103DC00001009385256C17D501001305A5F397B065
:103DD0000100E780A0214C4017E501001305858C08
:103DE00097B00100E78080203DA058410DEF97D5A6
:103DF00001009385256917D501001305A5F097B03B
:103E00000100E780A01E17E501001305258B97B080
:103E10000100E780A01D2244B2402945410117B3AB
:103E2000010067008321A1679386D7036313D7023C
:103E300097D501009385056517D50100130585EC1D
:103E400097B00100E780801A17E501001305058887
:103E50007DBFED0797D501009385C56217D5010099
:103E6000130545EA631BF70097B00100E7800018CF
:103E700017E501001305C58659BF97B00100E7801B
:103E8000E0164C4017E501001305858791BF4111ED
:103E900097D501009385855A17D50100130585E64E
:103EA00006C697B00100E7806014B2402945410181
:103EB00017B3010067006318797122D426D24AD063
:103EC0002E842A898145B2844800714606D697E03F
:103ED000FFFFE780C02297F7FF1F9387A74CDC47BF
:103EE00083D70700231421012313F100975000000A
:103EF000E78020309547A305F1009307401F3EC699
:103F0000FD572305A100230AF10097500000E78028
:103F100080422686A285480097500000E780403006
:103F2000B250225492540259456182809727002052
:103F3000239D07949727002023860784B7E7040072
:103F4000BC47411106C641468145170500201305AF
:103F5000A531829797200000E780807197200000AC
:103F6000E7808052014597600000E78060BD170739
:103F70000020034767319307F00A6315F7029307A0
:103F8000F0F88945170500201305053017070020B4
:103F9000230CF72E97070020A388072E97600000B8
:103FA000E780A0E497600000E780001181453705B5
:103FB00004009707002023A7072A970700202391D2
:103FC000072A97070020238E072897070020239FA2
:103FD000072097070020239D071E970700202390A6
:103FE0000728970700202399072897300000E780CB
:103FF0002073014597600000E78020E897D5010015
:104000009385454617D501001305C5CF97B001002C
:10401000E780C0FD17D501001305C57497B00100F6
:10402000E780C0FCB2402945410117B30100670099
:10403000C300411122C406C626C293F715002E8480
:10404000638F0710814617F6FF1F1306E63285457A
:10405000170500200355851797C00000E780C06A48
:1040600015C997D501009385A54017D50100130503
:1040700065C997B00100E78060F717D50100130507
:10408000E5E197B00100E78060F6294597B00100AF
:10409000E780A0FA97D501009385853D17D50100EB
:1040A000130545C697B00100E78040F417D501001D
:1040B000130505E097B00100E78040F3294597B06C
:1040C0000100E78080F717F5FF1F1305A52D5C455C
:1040D00005472390E70097400100E780401B97D5F4
:1040E00001009385E53817D501001305A5C197B0E8
:1040F0000100E780A0EF17D501001305A5DC97B0FC
:104100000100E780A0EE294597B00100E780E0F2CA
:10411000930710F8170700202308F71697070020C9
:1041200083D7870A17070020A300F716170500207A
:1041300013058515A1839145170700202307F71460
:1041400097070020A383071497600000E780E0C969
:1041500013451400B240224492444101828093F7F7
:104160002500E1C3170700200357870F45CB9706AB
:1041700000209386260F944297D70100938787608B
:10418000170600200346E60D81451705002013059C
:10419000A50D97700000E7808076AA8441C197D56D
:1041A00001009385A53517D501001305A5B597B076
:1041B0000100E780A0E3A68517D50100130505D20D
:1041C00097B00100E78080E2294597B00100E780C1
:1041D000C0E69707002023950708930710F81707F4
:1041E00000202303F70A9707002083D7E7FD17076E
:1041F0000020A30BF708A183170700202307F70867
:1042000091458D4717050020130505081707002065
:10421000A30DF70697600000E78020BD134524003A
:1042200015BF93F74500D1C397D501009385052DA0
:1042300017D50100130505AD97B00100E78000DB3D
:1042400017D50100130545CB97B00100E78000DAD0
:10425000294597B00100E78040DE930720F8170753
:1042600000202303F7029707002083D727F81707BA
:104270000020A30BF700A183170700202307F700F6
:10428000854717070020A302F70097500000E7803A
:10429000800A17050020130525FF9145976000004F
:1042A000E780A0B41345440075B593F78500A9C70E
:1042B00097D501009385852417D50100130585A4A2
:1042C00097B00100E78080D217D50100130505C41F
:1042D00097B00100E78080D1294597B00100E780C1
:1042E000C0D597070020239D07F697700000E78050
:1042F000E07013458400B9BD93F70501D1C385452E
:1043000017050020035585EE97600100E780002324
:1043100097D501009385851E17D501001305859E4D
:1043200097B00100E78080CC17D50100130545BF89
:1043300097B00100E78080CB294597B00100E78066
:10434000C0CF930730F817070020230FF7F2970725
:10435000002083D7A7E917070020A307F7F2170566
:104360000020130565F2A1838D4517070020230E59
:10437000F7F097600000E78040A713450401D9BB20
:1043800093F70502D1C797D501009385251717D557
:1043900001001305259797B00100E78020C517D5C8
:1043A0000100130525BA97B00100E78020C4294514
:1043B00097B00100E78060C8930740F81707002016
:1043C0002304F7EC9707002083D787E01707002026
:1043D000A30CF7EAA183170700202308F7EA854713
:1043E00017070020A303F7EA97070020239207DEB0
:1043F00097500000E78020F4170500201305C5E85A
:10440000914597600000E780409E1345040299B3F0
:1044100093F70504FDC397D501009385250E17D5A5
:1044200001001305258E97B00100E78020BC17D549
:1044300001001305A5B297B00100E78020BB294514
:1044400097B00100E78060BF9707002083C7C7E3EC
:104450001307700A6386E7061307800A638CE70870
:104460001307600A6393E704930760F817070020B7
:10447000230CF7E09707002083D767DE170700209B
:10448000A304F7E0A183170700202300F7E0854786
:1044900017070020A30FF7DEB1451705002013050D
:1044A000A5DE97600000E780409497500000E78009
:1044B00080E81345040497070020239207DA59B9CE
:1044C000930770F8170700202300F7DC97070020F8
:1044D00083D7E7D817070020A308F7DAA1831707C7
:1044E00000202304F7DA854717070020A300F7DA36
:1044F000994565B7930780F8F1B793F7050801452B
:10450000E38A07C497D50100938545FF17C50100CD
:104510001305457F97B00100E78040AD17D5010036
:10452000130545A597B00100E78040AC294597B039
:104530000100E78080B09307A0F81707002023054B
:10454000F7D49707002083D727D317070020A30DA0
:10455000F7D2A183170700202309F7D28547170751
:104560000020A304F7D297070020239707D0975085
:104570000000E78040DC170500201305E5D09145D9
:1045800097600000E780608613450408E1B641119A
:1045900022C497D50100938525F02A8417C5010010
:1045A0001305457606C697B00100E78020A44C406D
:1045B00017D501001305850C97B00100E78000A313
:1045C000294597B00100E78040A7034704009307FF
:1045D000F00F631FF70297D501009385E5EB17C530
:1045E00001001305257297B00100E78020A04C4020
:1045F00017D501001305850997B00100E780009FDA
:104600002244B2402945410117B301006700E3A2EB
:10461000B240224441018280B1C1411122C417C578
:1046200001001305256E2E8497D501009385C5E101
:1046300006C697B00100E780609BA28517D50100F0
:104640001305051097B00100E780409A2244B2405C
:104650002945410117B301006700239E8280411163
:1046600022C426C22E84AA8497D50100938585DEB4
:1046700017C501001305056906C697B00100E7805C
:10468000E09617D501001305650C97B00100E7808F
:10469000E095294597B00100E780209A97D5010061
:1046A000938545DB97070020239297B217C5010039
:1046B00013054565854497070020239787B0970722
:1046C0000020239497B0971700202390871C97B061
:1046D0000100E780A0919715002083D5051B17D511
:1046E00001001305250797B00100E78020902945B8
:1046F00097B00100E7806094971700202384970803
:1047000097200000E78040D8228597500000E7807E
:104710002043054597500000E780207697F7FF1F5C
:10472000938747C8DC4703D70700C167FD176312AB
:10473000F7022244B7E70400B240924403A387057E
:1047400017F5FF1F034585271306000A854541011C
:104750000283B2402244924441018280011122CC62
:1047600037E404005C5C06CE354697D5010093859E
:1047700065E617E501001305A5CE829711E917C577
:1047800001001305E55D97B00100E780009E01A0E0
:1047900097F7FF1F938747233EC4B7F50700856748
:1047A00093870780814617F6FF1F13066621E105F0
:1047B00019453EC697E0FF1FE78080017C441946FB
:1047C00097F5FF1F9385C51F17050020130545A208
:1047D0008297340017F6FF1F1306861E97D5010037
:1047E0009385853017D5010013058531977000003A
:1047F000E780E0E52A841DCD97D50100938505CD9E
:1048000017C501001305055097A00100E780007E41
:10481000A28517D501001305E5DC97A00100E7800C
:10482000E07C294597B00100E7802081F240624496
:104830000561828097E00000E780404817D50100BD
:10484000130545D197600000E78020DA97B000009B
:10485000E780809C97600100E780000117F5FF1F4B
:104860001305C5B097600100E780A0E917D50100E6
:10487000130545CF97600100E78080012A84976087
:104880000000E780604097100100E780E0D8978043
:104890000100E780007297800000E780A098977081
:1048A0000000E78060B697400100E780409A97D506
:1048B00001009385A5C117C501001305A54419C8BA
:1048C00097A00100E7808072A28517D5010013052B
:1048D000A5D3A1B797A00100E780407117D50100CB
:1048E0001305C5D497A00100E7804070294597A023
:1048F0000100E780807497300100E7802076970000
:104900000100E780E09455C98545370504009730DC
:104910000000E780E0E097D50100938525BB17C52F
:1049200001001305253E97A00100E780206C17D5F4
:104930000100130525D197A00100E780206B2945D0
:1049400097A00100E780606F97F7FF1F9387479557
:1049500083D70700171700202319F7F28547171789
:1049600000202301F7E297200000E780E0CA9720AB
:104970000000E78060B117150020035505F197503E
:104980000000E780E01B054597500000E780E04EFF
:1049900097D50100938585B317C5010013058536AA
:1049A00097A00100E780806417D501001305C5CBEF
:1049B00097A00100E7808063ADB597D5010093858E
:1049C000E5B017C501001305E53397A00100E780A6
:1049D000E06117D501001305E5D897A00100E78035
:1049E000E060294597A00100E7802065014569BF87
:1049F000411122C437E404008327041A06C68297B3
:104A000097500000E78080178327040817F5FFFF01
:104A100013056562829797F7FF1F2381A7FA17F5A1
:104A2000FF1F1305259897500000E78060C32244BC
:104A3000B240410117030000670083D2411106C64E
:104A400022C426C299C1AA8415ED97D50100938589
:104A5000E5A817C501001305E52A97A00100E78026
:104A6000E05817C501001305A54197A00100E78094
:104A7000E0572244B24092442945410117A3010066
:104A80006700A35B37E404007C44414617F5FF1F31
:104A90001305857D829717F5FF1F1305E57C972089
:104AA0000000E78080B097200000E780E09D0323AE
:104AB0008405224497F7FF1F2394977AB2409244CB
:104AC00017F5FF1F034585EF1306000A89454101CD
:104AD0000283B7E70400FC471171A2DDCAD986DF63
:104AE000A6DBCED72E8432892E86AA8517F5FF1F26
:104AF00013058579829717F7FF1F1307E778834718
:104B00000700930680029387E70793F7F70FE3EC1C
:104B1000F610BA898A0717C701001307E727BA9763
:104B20009C43BA9782878D4797D501009385459E10
:104B300017C501001305051D630FF40097A00100C0
:104B4000E780C04A17C501001305455997A0010029
:104B5000E780C049BDA497A00100E780204917C5A0
:104B600001001305255997A00100E7802048294539
:104B700097A00100E780604C930720F8114697F555
:104B8000FF1F938565704A8517F7FF1F230EF76E89
:104B900097F7FF1FA38B076E97F0FFFFE7800032A8
:104BA0002A841DC997D501009385859617C50100F4
:104BB0001305451597A00100E7804043A28517C55E
:104BC00001001305E55697A00100E7802042294522
:104BD00097A00100E780604697D501009385459333
:104BE00017C501001305051297A00100E7800040DA
:104BF00017C501001305055597A00100E780003F88
:104C0000294597A00100E78040434165930730FAAA
:104C1000054697F5FF1F938525677D1517F7FF1F3D
:104C20002304F76697F0FFFFE78040292A841DC917
:104C300097D501009385C58D17C501001305850C17
:104C400097A00100E780803AA28517C501001305EF
:104C5000254E97A00100E7806039294597A0010003
:104C6000E780A03DB7E70400BC4F0566130606C801
:104C7000A14517F5FF1F034565D48297FE506E547A
:104C8000DE544E59BE591161828091476303F4028C
:104C900097D501009385C58717C5010013058506C3
:104CA00097A00100E780803417C501001305C54CAB
:104CB00071BDB7E70400FC4F914517F5FF1F034591
:104CC000E5CF829797D501009385858417C50100AC
:104CD0001305450397A00100E780403117C5010087
:104CE0001305454B97A00100E7804030294597A068
:104CF0000100E780803497400000E780C063914561
:104D000035A485476303F40297D501009385458058
:104D100017C50100130505FF97A00100E780002DCE
:104D200017C501001305854815B597F7FF1F239F89
:104D3000274BB7E704000566BC4F130606C8C145FC
:104D40000DBF8D476303F40297C501009385457C31
:104D500017C50100130505FB97A00100E780002996
:104D600017C5010013054546D5B3930740F8114612
:104D700097F5FF1F938545514A8517F7FF1F2305B8
:104D8000F75097F7FF1FA382075097F0FFFFE780C8
:104D9000E0122A84E30405EE97C501009385457768
:104DA00017C50100130505F697A00100E780002450
:104DB000A28517C501001305A53797A00100E7805C
:104DC000E022294597A00100E780202745BD9147B3
:104DD000E31CF4F6B7E70400FC4F9305000217F557
:104DE000FF1F0345A5BD829797C5010093854572B6
:104DF00017C50100130505F197A00100E780001F0A
:104E000017C501001305C53DF1BD894763E387025E
:104E100097C501009385C56F17C50100130585EE81
:104E200097A00100E780801C17C501001305853C91
:104E300031BB97F4FF1F83C4444597F7FF1F83C717
:104E4000B74497C501009385A56CA20417C501005E
:104E5000130545EBDD8C97A00100E7802019A285A2
:104E600017C501001305453A97A00100E780001817
:104E7000C204294597A00100E780201CC184930546
:104E8000D4FF93960401C1824A8693F5F50F17F576
:104E9000FF1F1305953F97300000E780208CE35FEC
:104EA00090DC930750F817F7FF1F230FF73C83C7D9
:104EB0003900228697F5FF1F9385053D85074A85B2
:104EC00017F7FF1FA303F73C97F0FFFFE78000FFF2
:104ED0002A84E30505DA97C501009385656317C544
:104EE0000100130525E297A00100E7802010A285AC
:104EF00017D501001305C583C9B5894763E3870248
:104F000097C501009385C56017C50100130585DFAE
:104F100097A00100E780800D17C5010013058530BB
:104F200035B197400000E7800041A28517F5FF1FCB
:104F30001305853597500000E78020EB81B38D473E
:104F40006303F40297C501009385855C17C50100D2
:104F5000130545DB97A00100E780400917C5010054
:104F60001305052EE5B6B76602000146B7750200C7
:104F7000054597E0FF1FE780A085930760F817F7C6
:104F8000FF1F2303F73097F7FF1FA3800730930716
:104F9000000617F7FF1F230BF72E894717F7FF1F90
:104FA000A306F72E97F7FF1F2383072E97F7FF1F00
:104FB000A38F072CC14717F7FF1F230BF72C93076D
:104FC00020F917F7FF1FA305F72C314697F7FF1FAE
:104FD000A381A72C97F5FF1F9385052B4A8597F78B
:104FE000FF1F2388072A97F0FFFFE78020ED2A8420
:104FF000E30605C897C501009385855117C50100D3
:10500000130545D097A00100E78040FEA28517C593
:1050100001001305652455B3B1476303F40297C536
:1050200001009385E54E17C501001305A5CD97A096
:105030000100E780A0FB17C501001305A52339B6C1
:10504000B7E70400FC4F9305000417F5FF1F034565
:10505000E596829797400000E780E02DB145F9B5CD
:10506000914763E3870297C501009385654A17C599
:105070000100130525C997A00100E78020F717C597
:1050800001001305E520D9B497F4FF1F83C4042061
:1050900097F7FF1F83C7771FA204DD8C8E04B777B5
:1050A00002006D14BE942286A68517C50100130563
:1050B000651F97A00100E78060F3B7E70400FC4795
:1050C000228697F5FF1F9385751C280082979316FB
:1050D0000401C1823000A685094597D0FF1FE780F3
:1050E000206F2A8409C917C501001305651D97A003
:1050F0000100E7808007930770F8194697F5FF1FB6
:10510000938585184A8517F7FF1F230FF71697F722
:10511000FF1FA38D871697F0FFFFE78020DA2A8410
:10512000E30E05B497C501009385853E17C50100C0
:10513000130545BD97A00100E78040EBA28517C588
:1051400001001305E51895B99947630BF41297C54B
:1051500001009385E53B17C501001305A5BA97A08B
:105160000100E780A0E817C501001305E517F9BAAB
:10517000914763E3870297C501009385653917C599
:105180000100130525B897A00100E78020E617C5A8
:1051900001001305E5165DBA97F4FF1F83C4040FE1
:1051A00097F7FF1F83C7770EA204DD8C8E04B777B5
:1051B00002006D14BE942286A68517C50100130552
:1051C000651597A00100E78060E2B7E70400FC479F
:1051D000228697F5FF1F9385750B280082979316FB
:1051E0000401C1823000A6850D4597D0FF1FE780DE
:1051F000205E2A8409C917C501001305651397A00D
:105200000100E78080F6930780F8194697F5FF1FA5
:10521000938585074A8517F7FF1F2307F70697F73A
:10522000FF1FA385870697F0FFFFE78020C92A8428
:10523000E30605A497C501009385852D17C50100D8
:10524000130545AC97A00100E78040DAA28517C599
:1052500001001305250F95B699476303F40297C51E
:1052600001009385E52A17C501001305A5A997A09C
:105270000100E780A0D717C501001305250EF9B07E
:10528000B7E70400FC4F9305000417E5FF1F034533
:10529000E572829797400000E780E009994579B16F
:1052A0008D476303F40297C501009385652617C5F2
:1052B0000100130525A597A00100E78020D317C59D
:1052C00001001305250B59B017C501001305850B07
:1052D00097A00100E78060E91305C01297D0FF1F77
:1052E000E7802006014597E0FFFFE780E0D90D4504
:1052F00097100000E780E0A3294597D0FF1FE780C3
:10530000400497D0FF1FE780A0F48DBA994763034C
:10531000F40297C501009385A51F17C50100130569
:10532000659E97A00100E78060CC17C501001305BA
:10533000250629B817F7FF1F034757F597F7FF1FF3
:1053400083C7C7F422075D8F9166BA96C2061166BD
:10535000C1821306F6EF8D476365D60297E7FF1FFC
:10536000938747049C4B17F6FF1F034616F293865C
:10537000C7002DC203D6070069CA8907E39CD7FE80
:1053800089471307A0F8114697F5FF1F9385C5EFCE
:105390004A8597F6FF1F2389E6EE17F7FF1FA3063E
:1053A000F7EE97F0FFFFE78060B12A84E308058CF1
:1053B00097C501009385C51517C501001305859490
:1053C00097A00100E78080C2A28517C501001305E0
:1053D00065FDE5B203D60700630EE60A8907E39B85
:1053E000F6FE8D4779BF91476304F40297C501002B
:1053F0009385051217C501001305C59097A00100FC
:10540000E780C0BE17C50100130545FB6FF00FF420
:10541000B7E70400FC4F9305000817E5FF1F03459D
:10542000E5598297C9B897C501009385650E17C5E0
:1054300001001305258D97A00100E78020BB17C54B
:105440000100130525F96FF06FF02390E70017E5D1
:10545000FF1F130525F597300100E780A0E597C5EC
:1054600001009385E50A17C501001305A58997A0DA
:105470000100E780A0B717C501001305A5F697A0A6
:105480000100E780A0B6294597A00100E780E0BAB7
:105490008147C5BD2390070017E5FF1F130585F061
:1054A00097300100E78000E197C50100938545062C
:1054B00017C501001305058597A00100E78000B31B
:1054C00017C50100130585F35DBF411122C406C64F
:1054D00026C24AC0834705002A84A1C397C501009C
:1054E0009385C5FC17C501001305C58197A0010070
:1054F000E780C0AF4C4017C501001305A52997A050
:105500000100E780A0AE2244B240924402492945FE
:10551000410117A30100670043B25841B707CF000C
:105520009387777D631CF70804456385041203594C
:10553000C500630109120354E50097C50100938576
:10554000E5F617B501001305E57B97A00100E7809C
:10555000E0A903C60400A286CA8517C50100130589
:10556000E52497A00100E78060A8294597A00100E5
:10557000E780A0AC4A86A685228597200000E780B8
:1055800000F783C7140003C70400A207D98F13973D
:105590008700A183D98FC2073167C1831307C7551D
:1055A000638AE70A22862244B240CA8526850249D8
:1055B0009244410117F3FFFF6700E351B707CC00A6
:1055C0009387777D6310F70697C50100938505EEF5
:1055D00017B501001305057397A00100E78000A12E
:1055E0001C448355C4008356E40003C6070017C556
:1055F00001001305A51B97A00100E780209F294506
:1056000097A00100E78060A30356C4000C44035533
:10561000E4002244B24092440249410117230000B1
:105620006700E3ECB707CE009387777D6304F7024A
:1056300097C50100938585E717B501001305856CB3
:1056400097A00100E780809A4C4017C50100130520
:10565000250B75B5B2402244924402494101828033
:10566000B7E70400FC4741112E8606C622C426C2B5
:105670004AC02E842A89AA8517F5FF1F1305C5C0C5
:10568000829797C50100938565EA17B50100130558
:10569000656797A00100E780609597F5FF1F83C5B8
:1056A000A5BE17C501001305658E97A00100E78010
:1056B000E093294597A00100E780209897F4FF1F09
:1056C000938484BC83C7040041479387070693F7FC
:1056D000F70F636AF75C17B70100130727768A078D
:1056E000BA979C43BA9782879D476307F40297C590
:1056F00001009385A5E317B501001305A56097A0E8
:105700000100E780A08E17C501001305A58897A0AA
:105710000100E780A08DADAC97F7FF1F83C7D7B618
:10572000DDCB17F7FF1F034757B697F7FF1F83C758
:10573000C7B522075D8F97F7FF1F83C727B5C2073D
:105740005D8F97F7FF1F83C777B4E207D98F17F7ED
:10575000FF1F2329F7B083C7640097C50100938515
:10576000E5DC17B501001305E55917F7FF1F230AFC
:10577000F7AE97A00100E780608797F7FF1F938738
:1057800067AE8C4317F6FF1F0346A6AD17C5010091
:105790001305058297A00100E7804085294597A061
:1057A0000100E780808997F7FF1FA38F07AC224491
:1057B000B24092440249930700F817F7FF1F2305F0
:1057C000F7AC9D4517F5FF1F130505AC41011743C5
:1057D00000006700836197600000E780A03197F7C1
:1057E000FF1F2384A7AA9357850017F7FF1FA30E57
:1057F000F7A8935705012A8417F7FF1F2308F7A876
:1058000093578501014517F7FF1FA301F7A897607C
:105810000000E780E02E97F7FF1F238AA7A697C511
:1058200001009385A5D017B501001305A54D9790EC
:105830000100E780A07B17F6FF1F034646A5A2855F
:1058400017B5010013054578B1B7CD476303F402DE
:1058500097C50100938585CD17B501001305854ACD
:1058600097900100E780807817B501001305457710
:1058700079BD37E404007C44414697F5FF1F9385CA
:10588000B5A017F5FF1F1305259E829717F5FF1F7B
:105890001305859D97100000E78020D19710000028
:1058A000E78080BE97F7FF1F83C7279F17F7FF1F6B
:1058B0000347979EA20703238405D98F17F7FF1F7D
:1058C0002310F79A1306000A89452244B2409244F5
:1058D000024917E5FF1F0345650E410102838D470D
:1058E0006303F40297C50100938545C417B5010011
:1058F0001305454197900100E780406F17B50100FF
:105900001305C57D29B517F4FF1F0344049897F7C5
:10591000FF1F83C7779797C50100938525C1220490
:1059200017B501001305053E5D8C97900100E780D7
:10593000E06BA28517B501001305056C9790010077
:10594000E780C06A294597900100E780006F0D4607
:1059500097F5FF1F93854593228597E0FFFFE7802A
:10596000E055AA8421C197C50100938525BC17B5D0
:1059700001001305253997900100E7802067A6856F
:1059800017B501001305856897900100E780006650
:105990002244B24092440249294541011793010033
:1059A0006700A36997F7FF1F23928784B7E7040076
:1059B000116603A38705130606E8914539B78D479D
:1059C0006303F40297C50100938545B617B501003E
:1059D0001305453397900100E780406117B501003A
:1059E0001305857E2DB317F4FF1F0344048A97F730
:1059F000FF1F83C7778997C50100938525B32204CC
:105A000017B50100130505305D8C97900100E78004
:105A1000E05DA28517B50100130585609790010030
:105A2000E780C05C294597900100E78000610D4642
:105A300097F5FF1F93854585228597E0FFFFE78057
:105A4000E047AA841DC197C50100938525AE17B50F
:105A500001001305252B97900100E7802059A685AA
:105A600017B501001305055D05B797E7FF1F2391E3
:105A70008776B7E70400116603A38705130606E8D7
:105A80009305000299B5894763E3870297C5010032
:105A90009385C5A917B501001305C5269790010088
:105AA000E780C05417B501001305C5748DB197E4A4
:105AB000FF1F83C4847D97E7FF1F83C7F77C97C5CB
:105AC00001009385A5A6A20417B50100130585233F
:105AD000DD8C97900100E7806051A68517B5010025
:105AE0001305C55697900100E780405029459790CF
:105AF0000100E7808054228697E5FF1F9385C578D3
:105B0000268597E0FFFFE780603B2A84630E051A35
:105B100097C50100938585A117B501001305851E62
:105B200097900100E780804CA28517B5010013050E
:105B3000255399BD854763F9871883451900224489
:105B4000B24092440249B335B00097E7FF1F238962
:105B5000B76A17B501001305E5514101179301001C
:105B60006700C348A2852244B24092444A85024954
:105B70004101170300006700032299476303F40201
:105B800097C501009385859A17B501001305851700
:105B900097900100E780804517B501001305457F08
:105BA000BDB617E4FF1F0344446E97E7FF1F83C78A
:105BB000B76D97C5010093856597220417B501005D
:105BC000130545145D8C97900100E7802042A28563
:105BD00017B501001305854B97900100E780004140
:105BE000294597900100E7804045194697E5FF1F3A
:105BF00093858569228597E0FFFFE780202CAA84A2
:105C00001DC197C501009385659217B50100130565
:105C1000650F97900100E780603DA68517B50100EC
:105C20001305C54795B397E7FF1F23978764B7E729
:105C30000400116603A38705130606E89305000810
:105C400069B1854797C501009385458E17B5010059
:105C50001305450B630BF40097900100E7800039B2
:105C600017B501001305C5445DB497900100E780A6
:105C7000E03717B501001305254597900100E7802F
:105C8000E036294597900100E780203B2244B2404E
:105C90009244024997E7FF1F2394075C4101176371
:105CA00000006700A3D597C501009385258817B527
:105CB00001001305250597900100E780203317B5F3
:105CC000010013052571A1B4B24022449244024957
:105CD00041018280411106C622C497E0FFFFE780A0
:105CE000E01D9377F50FA1C32A8497C50100938522
:105CF000658517B501001305E50097900100E78061
:105D0000E02E9375F40F17C50100130565A2979057
:105D10000100E780A02D2244B2402945410117939C
:105D2000010067008331B240224441018280411169
:105D300022C491462A8417E6FF1F130626639D6539
:105D40002D4506C697D0FF1FE78080A8B7F707004C
:105D500003C70701A5476313F70001A093060010CE
:105D600001469D65254597D0FF1FE78060A697E710
:105D7000FF1F238D875E2244B240914617E6FF1F26
:105D80001306C65E9D652945410117D3FF1F6700B5
:105D900023A41171CED7B7E9040083A7C904CAD9D7
:105DA00017E9FF1F1309494EA2DD2E8686DFA6DB09
:105DB0002E84AA854A85829797E7FF1F83C7C74C21
:105DC0001307700A6385E710636DF7001307600A15
:105DD0006385E704FE506E54DE544E59BE5911617E
:105DE00082801307800A6385E7161307900AE393FE
:105DF000E7FE8D476306F41C97C50100938585A6D1
:105E000017B50100130505F097900100E780001E0B
:105E100017C50100130545A225A08D47630CF402A8
:105E200097C50100938505A417B50100130585EDFD
:105E300097900100E780801B17C5010013050599A5
:105E400097900100E780801A294597900100E7802C
:105E5000C01E49B7854717C501001305E59817E728
:105E6000FF1F230FF73897900100E7800030B775C8
:105E70000200B76602000146054597D0FF1FE78084
:105E80002095930760F817E7FF1F230FF73E97E76A
:105E9000FF1FA38C073E9307002617E7FF1F23274A
:105EA000F73EE5779387072117E7FF1F2312F73E99
:105EB000B14597E7FF1F238E073C97E7FF1FA38A93
:105EC000A73C4A8597000000E780401621B791471C
:105ED00063E3870297C501009385C59817B5010054
:105EE000130545E297900100E780401017C50100B7
:105EF00013058591B1B797E4FF1F83C4243997E751
:105F0000FF1F83C79738A204DD8C83A7C9046D14D3
:105F1000228697E5FF1F93857537280082978E04A8
:105F200093160401B7750200C1823000A695094599
:105F300097D0FF1FE780C089930770F817E7FF1F0E
:105F40002304F734994597E7FF1FA381A73495BF32
:105F5000914763E3870297C501009385A59017B524
:105F60000100130525DA97900100E780200817C586
:105F700001001305E58AE9B597E4FF1F83C40431E6
:105F800097E7FF1F83C77730A204DD8C83A7C9047E
:105F90006D14228697E5FF1F9385552F2800829761
:105FA0008E0493160401B7750200C1823000A695D5
:105FB0000D4597D0FF1FE780A081930780F8BDBFF4
:105FC00017C501001305858897900100E780E01947
:105FD000930790F82304F100834719008D452800AA
:105FE000A304F100834729002305F1009700000076
:105FF000E780C0031305C01297C0FF1FE78060341D
:10600000014597D0FFFFE78020080D45970000006D
:10601000E78020D2294597C0FF1FE780803297C0D4
:10602000FF1FE780E0227DB397E7FF1F93870735C7
:1060300003A3070063030300028317430000670004
:10604000C3DA41114AC09706002083D606843289FC
:1060500017D6FF1F0356263722C426C206C62A8437
:10606000AE8497000000E780806835C12DC0994755
:1060700063FF97048347140003470400A207D98FE6
:1060800013978700A183D98FC2073167C183130794
:10609000C755639EE70297D7FF1F83D7C732A30177
:1060A000F400A1832302F40097F7FF1F83D7E77D55
:1060B00091C7A302F400A1832303F400A68517B5BA
:1060C00001001305257E97900100E78020F297F7E5
:1060D000FF1F83C7276BB9CF97D5FF1F83D5A52E89
:1060E00017B501001305C57D97900100E78000F00A
:1060F0002686A28517D5FF1F0355E52C97000000C3
:10610000E78080BD6301090497E7FF1F83C7472726
:106110009DCB95C897E7FF1F83C7870E8DE7228524
:106120002244B2400249A68592444101174300002F
:106130006700A3CB17B5010013058579979001007F
:10614000E780A002C1B7B240224492440249410113
:106150008280011126CA06CE22CC03445500834713
:106160004500AA8422045D8C2EC617B501001305D4
:106170002572A28597900100E78040E7228562445E
:106180003246F240A685D24405611703000067003D
:10619000A3B4011122CC2A8417B501001305456E62
:1061A00006CE2EC697900100E78020FC228562442F
:1061B000B245F2400561171300006700A3418D4707
:1061C00063FBB70A011126CA06CE22CC0344350070
:1061D00097E4FF1F83C4D41A97B501009385057017
:1061E000B337800017E7FF1FA30CF71809C497B552
:1061F00001009385656F17B501001305656F9790D2
:106200000100E780A0DE97E7FF1F83C7771763864B
:10621000970097000000E780402B97E7FF1F83C798
:1062200037168DC785472306F100B7E7040083A71B
:1062300047177000854513055030829717B5010048
:106240001305056C97900100E78020F2996793870A
:1062500057EE2316F100680085479145A30781009A
:106260002307F10097000000E78040DCF240624421
:10627000D244056182808280894763F7B7080111A3
:1062800022CC06CE26CA8344250085472A84639DF6
:10629000F404914763F5B704034545008347340090
:1062A00022055D8D97D7FF1F239FA7109700000041
:1062B000E780C04C9967938767EE2314F10083470A
:1062C000340023059100A305F10083474400954560
:1062D00028002306F10097000000E78020D5F24057
:1062E0006244D24405618280FDF89967938767EE26
:1062F0002314F10097D7FF1F83D7E70CA305F10004
:1063000023050100A183E1B782800111996722CCA6
:10631000D51717F4FF1F1304E4462314F100834735
:10632000040026CA97F4FF1F938424562305F10026
:1063300083D7040028009545A305F100A18306CE6C
:106340002306F10097000000E78040CE03D604004A
:106350008345040017B501001305055C9790010003
:10636000E780C0C8F2406244D244056182809D67E4
:106370007971D9172316F10097F7FF1F83C787405C
:1063800006D62307F100A9C3B7E70400FC4741463E
:1063900097E5FF1F938545ED1305F100829768008F
:1063A000CD4597000000E78060C897F5FF1F83C5C3
:1063B000653D17B501001305255997900100E78049
:1063C000E0C2B25045618280B7E70400BC47414655
:1063D00081451305F1008297D9B745C5411106C61D
:1063E00022C4930750FA2300F5009307A005A300E9
:1063F000F50089472301F5009147A301F5009307B4
:10640000B002A302F50097F7FF1F9387A73783C752
:106410000700230205002A842303F50097E7FF1FE6
:10642000938717F683C70700414697E5FF1F9385BB
:10643000A5E3A303F50097F7FF1F83D707452304C0
:10644000F500A183A304F50097D7FF1F83D7A7F713
:106450002305F500A183A305F500B7E70400FC4779
:10646000310582972285F14597000000E7802024BE
:10647000230EA4002181A30EA400B24022444101B6
:10648000828082805D710A8586C6A2C49700000062
:10649000E780E0F437E404007C448A8508107946FC
:1064A00082973C441305E103094681458297101009
:1064B00093050002014597D0FFFFE7802023B640F7
:1064C000264461618280B7C7A55A01119387C733FB
:1064D0003EC497E7FF1F83C7B7EA3EC6B7F707007A
:1064E00003C7070106CE22CCA5476313F70001A01E
:1064F0001164930504F0930600100146254597C0EA
:10650000FF1FE780E02C3000930504F0A1462945E9
:1065100097C0FF1FE780C02B97E5FF1F83C555E697
:1065200017B501001305055397900100E78000ACF3
:10653000F24062440561828001119165A1463000FC
:10654000938505F02D4506CE97C0FF1FE7804028B4
:106550002247B7C7A55A9387C7336314F702B245DA
:1065600017B5010013054542B335B00097E7FF1F8B
:10657000A388B7E097900100E78040A7F24005614B
:106580008280814517B501001305454297E7FF1F3B
:10659000A38807DE97900100E78040A597000000E0
:1065A000E780A0F2E1BFB7C7A55A79719387F735A5
:1065B0003EC6B7E70400FC47AA8506D622D441466A
:1065C00008088297B7F7070003C70701A5476313B9
:1065D000F70001A01164930504E89306001001463A
:1065E000254597C0FF1FE780A01E7000930504E8B3
:1065F000D146294597C0FF1FE780801D17B50100D0
:106600001305054997900100E78020B6B250225447
:106610004561828079719165D1467000938505E866
:106620002D4506D697C0FF1FE780801A3247B7C7AF
:10663000A55A9387F73517B501001305253F631059
:10664000F702B7E70400FC4717E5FF1F1305C5C1B4
:1066500041460C08829717B501001305253B97901A
:106660000100E78080B0B25045618280B7F7070033
:1066700003C70701A5476313F70001A09165411106
:10668000930600100146938505E8254506C697C088
:10669000FF1FE780E013B24017B501001305052D79
:1066A000410117930100670043ACC16769768146D9
:1066B000FD1705061397060141836364B7003E8505
:1066C00082803307D50003470700B98F214713F8AD
:1066D0001700858363050800B18FC207C1837D174A
:1066E0001377F70F6DF78506F1B741C5A547054745
:1066F00063F2B70883471500034705003168A20716
:10670000D98F13978700A183D98FC207C18313083C
:10671000C855054763900707411106C622C426C223
:1067200003442500914763F087049307540063EC0A
:10673000F502A301C50021822302C50093043400A1
:1067400091C6A302D500A1822303D5002A84A68581
:1067500097000000E780A0F526942300A400218183
:10676000A300A4000147B240224492443A8541016B
:10677000828005473A858280B7C7A55A0111938761
:10678000E7343EC42AC6B7F7070003C7070106CEA1
:1067900022CC26CAA5476313F70001A091642A847E
:1067A000938504EE930600100146254597C0FF1F10
:1067B000E78000023000A146938504EE294597C08A
:1067C000FF1FE780E000A28517B501001305852AA9
:1067D00097900100E780808197000000E780C0CAA1
:1067E000F2406244D2440561828001119165A14664
:1067F0003000938505EE2D4506CE97C0FF1FE7803C
:1068000020FD2247B7C7A55A9387E7346318F702DC
:10681000B24517B501001305651B97D7FF1F2394D9
:10682000B7BAC205C18197800100E780207C97003C
:106830000000E78060C5F24005618280D147D14504
:1068400017B501001305851A17D7FF1F231DF7B6CB
:1068500097800100E780807917D5FF1F0355A5B603
:1068600097000000E78080F1F9B721C1411126C2ED
:1068700006C622C4AE848DC52A8497100000E78026
:1068800060E697E7FF1F83C7A7AF99CB2285224415
:10689000B240A68592444101173300006700E354DB
:1068A000B2402244924441018280828001114AC850
:1068B00006CE22CC26CA4EC693F715002E899DCB54
:1068C000AD67371700409387A7AA1CC3B7E704003A
:1068D000BC4F13060019854517D5FF1F034585AE2C
:1068E000829713451900F2406244D2444249B249AA
:1068F0000561828093F725006382071C17F7FF1F4D
:10690000035787F8954763F9E70C014417F6FF1F13
:10691000130686E793063005130550041308100488
:106920009308B00413039005930764006374F7049D
:106930003A84FD5997F4FF1F83C404E597F7FF1FBE
:1069400083C797E4A204DD8CAD679387B755638353
:10695000F41463E3970AA9679387A7556386F41431
:10696000A28517F5FF1F130525E297000000E780B9
:1069700000F0F5A8B307860083C50700639AD50425
:1069800083C517006396A50483C527006392050598
:1069900083C53700639ED50283C54700639A1503FC
:1069A00083C7570063966702A2890DE897F5FF1F1A
:1069B00083D585EDB3853541C20517F5FF1F130556
:1069C000A5DCC1814E9597000000E78040EA65A8EC
:1069D00005044204418089BF3A84FD598547E3EBB1
:1069E00087F459CC854517F5FF1F1305E5D99700A6
:1069F0000000E780C0E769A0B1679387C75563804F
:106A0000F404B5679387D755E39CF4F4A28517F592
:106A1000FF1F130565D797300000E780003D8947C9
:106A20006307F4049305E4FFC205C18117F5FF1F56
:106A30001305A5D597100000E780C0CA0DA89710D0
:106A40000000E78080C911C9A28517F5FF1F130553
:106A5000A5D397100000E780E0C80546A28517F58A
:106A6000FF1F130565D297F0FFFFE780C05DA68585
:106A700017B501001305C50397800100E780005793
:106A8000FD57E395F9F297F7FF1F239F07DE1345A4
:106A9000290091BDA28517F5FF1F1305E5CE97F0DC
:106AA000FFFFE780406BE1B7A28517F5FF1F1305D5
:106AB000A5CD97F0FFFFE780006E55BF93F7450027
:106AC0000145E38207E217B501001305A5FF978092
:106AD0000100E780806997300000E780A05F1345E0
:106AE000490011B5411122C437E404005C5C06C6BC
:106AF000354697B501009385E5AD17C5010013052F
:106B00002596829711E917B50100130565FC97805A
:106B10000100E780806501A08327041C82972A84F6
:106B2000054597C00000E780C01897700100E78016
:106B3000E09D97600100E780E07297B00000E78079
:106B4000402A2285B2402244410182801567B7174E
:106B500000401307575598C3D8439D66558FD8C337
:106B6000D843FD76758FD8C3D8431367F70FD8C3C2
:106B700035671307C7CC98C382804111054506C607
:106B800022C426C297C0FFFFE780E0391305A004A6
:106B900097B0FF1FE780A051757585457D1597C09B
:106BA000FFFFE78080237D7585451305F53697C087
:106BB000FFFFE780E02C371400408327840A8D45CF
:106BC0001305002093E707202324F40A97C0FFFF52
:106BD000E780A020B7E4040097C0FFFFE780C0650E
:106BE000C85897800100E780405817C50100130579
:106BF000258797800100E78040578327840C8545CF
:106C0000414593E707082324F40C97C0FFFFE78072
:106C100020278D451305000897C0FFFFE780402619
:106C200097C0FFFFE780205337A507001305051223
:106C300097C0FFFFE780C04E014597C0FFFFE78088
:106C4000E05495450545894717F7FF1F2300F7C412
:106C500097C0FFFFE7802055B7E700E01307000665
:106C6000238DE7403707000423A0E71097D0FFFFEC
:106C7000E78020E697D0FFFFE780E0F9970000006B
:106C8000E78080E697000000E780408B97000000D7
:106C9000E780E0B597E0FFFFE780C0D597100000E0
:106CA000E78080A597000000E780602D9710000026
:106CB000E780209E83A7040817050000130545BF41
:106CC000829797C7FF1F238FA76EBC4C13060064E3
:106CD0008545829797000000E78080E797B0FF1F07
:106CE000E780007101458280B7F7070003C70701FD
:106CF000A547AE866316F7009397450191C301A09F
:106D0000AA850146254517C3FF1F670063AC4111E3
:106D1000B2862E86AA852D4506C697C0FF1FE7803E
:106D200020ABB2400145410182809307000463E833
:106D3000C7021D71A2CC2A84080886CE32C697806D
:106D40000100E780401FB2461008A285294597C080
:106D5000FF1FE780E0A7F640664425618280395531
:106D6000828097F7FF1FA38107B897F7FF1F238D36
:106D700007CC97F7FF1F238907B6B7E70400FC5F2E
:106D8000411106C682978967938707F4B2403E9502
:106D900097F7FF1F23A8A7B4410182809306000242
:106DA0002547830705006385D7006383E70082805A
:106DB0000505C5BF17F5FF1F0345A5B20DE5411138
:106DC00022C417F4FF1F1304E4B11C4006C681CB94
:106DD000B7E70400FC5F82971C401D8D7D81B240A7
:106DE000224441018280054582808145B307B50078
:106DF0008387070091E789C917230000670043F3E1
:106E00008505C205C181DDB78280AA871375F50F9C
:106E1000130705FD1377F70FA54663E5E600138515
:106E200007FD82801307F5F91377F70FE54663E650
:106E3000E600011593178501E1871387F7FB1377A8
:106E4000F70F95467D5563E4E600138597FC828035
:106E500035C5011126CA4AC84EC652C406CE22CC38
:106E6000AE8997000000E780A0F32A898144414A57
:106E70000305090097000000E78060F92A840305F4
:106E8000190097000000E78080F86347040263451B
:106E900005021204B3879900498C2380870085047A
:106EA0000909E39744FD0545F2406244D244424952
:106EB000B249224A056182800145FDB701458280C1
:106EC0008147E5483387F5000307070019E30545C7
:106ED0008280B306F500038606009376F60F1388CA
:106EE000F6F91378F80F63E6080181161396860108
:106EF00061869376F70F1388F6F91378F80F63E637
:106F00000801138706FE620761876316C7008507BD
:106F1000C207C18345BF01458280011122CC2A846A
:106F20002E8526CA4AC84EC606CE2E8997800100F5
:106F3000E780003493140501C1809309D0038307CF
:106F4000040099E301450DA0CA8522859700000041
:106F5000E78040F70DC1B307940083870700639C67
:106F60003701138514002295F2406244D24442490D
:106F7000B249056182800504D9B797F7FF1FA38541
:106F8000079697F7FF1F238107AC97F7FF1F238D05
:106F9000079497F7FF1F2395079497F7FF1F238206
:106FA000079497F7FF1F23AF07928280011106CE47
:106FB00022CC26CA4AC84EC697200000E78060D679
:106FC00005E197F7FF1F238E079097F7FF1F23AB6D
:106FD0000790F2406244D2444249B249056182803E
:106FE00097000000E78040DD6DF597F4FF1F938464
:106FF000E48F130940078D4997F6FF1F83C6C68E9D
:10700000E9DA17F7FF1F0347378EB30727033384E7
:10701000F4000355240083550400636FB500050791
:1070200033773703FD1697F7FF1F238FD78A97F71C
:10703000FF1FA38BE78AC9B7898D91073E95C205CB
:10704000C181269597200000E780A0D759D18357AA
:1070500024003E952311A40045B7630705486385C6
:107060000548717156CBC16A26D34AD14ECF52CD55
:107070005AC95EC762C506D722D566C36AC12E8AC1
:10708000AA890149B54B17FBFF1F130B6B80F91A37
:1070900097D4FF1F9384441D17BC0100130C4CB8F8
:1070A00093170901C18363E04703BA502A549A54E5
:1070B0000A59FA496A4ADA4A4A4BBA4B2A4C9A4C5C
:1070C0000A4D4D618280B38729010387070097F736
:1070D000FF1F83D7E78063057701A9466313D73A7B
:1070E000D5CFDA9717E5FF1F1305857A23800700B0
:1070F00097000000E780C0CA97B50100938505A4FA
:107100002A8497000000E780E0DB49C5130564008E
:1071100097000000E780C0C82A8497000000E7803D
:1071200080C497B501009385E5A1228597000000F2
:10713000E78040D915CD8307240013F7F7FD01C779
:1071400025476397E7021308B0028147114797B6B6
:1071500001009386669F17B601001306A69F93054C
:1071600000080A8597800100E78060010A8539A838
:1071700097B50100938585A0228597000000E780E0
:1071800060D419CD17B501001305C59F9700000005
:10719000E780E0C597E7FF1F23940774050909B747
:1071A00097B501009385C5A2228597000000E7806E
:1071B00060D179C583073400130700026385E700B7
:1071C0002547639FE70A1305340097000000E78016
:1071D00020BD97B501009385E59F2A8497000000A4
:1071E000E78040CE0DC19307B0020147914617B624
:1071F00001001306669E930500080A85978001002A
:10720000E780E0F7A5B797B501009385659E2285D5
:1072100097000000E78000CB0DC517E7FF1F03476D
:10722000675697E6FF1F83D6466617B6010013061A
:10723000A69C930500080A8597800100E78020F44A
:1072400035B797B501009385659D228597000000AD
:10725000E78040C70DC181474147B386970083C689
:107260000600639E06228507E399E7FE17B5010035
:10727000130545B021BF17B501001305E59A39B7CD
:1072800097B501009385459C228597000000E78013
:1072900060C36303051E8307340013070002638580
:1072A000E7002547639AE71C1305340097000000A8
:1072B000E78000AF97B50100938545992A84970030
:1072C0000000E78020C02DC19305D0032285978060
:1072D0000100E78020F711C9830615000547938751
:1072E00006FD93F7F70F6377F70017B50100130555
:1072F000659669BD93071003639FF60097E7FF1F2C
:107300002381E75E97000000E780E0A517B5010044
:107310001305C596A5BD97E7FF1F2384075C97E774
:10732000FF1F23A1075CDDB797B501009385058F8B
:10733000228597000000E780E0B831C99305D003AB
:10734000228597800100E780E0EF11E517B5010085
:107350001305459425BD8A85050597000000E78043
:1073600060AF6DD5B7E70400FC4741468A852685A6
:107370008297268597F0FFFFE780202397F0FFFF95
:10738000E780801017B501001305059301B597B587
:1073900001009385E585228597000000E78080B293
:1073A00079C597B501009385659222859700000005
:1073B000E780E0B62A8D97B5010093852586228562
:1073C00097000000E780A0B5AA8C63080D046A85C9
:1073D00002C097000000E780A09C01468A852A8DA4
:1073E00097800100E780800082472A846307FD02BE
:1073F0009307F5FF63E3FA0263960C028147414766
:10740000B386970083C60600B1E68507E39AE7FED8
:1074100017B501001305C59795BB17B501001305F6
:10742000658BADB38A85668597000000E78080A2F2
:1074300011E517B501001305258C89BBB7E70400DA
:10744000FC47268541468A858297268597F0FFFF6F
:10745000E780A015131504014181A68597D0FFFF91
:10746000E780005E17B501001305458B05B317B51E
:1074700001001305258C19BB17B501001305858D77
:1074800031B3938617001306F004E365D6D0DA977C
:1074900017E6FF1F2316D6442380E70001B397B5F4
:1074A00001009385258E0A8597800100E78020DB07
:1074B000814C1304B100414DB387940103C607000A
:1074C0002285E285850C97800100E780C0D20904FF
:1074D000E394ACFF97A50100938545E5228597804D
:1074E0000100E780C0D759B18280F5C1854763F0BC
:1074F000C70E83C7150003C70500A207D98F1397CE
:107500008700A183D98FC2073167C1831307C7558D
:10751000639FE70A97E7FF1F83D727376389A70A87
:10752000011122CC06CE32C62E842AC49700000058
:10753000E780808835ED324693070007A24563ED6A
:10754000C70617E7FF1F0347273A894763E6E706A1
:1075500097E7FF1F83C7474F13074007B387E7022B
:1075600017E5FF1F13058538A2853307F5002310A3
:10757000C7002311070037E70400784791073E95BD
:10758000029797E7FF1F83C7274C0D478507B3F77F
:10759000E70217E7FF1F2309F74A97E7FF1F9387C3
:1075A000A73483C70700850717E7FF1F230EF732AD
:1075B000F2406244056182806244F24017A50100F6
:1075C0001305457F056117830100670023A28280B0
:1075D000011106CE22CC26CA01C5D54763EFB700FC
:1075E00017A501001305057F97800100E780E0B72C
:1075F000F2406244D244056182800347050093074C
:10760000500A2A846318F700034715009307A00562
:107610006307F70017A501001305457DF1B7034780
:1076200035009307100A630EF70059476386E5009B
:10763000034745006305F70217A501001305457CC4
:1076400065B7D1449147D1465D476393D40059470C
:1076500063FAE50017A501001305057C71B7D54451
:107660009547D5B737E704007847B305F4000A8596
:1076700041460297269483471400034504008A85F7
:10768000A2075D8D97D0FFFFE780803B95B7411142
:107690000D658D4506C697B0FFFFE7800074B717EC
:1076A00000408D6623A6D70A17E5FF1F1305053A8C
:1076B0001387C70A9387870A1CC15CC585668967DB
:1076C0005CC958C114C518C9B7E70400B24003A388
:1076D000871E4101028317E5FF1F0345A5388280FD
:1076E00097E7FF1F83C7173889E717130000670064
:1076F0002364828097E7FF1F83C7E73699EF411124
:1077000006C697100000E780A059B240854717E7EA
:10771000FF1F230AF734410182808280411126C273
:10772000AE848D4522C406C62A8497B0FFFFE78049
:107730002075B717004099C803A5C70C418D23A633
:10774000A70CB240224492444101828003A5870CD9
:10775000418D23A4A70CF5B7834705000347150007
:10776000A207D98FC2076177C18713072720639AC1
:10777000E700834525003705040017030000670074
:1077800023FA828017E6FF1F1306462E8147B28632
:107790001303F00FA9483308F6000348080013F755
:1077A000F70F6307A80C630668008507E39517FFCA
:1077B0002947B387E6002380A70097E7FF1F938739
:1077C000A72B5DA8411113D765001347170006C604
:1077D00093F63500058B954791CA0546994763870F
:1077E000C60009469D476383C600A14713F64500BE
:1077F0003336C00093F68503050685C2A145638B29
:10780000B604E145638AB604930580026388B60432
:10781000930580036393B600914697E5FF1F23828B
:10782000F54C97E5FF1F238DC54A97E5FF1FA389F8
:10783000D54ABE8517A501001305056297700100A2
:10784000E780C07AB240854717E7FF1FA30BF748D0
:10785000410182808546D1B78946C1B78D4675BF43
:1078600017A501001305C5611773010067000378B0
:1078700017E7FF1F13074720BA972380B700E14798
:10788000E302F5F493077002E30CF5FC82802A878B
:1078900023800500814717E5FF1F1305251D1308E9
:1078A000F00F2946B306F50083C606006396E6028C
:1078B00097E6FF1F9386461CB69783C707000545CA
:1078C0002380F5009947636EF7029D4763FDE7004B
:1078D000E147630DF7008280638506018507E39326
:1078E000C7FC0145C5B7238005008280B73700403B
:1078F00003C7370083C7050093F70704D98F238098
:10790000F5008280797126D24AD097E4FF1F83C4A4
:10791000244F17E9FF1F1309E94D06D622D44ECE96
:1079200052CC56CA5AC8B307990083C7070093F7C9
:10793000F70FA5C79387140093F7F70F0D476361FF
:10794000F70C17E7FF1F230DF74A97E7FF1F9387F1
:10795000E74AA69783C707001307100293F7F703B8
:107960006389E7226363F70A054463808720E38223
:10797000076809476389E71413070002E387E752A2
:10798000B7E700E03707400023A0E7180100010037
:10799000CA942380040023A0E710B787004003C7E0
:1079A0006700058BE308077297E6FF1F83C66645ED
:1079B0000547E393E67029472381E70209472383BC
:1079C000E7022385E70297E7FF1FA38D073097E7BC
:1079D000FF1FA3880742B7870040A381070017E76E
:1079E000FF1FA303073005472383E700B25022544B
:1079F00092540259F249624AD24A424B456182800E
:107A000097E7FF1F238E073E89B71307300263866F
:107A1000E70A63E6E71413074002638AE7081307DF
:107A20000003E39FE7F497E7FF1F9387E73CA697E0
:107A300003C70700A1471377F70FE313F71617EAF9
:107A4000FF1F130A2A0483476A0097E6FF1F23815A
:107A5000F62897E7FF1F83C7570391C7FD5797E69F
:107A6000FF1F2387F62697E5FF1F83C5B50197E71C
:107A7000FF1FA38FB72497E7FF1F83C7A70093F9C2
:107A800007089306000493F70706639DD74A9307F8
:107A9000A0096387F51463E4B7109307F0056384C6
:107AA000F548930750096382F52801440DABFD5753
:107AB00017E7FF1F230DF720E1B5FD5717E7FF1F5D
:107AC0002306F72075BD17A501001305E54C977037
:107AD0000100E780806997E7FF1F9387E731A6974A
:107AE00003C40700814917EAFF1F130A2A121374FF
:107AF000F40F97AA0100938AAA4A63C7890429450B
:107B000097700100E7806053854717E7FF1FA30DBB
:107B1000F70E17E7FF1F230A870E17E7FF1F230340
:107B2000F71C37E700E0B70640002320D718010014
:107B30000100378600408347A60293F7370F2305DD
:107B4000F6022320D7102DBDB3073A0183C50700E5
:107B50005685850997700100E780404979BF8547C0
:107B600017E7FF1F2302F70A21BD17E7FF1F1307BF
:107B7000A72826970347070097E6FF1FA384F6FC74
:107B800097E6FF1F2381E6FC17E7FF1F230CF7147E
:107B9000C5BB854717E7FF1F2306F7FAD5B3930741
:107BA000400A638DF5349307200B6388F5369307FD
:107BB000100AE39CF5EE83072A00014463D10742D3
:107BC00097E7FF1F83C737EC93F63700638E061ADB
:107BD0000546638EC62209466399C61A1D4775A2DB
:107BE00017E5FF1F034525EAC94717EAFF1F034AA8
:107BF0009AE997E5FF1F83C525E917E4FF1F0344B2
:107C0000B4E86319F510CD476316FA1093077008AE
:107C1000639CF5021307300FB7170E006308E400EA
:107C20001307900DB7B704006314E40817E7FF1FAC
:107C30002326F70ABE8517A501001305E5369770C0
:107C40000100E780A03A95B593078008639DF50091
:107C500033048040B77746001374F40F938787CDC1
:107C6000B3D78702E1B793079008639AF50033040E
:107C7000804091671374F40F9387C766D5B7930755
:107C8000A008639BF50033048040B7173D001374D0
:107C9000F40F93870790E9B79307B008639AF5004C
:107CA0003304804091671374F40F938797D04DBFCE
:107CB00093F5F5078D47639BF50033048040B79734
:107CC0005B001374F40F938707D859BF8947639BF0
:107CD000F50033048040B7770B001374F40F9387DB
:107CE000071BBDBF8547639AF50033048040DD67FD
:107CF0001374F40F938767E3A5B789E933048040D1
:107D00008D671374F40F938777DC99BFF1679387BE
:107D1000072029BF97000000E78000A7A2855285B1
:107D200097000000E78040A649B39305610017E57E
:107D3000FF1F034545D517E4FF1F0344D4D4970024
:107D40000000E78000B593057100228597000000D0
:107D5000E78020B43C0017E7FF1F232BF708834779
:107D600061002304F10083477100A304F1008947F7
:107D700017E7FF1F230EF7F48357810017E7FF1F54
:107D80002312F7D00944A1AC154793F64700B33648
:107D9000D00093F78703850685C32146638BC7060A
:107DA0006146638AC706130680026388C706130606
:107DB00080036393C700914717E6FF1F2302D6F2A3
:107DC00097E6FF1FA38EF6F097E7FF1F238BE7F0E0
:107DD00017E7FF1F034747CB9376070497E7FF1F7B
:107DE00083C797CA8DEE1377770C93067008630CE0
:107DF000D7021377F7078D46631ED70AB307F04003
:107E0000B7955B0093F7F70F938505D881A81947BD
:107E1000ADBF854755B7894745B78D4771BF9306B5
:107E200070086311D7021307300FB7150E0063896E
:107E3000E7021307900DB7B504006383E702130749
:107E4000700845BF9306800C6311D702B307F0405A
:107E5000B775460093F7F70F938585CDB3D5F50237
:107E600097E7FF1F23ACB7E6F9B39306900C631AAC
:107E7000D700B307F040916593F7F70F9385C56678
:107E8000F1BF9306A00C631BD700B307F040B715F2
:107E90003D0093F7F70F93850590C9B79306B00C93
:107EA000E319D7F4B307F040916593F7F70F938583
:107EB00095D06DB78946631BD700B307F040B775FF
:107EC0000B0093F7F70F9385051B49BF8546631A8F
:107ED000D700B307F040DD6593F7F70F938565E3AF
:107EE000B5BF09EBB307F0408D6593F7F70F9385A6
:107EF00075DCADB7F165938505209DB783472A00F2
:107F0000C18B99C7854717E7FF1F2306F7DC71BEB2
:107F100097E7FF1F238107DC49BE854717E7FF1F4F
:107F2000A301F7DC59B63C0017E7FF1F2322F7EC4B
:107F30000947930700032314F10097E6FF1F2389E5
:107F4000E6D82DBD63990758A94763EBB74417A737
:107F500001001307A7ED8A05BA959C41BA9782875D
:107F600017E4FF1F034434B2094A630C440F636CE7
:107F70008A0885476309F40A9307F00F17E7FF1F84
:107F8000034707D563F6E70017E7FF1F2302F7D47F
:107F900017EAFF1F034ACAD3930700041374FA0FAA
:107FA00063F447011304000497E7FF1F938747E436
:107FB00083AA0700228617E5FF1F1305A5ACD68507
:107FC000330A8A40A29A97700100E780C0F697E7CB
:107FD000FF1F238F47CF97E7FF1F23AB57E197E79B
:107FE000FF1F83C7F7CE15476399E762B7E700E045
:107FF0003707400023A0E71801000100B7860040C2
:108000002380860285A58D47630CF40A9947E31502
:10801000F4F697A701009387E7E717E7FF1F2329E7
:10802000F7DCA947A1BF17E7FF1F034787DD97E7E5
:10803000FF1F9387E7CB494697A50100938585EEFF
:108040006306870097A501009385C5E93E85977073
:108050000100E78040EE17E7FF1F232BA7D8C94791
:1080600031BF97E6FF1F83C6C6D9054797E7FF1FB5
:10807000938707C86394E6023E851306700297A5AE
:1080800001009385A5E797700100E780C0EA17E734
:10809000FF1F232FA7D493077002CDB53E8513068B
:1080A000300497A501009385A5DF97700100E78054
:1080B00080E817E7FF1F232DA7D2930730047DBD6B
:1080C00097E5FF1F83C5259C17A50100130505EF44
:1080D00097700100E78080F1854A17EBFF1F034B83
:1080E0004BD297E5FF1F83C5059A17A5010013051D
:1080F000E5EC63185B0B97700100E78020EF97E7D2
:10810000FF1F83C74798B5CBE368F4E617A40100C7
:10811000130484E5638C670117A40100130444E58C
:108120006386470117A40100130404E622859770B3
:108130000100E780E0131375F50F9307150086071C
:1081400017E7FF1F2306F7BA8D4717E7FF1FA301A5
:10815000F7BA97E7FF1F9387A7B90147BE86137643
:10816000F70F89076365A60297E7FF1F23A2D7C809
:1081700097E7FF1F83C7C7B711B597A7010093877C
:10818000A7D717E7FF1F2325F7C69147C5BB3306BF
:10819000E40003460600A380070005072380C7000C
:1081A0007DBF97700100E78060E497E7FF1F83C7FA
:1081B000878DE1D7E362F4DC17A401001304C4D770
:1081C000638C570117A40100130484D76386470109
:1081D00017A40100130444D8228597700100E7809A
:1081E00020091375F50F93071500860717E7FF1F82
:1081F0002300F7B08D4717E7FF1FA30BF7AE97E7F4
:10820000FF1F9387E7AE0147BE861376F70F8907F6
:10821000E37CA6F43306E40003460600A3800700CF
:1082200005072380C700D5B797E5FF1F83C5A58540
:1082300017A50100130545D997700100E78000DB01
:1082400097E7FF1F83C797AA93E7470017E7FF1F2A
:10825000A30EF7A883472A0017E7FF1FA306F7A876
:10826000A9B017A50100130565D797700100E78035
:10827000C0EF97E7FF1F938727A783C7070017E77C
:10828000FF1F2301F78017E4FF1F034464A4333466
:108290008000B1B317A50100130585D597700100C3
:1082A000E780A0EC97E7FF1F83C757A493E7070178
:1082B00017E7FF1FA30CF7A283472A0017E7FF1F4A
:1082C0002304F7A26FF06FFE17A50100130585D3F5
:1082D00097700100E78060E903470A007D8B51EF4A
:1082E000B787004003C767021377C70B13672700E0
:1082F0002383E70203C7A7021377C70B136727007F
:108300002385E70203C7E7021377C70B136727002C
:108310002387E70203C727031377C70B13672700D9
:108320002389E702854717E7FF1F230DF78017E72B
:10833000FF1F230BF78C17E7FF1F2309F79817E799
:10834000FF1F2306F79897D7FF1FA38D077E97E798
:10835000FF1FA38B078A97E7FF1FA389079697E75D
:10836000FF1FA386079697E7FF1FA38D079697E742
:10837000FF1FA38807A86FF04FF389476312F70226
:1083800097D7FF1F83C747709146638CD70863E078
:10839000F604638EE70C6369F70A05476380E70E0E
:1083A000FD5717E7FF1FA305F79237074000B7E710
:1083B00000E023A0E71801000100B7860040130683
:1083C000F0FC2381C60223A0E7106FF06FDB1307D8
:1083D00020086382E7086362F70213071008E3913D
:1083E000E7FC378700408347670293F7C70B93E7A3
:1083F00027002303F7026FF04FEB13073008638960
:10840000E70213074008E39DE7F8378700408347FA
:10841000270393F7C70B93E727002309F7026FF0B1
:10842000CFE8378700408347270393F73707F5B72F
:10843000378700408347E70293F7C70B93E727008E
:108440002307F7026FF06FE6378700408347E702A4
:1084500093F73707F5B7378700408347A70293F7AD
:10846000C70B93E727002305F7026FF00FE4378768
:1084700000408347A70293F73707F5B737870040D7
:108480008347670293F73707ADB717A501001305B8
:1084900065B897700100E78040CD97D7FF1F238311
:1084A000075ED5B317A501001305C5B79770010086
:1084B000E780A0CB97D7FF1F2396075C97E7FF1FA6
:1084C0009387078103C40700894763F38700094442
:1084D0001374F40F29B613070002E393E7EC6399D2
:1084E000090A638FF500930720026381F50817A539
:1084F00001001305A5B697700100E78020AF4DB5C8
:1085000017A501001305C5B297700100E780E0C50B
:10851000014417AB0100130BEBB2A14AB3078A0069
:1085200083C507005A85050497700100E78000ACF9
:10853000E31654FF17950100130545E597700100F8
:10854000E780A0C217D4FF1F0344045411E497D757
:10855000FF1F238B075061B48947E313F4E4854779
:1085600017D7FF1F2302F7506FF02FD417D6FF1F26
:108570000346765197D5FF1F83C5E55017A5010027
:108580001305C5AC97700100E78040A66FF0EFD1EE
:10859000638FF50493071002E39BF5F497D5FF1F53
:1085A00083C5854E17A50100130545AC97700100E2
:1085B000E780C0A397E7FF1F23AC478397D7FF1F30
:1085C0009387C771944383D7470017D7FF1F03478B
:1085D000477117D6FF1F2327D64A1D4497D6FF1F82
:1085E0002394F64A97D7FF1F2381E74ACDBA97D540
:1085F000FF1F83C5654917A501001305A5A897703E
:108600000100E780A09E97D7FF1F238F074497D7CD
:10861000FF1F239907466FF0EFF62547E388E79C95
:1086200019476391E702B786004023808602B7E7C7
:1086300000E03707400023A0E718010001001306FF
:1086400000FC41B31307100A6391E702B7860040AC
:1086500023808602B7E700E03707400023A0E71831
:1086600001000100130680FCA9BB1307A009E38FDA
:10867000E7FC1307400AE38BE7FC13072002E387BC
:10868000E7960547E384E796B7E700E03707400041
:1086900023A0E718E392099601000100B786004085
:1086A00023808602130620FC29BB17D7FF1F034730
:1086B00037626308F71E63E7E7029547630EF70E1C
:1086C00099476308F704B786004023800602B7E79E
:1086D00000E03707400023A0E7180100010013065F
:1086E000A0FCC5B19307F005630AF7009307500992
:1086F0006306F70093071002E317F7FCB7E700E003
:108700003707400023A0E71801000100B7860040AA
:1087100051BF97D9FF1F83C9A95B93070004CE8A75
:1087200063F43701930A000497D7FF1F9387476CC0
:1087300003AA070013F4FA0F2286D28517D5FF1F6C
:108740001305453497600100E780E07EB3878940D8
:10875000529417D7FF1F230DF75697D7FF1F23A952
:108760008768638E0902B787004023805703B7E606
:1087700000E03706400023A0C6180100010003C72F
:108780002702134707042381E70203C72702137751
:10879000C70F2381E70223A0C6106FF06F9EB78634
:1087A000004023800602B7E700E03707400023A01F
:1087B000E71801000100FDB5378700408347370007
:1087C00097D6FF1F83C6565293F70708D58FA3018C
:1087D000F700B7064000B7E700E023A0D718010074
:1087E00001001306A0FC2301C70223A0D7106FF0DD
:1087F0002F9997D7FF1F93872760A69783C70700F6
:1088000093F7F70FD9CF97D7FF1F83C7875FD1EBB8
:1088100017D7FF1F0347D74B930700026313F708CF
:1088200097D7FF1F9387072603AB070097DAFF1F31
:1088300083CA8A2517DAFF1F034A1A2597D9FF1F13
:1088400083C9A924D2875687CE865A8697D5FF1F1B
:1088500083C5852117A50100130545849760010094
:10886000E780C07897D7FF1F23AA674797D7FF1FD6
:108870002388574797D7FF1FA384474797D7FF1FE2
:108880002381374797D7FF1FA38F871CB7E700E0E7
:108890003707400023A0E71801000100B786004019
:1088A000D1B3B7E700E03707400023A0E718010085
:1088B0000100B786004025B529472381E702094713
:1088C0002383E7022385E7022387E7022389E70260
:1088D0006FF06F8F03C76700118B6309079083C721
:1088E0005700918BB5CF17D7FF1F03478751854797
:1088F0006313F70697D7FF1FA385E73E97D7FF1FA0
:108900002382072497D7FF1F2380073097D7FF1FA5
:10891000238E073A97D7FF1F238B073A97D7FF1F5E
:10892000A382072297D7FF1FA380072E97D7FF1F89
:10893000A38E073897D7FF1FA38B073897D7FF1F42
:10894000A382073A97D7FF1FA38D074AB787004036
:1089500011476FF06F8917D7FF1FA306F71079BF74
:10896000854717D7FF1F230FF71C17D7FF1F230DAE
:10897000F72817D7FF1F230BF73417D7FF1F23083C
:10898000F73469BF854717D7FF1F230DF71A17D78D
:10899000FF1F230BF72617D7FF1F2309F73217D71F
:1089A000FF1F2306F73217D7FF1FA30D071817D78E
:1089B000FF1FA30B072417D7FF1FA309073097D763
:1089C000FF1FA38607308280411106C69700000072
:1089D000E78080FBB787004023800700130740FC37
:1089E0002386E7001307C004A386E70017D7FF1FFD
:1089F000130747092398E70017D7FF1F1307870CB2
:108A0000239AE70017D7FF1F13070718239CE700D7
:108A100017D7FF1F13078723239EE70029472381CA
:108A2000E70209472383E7022385E7022387E7025A
:108A30002389E702A3810700930600F8A380D700EB
:108A4000930690022380D700FD562383D70023810D
:108A5000E700B706400037E700E02320D71003C740
:108A6000170013671700A380E700B24097D7FF1FD6
:108A7000239C072641018280411106C69700000011
:108A8000E78080F0B787004023800700130700FCD1
:108A90002386E7003147A386E70017D7FF1F130798
:108AA00067FE2398E70017D7FF1F1307A701239A34
:108AB000E70017D7FF1F1307270D239CE70029475F
:108AC0002381E70209472383E7022385E702A38185
:108AD0000700930600F8A380D70093069002238036
:108AE000D700FD562383D7002381E700B706400057
:108AF00037E700E02320D71003C7170013671700DC
:108B0000A380E700B24097D7FF1F239F071C4101B6
:108B10008280F1679387072017D7FF1F2320F71C58
:108B2000854717D7FF1F231DF71AA14717D7FF1F28
:108B30002309F71A97D7FF1FA385071A97D7FF1F97
:108B40002382071A97D7FF1F238007F297D7FF1FAB
:108B5000A38B07F0814717D5FF1F130525F1FD559E
:108B600017D6FF1F130646F12947B306F5002380E9
:108B7000B600B306F600238006008507E397E7FEFC
:108B800097D7FF1F2388072697D7FF1FA3840726A1
:108B900097D7FF1F2381072697D7FF1FA38B0712A5
:108BA00097D7FF1FA389071297D7FF1F23840712A8
:108BB00097D7FF1F238F071097D7FF1F238E07100C
:108BC00097D7FF1FA388071097D7FF1F238507108C
:108BD00097D7FF1FA3810722828017D7FF1F034764
:108BE000472285476316F70017030000670003E973
:108BF00017030000670083DD411122C406C617D7A2
:108C0000FF1F0347072085472E8613F4F50FAA851B
:108C10006317F70417D5FF1F130505FB97600100C5
:108C2000E780603197D7FF1F238007FEB78700409A
:108C300023848702B7E600E03706400023A0C61869
:108C40000100010003C7A7021377C70F2385E702BE
:108C5000B240224423A0C61001454101828017D5AD
:108C6000FF1F130525EA97600100E780C02C97D706
:108C7000FF1F238907ECB787004023828702B7E6EE
:108C800000E03706400023A0C6180100010003C71A
:108C900067021377C70F2383E7025DBF411106C642
:108CA00097000000E78020E7B24041011703000071
:108CB0006700E3F2411106C697F0FFFFE780C0C4EA
:108CC00097D7FF1F83C717E8A1CB97D5FF1F83C591
:108CD00085E789C917D5FF1F130505E797E0FFFF53
:108CE000E780E03797D7FF1FA38E07E497D7FF1FD2
:108CF000238A07FE37E700E0B70640002320D71895
:108D000001000100378600408347660293F7370F62
:108D10002303F6022320D710B2404101828017D5E9
:108D2000FF1F034565FC3335A000828041C9D9C5CA
:108D300097D7FF1F83C747FBD1C3011122CC4AC875
:108D40004EC656C25AC006CE26CA52C42E89AA8919
:108D50000144930A0004371B030063772403B3071D
:108D60008940C207C183BE8463F4FA0093040004FF
:108D7000C204C180130A1BD497D7FF1F83C787DCA7
:108D80009DE37D1A631C0A00F2406244D2444249CA
:108D9000B249224A924A024B0561828097F0FFFF56
:108DA000E78080B6D1BF338589002694A68542042A
:108DB00097000000E78080E4418045B78280411140
:108DC00006C622C429C12E8495C997D7FF1F83C721
:108DD000A7F195CB97D7FF1F83C7C7D68DC71307BA
:108DE0000004AE876374B70093070004139407016F
:108DF0004180A28597000000E78040E02285B240D4
:108E00002244410182800144D5BF97D7FF1F938739
:108E1000E70218429C4383D645000345070083C5FB
:108E2000C700035646006396A50083D5E700638D0F
:108E3000D502011106CE2386A7002397D700B705D8
:108E4000CF00DC4B9385757D05077D162EC2230070
:108E500001003AC42316C1002317D10099C30A8523
:108E60008297F240056182808280DC4DDC4B81CFAD
:108E7000B7E70400904503A38705914517D5FF1F69
:108E8000034505FC028382806D713C083EC6B7072E
:108E9000E500232291103EC8AA843C08328523268F
:108EA00011103ECA23248110232021112E899730CE
:108EB0000000E780005E2A84979501009385852154
:108EC00017850100130505E497600100E780001293
:108ED000A285179501001305653097600100E780B2
:108EE000E010294597600100E7802015B705CB0009
:108EF0009385757D680097100000E7802067A28544
:108F0000680097300000E780204B014781467000E1
:108F1000CA85268597200000E780A08A05CD2A848F
:108F2000979501009385051B17850100130585DDC5
:108F300097600100E780800BA2851795010013055B
:108F4000A52A97600100E780600A29459760010023
:108F5000E780A00E8320C1100324811083244110D8
:108F6000032901105161828097D7FF1F938707ED76
:108F700018429C43797122D406D60348070083C85F
:108F800007012A8483D645000355460063960801ED
:108F900083D82701638DD802238807010507239909
:108FA000D7003708CC00DC4B1308787D3ACC130788
:108FB000F5FF42CA23080100231EE100231FD10050
:108FC00099C7080832C62EC482973246A245228528
:108FD00097000000E78080EBB25022544561828008
:108FE0006D713C083EC0B707E5003EC23C083EC478
:108FF000232611102324811023229110231701000E
:109000002318010023190100231A0100231B01006A
:1090100097A7FF1F83D7873D99E3C167FD172316E5
:10902000F10097A7FF1F83D7873C91EB97D7FF1FCE
:109030009387C7E09C439C43DC4783D7070017A472
:10904000FF1F1304A43A584C2317F1008357440020
:10905000484B2318F10031E1979501009385850E67
:1090600017850100130505CA97600100E78000F825
:10907000179501001305450E97600100E78000F782
:10908000294597600100E78040FB8320C11003243D
:109090008110832441105161828097A7FF1F83C7ED
:1090A000573589EBB7E70400BC5782975C4C23AA7D
:1090B0000700E1BFFD1797A6FF1FA38CF6320356EA
:1090C0000701834704014C470A85230BF1009730C1
:1090D0000000E780802B97D7FF1F938727D69C43FC
:1090E0000147814688430A866C0097100000E7809C
:1090F000406DAA8429C1979501009385A504178521
:109100000100130525C097600100E78020EEA685C9
:10911000179501001305050597600100E78000ED34
:10912000294597600100E78040F1584CB7E70400FB
:10913000BC57484B9DBF97A7FF1F83C7972BF5D7F9
:10914000B7E70400BC4F1044854517D5FF1F034502
:1091500025CF82971DBF5C4EDC4BB9CFB1CD4111FD
:1091600022C4178501001305E5B92E8497950100E7
:10917000938585FB06C697600100E78020E7A285FE
:10918000179501001305C50097600100E78000E610
:10919000294597600100E78040EAB7E704002244D0
:1091A000B24003A3870517D5FF1F034565C9130602
:1091B00040069145410102838280411122C417A4D7
:1091C000FF1F130464201C4C06C689C7DC4399C3E7
:1091D0004C488297584CB7E70400BC57484B8297DD
:1091E0005C4CB240224423AA07004101828017A7A9
:1091F000FF1F1307671F834707009306F00B8507C0
:1092000093F7F70F63E9F60097A6FF1F238EF61C6E
:10921000034507008280930700F8FDB78357450098
:109220006386071001114AC817A9FF1F1309091CFB
:1092300052C4032AC90106CE22CC03274A0126CAFA
:109240004EC656C2F15735E31307D00DFD57636E76
:10925000C704B7E9040083A709072A841305860019
:1092600042054181B284AE8A8297232AAA0003254F
:10927000C9015C49A9E7979501009385E5E8178541
:109280000100130525A897600100E78020D61795F7
:109290000100130525F897600100E78020D52945D6
:1092A00097600100E78060D9DD57F2406244D24404
:1092B0004249B249224A924A3E850561828093879B
:1092C0004400B705CF002319F5009385757D31055E
:1092D00097100000E78080290325C90183456400B9
:1092E000310597300000E780200D0325C90126864F
:1092F000D685310597300000E78020097146A285A8
:109300004A8597600100E78000C3504419CA83A7CB
:109310008905854517D5FF1F034585B2829781478B
:1093200069B797000000E780E0CBD5BFFD573E85C9
:109330008280411126C297A4FF1F9384240BD84C2E
:1093400022C437E404003C54484B06C68297DC4CE8
:109350000323C4052244B240924423AA070017D530
:10936000FF1F0345E5AD854541010283411126C23A
:1093700097D4FF1F938484AC9C4006C622C44AC085
:10938000D5C3DC43C5C35CC12300B5002A849795CF
:1093900001009385A5D2178501001305A596976056
:1093A0000100E780A0C4294597600100E780E0C87C
:1093B0009C4023A4070023A2070097A7FF1F9387C1
:1093C000A700DC4FDC4B91C7295597000000E780D0
:1093D00000DF97A7FF1F93876701DC4FDC4B89C72E
:1093E00097000000E78020F537E904008327C905CE
:1093F000894517D5FF1F0345A5A482978327C90573
:10940000914517D5FF1F0345A5A382979C4003A351
:1094100047016309030022852244B2409244024975
:1094200041010283B24022449244024941018280B8
:109430000111328506CE22CC26CA2E849730000038
:10944000E7802005AA8497950100938565CA178552
:1094500001001305258B97600100E78020B9030701
:1094600084000356640083554400A68617950100C6
:10947000130505D497600100E78040B72945976040
:109480000100E78080BB97A7FF1F83C747F4639D58
:109490009700014597000000E78060D281450A856A
:1094A00097000000E780C0ECF2406244D2440561BE
:1094B00082806D71232481102326111023229110A4
:1094C00093F745002E84638707143C083EC0B70716
:1094D000E5003EC23C083EC42317010023180100EA
:1094E00023190100231A0100231B010097A7FF1F66
:1094F00083D787ED99E3C167FD172316F10097A77E
:10950000FF1F83D787EC91EB97D7FF1F93870793B4
:109510009C439C43DC4783D7070017A7FF1F130713
:10952000A7EA2317F100544F835747002318F1008F
:10953000DC4AA1E7979501009385C5BF1775010027
:109540001305457C97600100E78040AA179501004C
:10955000130585C097600100E78040A92945976001
:109560000100E78080AD134544008320C11003242F
:109570008110832441105161828097A7FF1F83C708
:1095800017E52555D9C3FD1717A6FF1FA301F6E45C
:1095900003D6060183470701CC460A85230BF10059
:1095A00097300000E78060DE97D7FF1F9387078919
:1095B0009C4317A7FF1F130727E197960100938687
:1095C000A6BC88430A866C0097100000E780601FE5
:1095D000AA8451D9979501009385C5B517750100E7
:1095E0001305457297600100E78040A0A685179596
:1095F0000100130525B797600100E780209F2945EA
:1096000097600100E78060A3268597000000E7804F
:1096100000BB91BF93F725009DC7B7E70400BC4787
:109620004146814528088297255597000000E7802C
:1096300000B928089305F00F97000000E78040D399
:10964000134524001DB793F71500014599DF9700D6
:109650000000E78020991345140001BF5C4D4111C3
:1096600006C688C317C7FF1F232AF77CB7E7040085
:1096700083A70708170500001305E5E38297B240AA
:1096800097C7FF1F238EA77A0145410182800111F0
:109690003335A000A307A100B7E7040083A747174D
:1096A00006CE1306F1008545130550308297F2402F
:1096B000056182808280411122C406C697C7FF1FC0
:1096C00083C78779014489EF97B7FF1F83C757CBBB
:1096D000054499E717C4FF1F0344C40A1344140048
:1096E000228597000000E780C0FA17950100130556
:1096F00025BE09E417950100130585BE2244B2403A
:109700004101176301006700638E797122D4A30FB2
:10971000010037E404008327841726D24AD006D6F6
:10972000AA842E89130550309305F10132C6829721
:1097300032468347F10193150601C18185CB01456E
:109740002EC697000000E780C0F483274417B24577
:109750004A8626858297054597000000E78060F3DA
:10976000B250225492540259456182808327441793
:109770004A8626858297EDB741119397050122C449
:1097800006C626C2C1872E8463D40702B7E404004C
:10979000FC5417A5FF1F034565C8829719C1BC5427
:1097A00082972165218DB2402244924441018280FA
:1097B00093F715008DC7B7E7040083A7471A17A6CC
:1097C000FF1F1306A6C497C5FF1F9385256817A51D
:1097D000FF1F0345A5C4829713451400E9B793F70B
:1097E000250099CFB7E70400BC4F130600648945F4
:1097F00017A5FF1F034585C282971345240065B74F
:1098000093F7850085CF97C7FF1F83C7A76585E7B7
:10981000B7E7040003A8871A1307401F97A7FF1F85
:1098200083C7C7BF814613064006994517C5FF1F6A
:109830000355C562029813458400B5B793F74500F8
:109840000145B5D3B7E4040083A7041817C5FF1F6B
:109850000355C5608297BC4C13060064914517A55B
:10986000FF1F0345A5BB8297134544002DBF97C733
:10987000FF1F83D7A75E6398A70217C7FF1F231098
:10988000B75E17C7FF1F231DC75C17C7FF1F231A2B
:10989000D75C2E86179501001305C5A9BE85175301
:1098A00001006700A37417950100130525AA17632B
:1098B00001006700838B0357450097C7FF1F83D7BD
:1098C000E759631EF704C1674111F91722C417C78E
:1098D000FF1F2325F75837E4040097C7FF1F23A174
:1098E000075897C7FF1FA389075697C7FF1F238BEA
:1098F00007567C4C06C6894517A5FF1F034505B2D0
:1099000082977C4C914517A5FF1F034525B182978F
:109910002244B240410117030000670003DA1795A3
:1099200001001305A5A217630100670003847D15DC
:10993000954763E2A71C17970100130727970A05AD
:109940003A951C41011122CC06CEBA972E8482870B
:1099500017950100130505A097600100E780E080DE
:10996000A1A203C7250099476311F7022E8597002E
:109970000000E78080F4834564001795010013051B
:10998000659E97500100E780606697B7FF1F2389A7
:10999000079E179501001305A59E7DBF03C72500EF
:1099A00095476319F702C16717C7FF1F0357074B96
:1099B000F91703D5A5006309F702B7E7040083A7E9
:1099C000C7178297179501001305859C97500100D2
:1099D000E780A079854717B7FF1F2303F79A1795EC
:1099E00001001305659D8DBF97C7FF1F2398A746EC
:1099F00083D7E50097C6FF1F2393F64683D705015B
:109A000097C6FF1F239EF64483D7250197C6FF1FE5
:109A10002399F64497C7FF1FA3800744631BE50201
:109A2000B7E70400BC4F096613060690A14517A5C9
:109A3000FF1F0345A59E82970356E4008355A400AB
:109A4000179501001305059697500100E780005A0D
:109A500051B79307700F2316F100B7E7040083A7EF
:109A6000870D17A6FF1F0346669B6C0082974DF972
:109A7000854717C7FF1FA301F73E5DB71795010084
:109A800013054594D1BD83C5250091476392F50226
:109A9000179501001305859497500100E780E06C4D
:109AA00097000000E78060C1F24062440561828057
:109AB00099476392F502228597000000E780E0DF76
:109AC00083456400179501001305C589975001006F
:109AD000E780C051D1BF9547639AF50083471400D2
:109AE000E1F3179501001305A591BDB51795010088
:109AF00013058591E1BF8280411122C417A4FF1F85
:109B000013040493AA86178601001306A67B2285F8
:109B1000C14506C697500100E780606603574400C0
:109B200097A7FF1F9387C7912393E700035764000C
:109B30002394E700B240224441018280411106C6CD
:109B400097000000E78080FBB7E7040083A7871435
:109B500017A6FF1F1306C68DD54501458297B24053
:109B60004D4697A5FF1F9385A58D130570304101C4
:109B7000170300006700A3B961712324811A37E439
:109B80000400832704082326111A2322911A232074
:109B9000211B232E311917050000130525BE8297BE
:109BA00017A9FF1F13098987994785442300A90036
:109BB000231CF100978501009385C5749307400627
:109BC0001775010013050514231CF10823089100E3
:109BD00097C9FF1F938969CB97500100E780004127
:109BE00083D50900178501001305C5709750010042
:109BF000E780C03F294597500100E780004403D526
:109C00000900896997000000E78040EF8327441727
:109C1000100885451305503082978327441717A6EF
:109C2000FF1F1306E681CD45130570308297832709
:109C300044171796FF1F1306A67EB545130560301F
:109C4000829783274417300889451305103182977E
:109C500083274417300989451305203182978327CC
:109C60004415938509900D45829783274415938564
:109C7000099011458297A3059100230691002308BE
:109C8000910002CD230C01008327841630099145F1
:109C9000130570408297832784161306B10085450B
:109CA00013050040829783278416700085451305AD
:109CB000104082978327841630088545130520407D
:109CC0008297832784161008854513055040829794
:109CD000832704157D558297832744137D558297EA
:109CE0007D5597A0FFFFE78040998327440C82971A
:109CF0009790FFFFE780A074832784141796FF1FB7
:109D000013060673D5450145829789471306700FE0
:109D1000814528092306F1009780FFFFE780203E58
:109D20008D471306000881452808230CF108978009
:109D3000FFFFE780C03C9147230CF10097770100BB
:109D40009387C7ED984383C747003AC8230AF100B9
:109D500097C0FFFFE780407370008545054597A0D9
:109D6000FFFFE780A09830099305700F094597A081
:109D7000FFFFE780A0973008930500080D4597A0E6
:109D8000FFFFE780A09610089545114597A0FFFFBB
:109D9000E780C095C16717C7FF1F1307270CF91786
:109DA0001CC3232207001795FF1F1305E56697A024
:109DB000FFFFE78080928327C41D17C5FF1F13058F
:109DC000650882973C4803450900854582978320B2
:109DD000C11A0324811A8324411A0329011A8329F1
:109DE000C1195D618280C16717C8FF1F035808074A
:109DF000F9176301F8083DCDB5CD011126CAB7E4C6
:109E0000040083A7841222CC2E862315B10006CE2F
:109E10002A8401478146ED45428582972AC611ED85
:109E2000178501001305054F97500100E780E033C7
:109E3000F2406244D24405618280FC440356A10092
:109E4000A28582972C0017C5FF1F0355250197A0F7
:109E5000FFFFE780409569DD178501001305C54CBC
:109E600097500100E780603083A7C412ED452800B9
:109E700082977DBF8280411106C61DC9854717970D
:109E8000FF1FA304F75A35469795FF1F9385455941
:109E9000130560309797FF1F238A0758970000002B
:109EA000E780E086B2404101170300006700E380CD
:109EB0009797FF1FA38B0756F9B797C7FF1F83C755
:109EC00067FAA9EFC16717C7FF1F035727F9F917EB
:109ED0006306F7044111854722C417C7FF1F2303F8
:109EE000F7F837E404007C4C06C6A1451795FF1F20
:109EF0000345C55282970323841A2244B2409797A0
:109F0000FF1F83C7A75117C5FF1F035525F513076B
:109F1000401F8146314699454101028382806D711F
:109F2000232481102326111023229110328401CD85
:109F30008947630AF5028320C1100324811083241A
:109F4000411051618280178501001305A54CAE8434
:109F500097500100E7806021A285268597B0FFFF1A
:109F6000E7804070C9BFB7E70400FC47280082972C
:109F7000178501001305C54A97500100E780E01ED0
:109F80008347810039C41307000B6380E7021387FE
:109F9000A7051377F70F8D4663EDE602A28528002B
:109FA00097C0FFFFE78020DF79B78547E3F587F8A3
:109FB00083459100177501001305C50BB335B0003B
:109FC00097A7FF1F238EB72297500100E78000025A
:109FD0009DB703479100A207D98F35671307D7555F
:109FE0006385E7086368F7022D671307B755638732
:109FF000E70631671307C755638AE7042967130724
:10A00000A7556394E702A285280097C0FFFFE78069
:10A01000801815B739679306E7656381D70863E948
:10A02000F6001307E7556384E706A28528003DB7CD
:10A030003D679306F755638AD7061307F766E396DD
:10A04000E7FE97C0FFFFE780C032F5B50146A28565
:10A05000280097C0FFFFE78000FFF1BDA285280020
:10A0600097C0FFFFE780200FF9B58947E3F587EC3C
:10A0700097000000E780A0E49305E4FFC205C181DA
:10A080001305A1009790FFFFE78080146DB5A285AE
:10A09000280097C0FFFFE780C01271BDA28528008D
:10A0A00097C0FFFFE780801D79B597C0FFFFE7806D
:10A0B000002651B5C16717C5FF1F035525DAF917EB
:10A0C0006307F500B7E7040003A3C7170283828084
:10A0D000854717C7FF1F2301F7D8014517F3FFFF77
:10A0E0006700235B1783FFFFE702C3FC2A84084550
:10A0F0002E89B28919C900C1971500009385A586DC
:10A10000610597300100E780800181447D5A9710F6
:10A110000000E780E03963C7A40481449710000081
:10A12000E780003A63C8A40497C7FF1F9387C7D38B
:10A130009C43DC47B307F94091872302F400638313
:10A1400009048327C900B307F4409587A302F400EC
:10A150001C4C89C79C4799C3228582971783FFFFB0
:10A16000670083F85C44139714008504BA97239022
:10A17000470171BF1C48139714008504BA972390B8
:10A18000070069BF832789000547B307F440958717
:10A19000A302F40083570400638EE7028DC30947CE
:10A1A0006384E7040D47E395E7FA978701009387F7
:10A1B000E7791CCC978701009387477A11A8978786
:10A1C0000100938727401CCC978701009387874025
:10A1D0005CC8BDBF978701009387C72B1CCC9787AE
:10A1E00001009387272CEDB7978701009387C77AE3
:10A1F0001CCC978701009387277BD9BF95E51783F0
:10A20000FFFFE702C3EC00461844834794007583C0
:10A210009D8B6317F70097100000E78060B448C477
:10A220001783FFFF6700E3EC82801783FFFFE702DD
:10A2300063E813893500C16442094111AA890144C8
:10A24000F11413590901054A2EC697100000E78042
:10A250002026B2456348A400014541011783FFFF52
:10A26000670083E883A7090013171400BA9783D700
:10A2700007006388B7006394970063742A0105049C
:10A28000E1B70545D9BF1783FFFFE702C3E1AA89FC
:10A290002E89328BB6843A8ABE8A97A00000E78066
:10A2A00020FB71C9268597200000E78020098D4793
:10A2B00063E7A7007D551783FFFF670043E283DB59
:10A2C000440097100000E780A0242A849710000023
:10A2D000E78040259307740031443305850263CD40
:10A2E000A70297100000E780A02297100000E780E7
:10A2F00020222A8497100000E780C0229307740070
:10A3000031443305850263C3A70497100000E7803A
:10A3100020209307450029A897100000E78080209F
:10A32000330585021307F0179307C017E35FA7FAF9
:10A330002D55E3C277F963040B02D6865286A685B3
:10A340004A8597200100E78020BAB5B79710000032
:10A35000E780401D330585029307C5FFD1BF8327E2
:10A3600049001385C90083D5270097000000E780C6
:10A3700000EC61F581B769553DBF97C7FF1F239773
:10A38000A7AE97C7FF1F938727AE904381470C4620
:10A390003307F500420741836393B7008280544638
:10A3A000139847008507C2962390E600D5B797C754
:10A3B000FF1F938767AB9C4303C58700828017C547
:10A3C000FF1F0355A5AA82801783FFFFE70223D052
:10A3D000C1671387D7FF630BE502636AA700F11714
:10A3E0006300F50201451783FFFF670083D01387E1
:10A3F000E7FF6302E502FD171D8D13351500E5B774
:10A4000097500000E780C0267D15C5BF975000001B
:10A41000E78040FBD5BF97500000E78060F9EDB7BB
:10A420001783FFFFE702A3CA4111AA8401442EC685
:10A4300097100000E780C008B2456348A4000145BA
:10A4400041011783FFFF6700C3CA9C48131514001E
:10A450003E9583570500E385B7FE0504C9BF034851
:10A460005500814693F7F60F63E5070181473E8566
:10A470008280584593975600BA9703D727006316F2
:10A48000B70003D70700E304C7FE8506E1BF834694
:10A49000450001479377F70F63E4D700814711A880
:10A4A0001C45131657000507B29703D60700E313A0
:10A4B000B6FE3E8582801783FFFFE702A3BF931796
:10A4C0000501C18797CAFF1F938A0A9A635BF00848
:10A4D00083A70A00C0479C4703570400198D420513
:10A4E00041816368F500014422851783FFFF6700FF
:10A4F000A3BF12052A94CDBFDC4713944900014A3B
:10A500003E94834744006341FA02014A8347540062
:10A510006349FA028509C20993D9090183A70A0090
:10A520009847E3EBE9FCC1B71C4413195A00A68510
:10A530003E994A8597000000E780C0EE05E1050AD4
:10A54000C9B75C4413195A00A6853E994A859700FD
:10A550000000E78020ED19E1050A4DBFE30C09FA80
:10A5600061B7AA8481495DBF1783FFFFE70223B665
:10A570001C452A8481E79307C5001CC51C4423128F
:10A5800004001CC09307F00F63EDB70093F5F50FBF
:10A59000228597200000E78020E21783FFFF6700F5
:10A5A00043B593940501C167C18063F9F500A685A1
:10A5B000228597200000E78040E5C5B7C18193F56B
:10A5C000F50F228597200000E78000DFA685228511
:10A5D00097200000E78040E0C9B797C7FF1F938727
:10A5E000A788884382801C4599C797C7FF1F23AD62
:10A5F000A786014582807D55828097C7FF1F93877C
:10A60000A786984383474500484792073E95828036
:10A610001783FFFFE702A3AB617100451C183EC61C
:10A62000B70780013EC81C183ECA8357440002CEBB
:10A6300002D002CC231EF100834784002A8902D273
:10A640002301F1023C083ED402D697000000E780C7
:10A6500000FB835705002316F10297500000E780A6
:10A6600060C42307A1025C4003556400F18313F723
:10A6700017008347F10252055181F99BD98FA30737
:10A68000F10297100100E780807539CDAA84035547
:10A69000050097A00000E78080BC83D704002AD281
:10A6A0006800231CF10083D72400231DF1001C48FF
:10A6B00003D647008C4397200000E78000CD8347F6
:10A6C000B400CA8617860100130646D68117A30573
:10A6D000F4006C00481097200100E780E0805D6185
:10A6E0001783FFFF6700E3A02155D5BF1C45B1CFFD
:10A6F00003C5A700894613576500630BD7028D4633
:10A70000630ED70285466300D70213074006330560
:10A71000E50203C7B700418B15CB83C7B700BD8BDC
:10A720003355F54082801375F5031307803EC5B796
:10A7300009671375F50313070771D1BF37270900A0
:10A740001375F5031307077CD9B70145828017837A
:10A75000FFFFE702C39703A98500630C0904834741
:10A76000B900AE8493F7070E85C30345990093059E
:10A7700020030D810505B305B502884461059730B6
:10A780000100E780E0A935A02E8597000000E78052
:10A7900020F62A8419CD97000000E780605C8325AD
:10A7A000C900B307B54063FA87002E94B305A440EF
:10A7B000E9F51783FFFF6700C39385457DBF1783C6
:10A7C000FFFFE702C3902A8403D50500011132C6BA
:10A7D00036C43AC22EC002CA02CC02CE97A00000F4
:10A7E000E780E0A782452ACA22852ECC9700000088
:10A7F000E780E0E003570500231EE10097500000CA
:10A80000E78040AAA24632469247230FA10036872E
:10A810004C08B2862285014697000000E780E0A63A
:10A8200005611783FFFF6700C38C1783FFFFE702F3
:10A83000038A61711C183EC6B70780013EC81C1808
:10A840003ECA3C0800453ED4AA8402CC02CE02D0C7
:10A8500002D202D697000000E78060DA8357050035
:10A8600035592316F10297500000E780A0A3230773
:10A87000A10209C48357440081EB21594A855D61D7
:10A880001783FFFF6700E38603556400520551817B
:10A8900097100100E780A0542A8965D18347B4004E
:10A8A00093F7070E99C71305840197300100E780DD
:10A8B000609983574400231EF100834784002301DD
:10A8C000F1025C4003550900D98313F70708834759
:10A8D0001102231CA10093F7F707D98FA300F102FF
:10A8E00083572900231DF1005C40F18313F7170003
:10A8F0008347F102F99BD98FA307F10297A00000CB
:10A90000E780E0952AD235D98347940068001397F1
:10A9100057008347B400FD8BD98FA305F4001C4872
:10A9200003D647008C4397200000E78000A6A68747
:10A9300017870100130787AF740005464C10268562
:10A9400097000000E78060942A890DD98347B400FE
:10A95000A685FD8BA305F40097000000E78060DF6B
:10A9600031BF1773FFFFE7028376832485FE2A84B5
:10A970004111268597000000E78080D7834734FF88
:10A9800093F7070E8DCB2AC6268597000000E78037
:10A9900060C809CD834734FFB245FD8BA309F4FE9F
:10A9A00091C5228597300100E780808741011773A8
:10A9B000FFFF670003747DD98327C4FF2685829734
:10A9C00075F5834734FF93F7070E91C722859730BB
:10A9D0000100E7802087032584FE97000000E780C0
:10A9E00000E5E9B71773FFFFE702636B9C41411174
:10A9F0002A8903C7070089472E849356670063801E
:10AA0000F6040D466388C6049307F0076304F70253
:10AA10002E8597200000E780C0A7AA848149C16BDA
:10AA2000130C490097B7FF1F938707449C4398472F
:10AA300063E4E90441011773FFFF6700036A03D76A
:10AA400045008547E3F8E7FE2E8597200000E78064
:10AA5000A0A9E1B703D74500E3FEE7FC2E859720C8
:10AA60000000E78000A3AA84228597200000E780E9
:10AA700060A4C204C98C5DB7DC470355A900139AD2
:10AA800049003E9A93170501C187635DF000835723
:10AA90000A006397A70263E774038327CA00034D84
:10AAA0005A002DA0A1672167A98F1307F7EFE37460
:10AAB000F7FE6397090097000000E780209161FD91
:10AAC00085098DB783278A00034D4A00835DA9005D
:10AAD00003576900216A138BC7003AC6814A33CAFB
:10AAE0004D01631E5D0197B7FF1F938767389C4335
:10AAF000E1DBA2866286814526858297D1B7A16770
:10AB00009387F7EF930C4BFF63F24703B2455A85E7
:10AB100097F0FFFFE780A0710DC103278B0010475E
:10AB200009CE10436382C4023107D5BFEE85668526
:10AB300097000000E780008F71F993861A0093FA5E
:10AB4000F60F130B0B0271BF835644005C43E3E91D
:10AB5000F6F622853AC697100000E780807DA1674F
:10AB60009387D7042A8A035D4400324763E897003D
:10AB70008347D90093E707F8A306F9001C476685C9
:10AB80002286E2858297C1670844FD17337AFA006E
:10AB9000529508C02312A40125B797B7FF1F9387CA
:10ABA000A72C9843814715C31447814763FFD500FD
:10ABB000939745004C47BE9519C903C75500814777
:10ABC0006375E600DC451606B2973E85828003C7B2
:10ABD00045008147E37BE6FE16069C45F5B71773F3
:10ABE000FFFFE702234DAA892E8A814497BAFF1FEF
:10ABF000938A8A2783A70A00984763E6E4001773BD
:10AC0000FFFF6700634EDC471394440001493E9404
:10AC100013BB140083474400634BF900014913BB85
:10AC2000140083475400634FF9008504E1B70844DA
:10AC3000931759005287DA860146A2853E9582997C
:10AC40000509C9BF4844931759005287DA8605465B
:10AC5000A2853E9582990509E9B71773FFFFE702C0
:10AC60000347814517F5FFFF1305054897B7FF1FF9
:10AC7000239E071E97000000E780A0F61773FFFFD2
:10AC80006700234797B7FF1F9387071E9C4395C311
:10AC90001773FFFFE702A343814517F5FFFF130575
:10ACA000A54497000000E780C0F31773FFFF67001B
:10ACB000434482801773FFFFE702C33F37E4040079
:10ACC0008327841241112315E100AE893289368A27
:10ACD0003A8681460147ED45AA8482972AC621C952
:10ACE0000356A100D28597400100E780C024832746
:10ACF000C413CE8526858297058905C98327440D0F
:10AD00002314210101462C00268582972A8401C93B
:10AD1000B7E7040083A7C712ED4528008297228574
:10AD200041011773FFFF6700233C4944D5B76554C1
:10AD3000FDB75C41FD175CC182801773FFFFE7021E
:10AD40000339B7E70400FC5F829795473305F502A6
:10AD500081450D811773FFFF6700A3391773FFFF4C
:10AD6000E702E336B7E70400FC5F829795473305B7
:10AD7000F5020D811773FFFF6700A3371773FFFFFD
:10AD8000E702E334B7E7040083A7870B0355050008
:10AD900082971773FFFF6700C3351773FFFFE70242
:10ADA0000333035505003287AE861786FF1F03560F
:10ADB000466F97B5FF1F9385E50B97000000E7806E
:10ADC000A0EF1773FFFF6700C3321773FFFFE7029F
:10ADD0000330B7E7040083A7C71782971773FFFFF5
:10ADE000670023311773FFFFE702632EB7E7040004
:10ADF00083A7871397B5FF1F9385C50782970145E2
:10AE00001773FFFF6700E32E1773FFFFE702232C82
:10AE1000B7E7040083A7C71F81451785FF1F0355A8
:10AE2000456482971773FFFF6700A32C1773FFFF1A
:10AE3000E702E329B7E7040083A7871397B5FF1F4D
:10AE400093854504829701451773FFFF6700632AC6
:10AE50001773FFFFE702A327B7E7040083A7C71F05
:10AE600081451785FF1F0355C56582971773FFFF3F
:10AE7000670023281773FFFFE70263252E8597805D
:10AE80000000E780E0AF97800000E780E0EC1773F8
:10AE9000FFFF670003261773FFFFE7024323978036
:10AEA0000000E780E0F61773FFFF670083245C492A
:10AEB000E1175CC95CC583572501A1072319F5007B
:10AEC00083570501A1072318F5008280F147330558
:10AED000F50297B7FF1F9387E7FC9C433E9582805E
:10AEE0008D476315F60803D74600854763F0E708EA
:10AEF0001773FFFFE702A31D368536842E8997104E
:10AF00000000E780005929C98357440093140501C4
:10AF1000C18063E39704228597100000E7806057A3
:10AF2000FD14231294009307A0026300F502930717
:10AF3000B0026307F50293079002631FF5002285B4
:10AF400097000100E780C08501A80146CA852285D7
:10AF500097A00000E78060B01773FFFF67006319D8
:10AF6000228597100000E780C003FDB7828097B666
:10AF7000FF1F938666F39C42014599CF9843D442C4
:10AF800017B6FF1F2322E6F26396D70097B6FF1F7E
:10AF900023AEE6F01385C7FE82801773FFFFE7023A
:10AFA000031397000000E780A04B7144330585022E
:10AFB000914597900000E78020E911E565551773EA
:10AFC000FFFF6700031397B7FF1F23ABA7EC9700A2
:10AFD0000000E780E0483305850291459790000026
:10AFE000E78080E661DD97B7FF1F23ADA7EA9700F2
:10AFF0000000E780E04697B7FF1F239DA7E8970072
:10B000000000E780E04597B7FF1F2396A7E89777F2
:10B0100001009387E74617B7FF1F2321F7E897073B
:10B020000000938707E917B7FF1F2327F7E60145BD
:10B0300079B71773FFFFE7028309AA8517B5FF1FCA
:10B04000130545E597100000E780C05B1773FFFF0D
:10B050006700230A1773FFFFE702630797000000EA
:10B06000E78060FD97100000E780405B97B7FF1F07
:10B07000938787E39C4391CF1387C7FE19CB83D572
:10B08000C7FF17B5FF1F1305A5E297200100E78052
:10B0900020191773FFFF6700C3051773FFFFE7024F
:10B0A000030397000000E780C0EC09CD83478500CB
:10B0B0002A8493F7070499EB0355E50097000000F5
:10B0C000E78080F91773FFFF6700A3028347C5007D
:10B0D0009304450117B9FF1F130909DD85E3832791
:10B0E00009005CC997B7FF1F23A097DC832749009D
:10B0F000F1FB97B7FF1F23AB97DAE9B7FD172306DC
:10B10000F500610597800000E780C0D683078400C2
:10B1100063CB07048347840093E707F82304F40014
:10B12000B7E704009C5F82974205A94741813375C8
:10B13000F5028347840093F707FCC98F2304F400CA
:10B140008347D4003E951C402318A40089CF984320
:10B1500019CB8347C4005040814585073305F5026C
:10B16000420541810297832709005CC897B7FF1FFA
:10B1700023AC97D28327490089E797B7FF1F23A7FE
:10B1800097D28347C4009DDF8355040117B5FF1F85
:10B19000130505D297200100E780800825B71773B3
:10B1A000FFFFE702C3F297B7FF1F9387A7F59C47FE
:10B1B00001448583858B85E3AE84B2853A869710FA
:10B1C0000000E780804B2A8419C597100000E780B3
:10B1D000C041829408CC22851773FFFF670063F19A
:10B1E0001773FFFFE70203ED41112E8932C6AA89CA
:10B1F00097000000E780C031324713060502CA8677
:10B20000970500009385C5CC17B5FF1F130585C8AA
:10B2100097000000E780E0F82A8425C99304C50060
:10B2200097000000E780E0411946AA85268597101F
:10B230000000E78080158545268597100000E7808F
:10B24000601117750100130565214E9583450500B2
:10B25000268597100000E78020165C48314681451E
:10B26000A1075CC85CC483572401E1172319F400CB
:10B2700083570401E1172318F4001C4C3E85977096
:10B28000FFFFE780C0E7A304250122854101177372
:10B29000FFFF670063E51773FFFFE70243E3411118
:10B2A000AA842EC632C497100000E7806036004D95
:10B2B000B2452246834784000CC050C093F7F70381
:10B2C00093E707042304F40023180400268597104D
:10B2D0000000E780803183479400A9462317A4002B
:10B2E00013D7370005073307D7029D8B8507230641
:10B2F000F400A306E40083C70401D8488507230FA0
:10B30000F7FE17B7FF1F130727BA5843232A040075
:10B310009307440129E317B7FF1F2329F7B817B78D
:10B32000FF1F2323F7B817B4FF1F130464B8228547
:10B3300097200100E78000E11C44858B5D8D19E5B5
:10B340008145228597200100E78080ED4101177338
:10B35000FFFF670003DA1CC317B7FF1F2328F7B4EA
:10B36000D9B71773FFFFE70283D6970500009385CF
:10B3700065B7014597000000E78000B001451773ED
:10B38000FFFF670003D71773FFFFE70243D497005F
:10B390000000E78080B01773FFFF670083D5834705
:10B3A000C500A5E31773FFFFE70263D22A840355A4
:10B3B000E50097000000E78000C821C183478400B2
:10B3C00093F7F7FB2304F4001C4091C7DC4381C7CB
:10B3D0004C400145829797000000E78080B917B57F
:10B3E000FF1F1305E5AC97200100E780A0E503559A
:10B3F000E40097000000E78020C61773FFFF670096
:10B4000043CF82801773FFFFE70263CC97B7FF1F1C
:10B41000938787A997050000938565C817B5FF1F17
:10B42000130505A923A0070023A207009720010008
:10B43000E780E0CE1773FFFF6700A3CB1C4D91CFD1
:10B44000DC4381CF1773FFFFE70263C88345070022
:10B4500082971773FFFF6700C3C9828097B7FF1FEA
:10B46000938747A79C4303C50700828097B7FF1FB8
:10B47000938747A69C4303C51700828097B7FF1F99
:10B48000938747A59C4303C52700828097B7FF1F7A
:10B49000938747A49C4303C54700828097B7FF1F4B
:10B4A000938747A39C4303C53700828097B7FF1F4C
:10B4B000938747A29C4303C55700828097B7FF1F1D
:10B4C000938747A19C4303C56700828097B7FF1FFE
:10B4D000938747A09C4303C57700828097B7FF1FDF
:10B4E0009387479F9C4303C58700828097B7FF1FC0
:10B4F0009387479E9C4303C59700828097B7FF1FA1
:10B500009387479D9C4303C5A700828097B7FF1F81
:10B510009387479C9C4303C5B70011E11D4582807A
:10B5200097B7FF1F9387079B9C4303C5C700828083
:10B5300097B7FF1F9387079A9C4303C5D700828064
:10B5400097B7FF1F938707999C4303C5E700828045
:10B5500097B7FF1F938707989C4303D50701828005
:10B5600097B7FF1F938707979C4303C527018280E6
:10B5700097B7FF1F938707969C4303D547018280A7
:10B5800097B7FF1F938707959C4303D56701828078
:10B5900097B7FF1F938707949C4303D58701828049
:10B5A00097B7FF1F938707939C4303C5A70182802A
:10B5B00097B7FF1F938707929C4303C5B70182800B
:10B5C00097B7FF1F938707919C4303C5C7018280EC
:10B5D00097B7FF1F938707909C4303C5D7018280CD
:10B5E00097B7FF1F9387078F9C438857828097B731
:10B5F000FF1F9387278E9C4303D5C702828097B78E
:10B60000FF1F9387278D9C4303D5E70219E113059C
:10B61000800C828097B7FF1F9387C78B9C4303C51D
:10B620000703828097B7FF1F9387C78A9C43C85B35
:10B63000828097B7FF1F938767898843828097B777
:10B64000FF1F9387E7888843828019E17D558280B8
:10B65000F5DE984265DFFDD917B7FF1F130787AAEC
:10B660001847AA877155058B631D072403C507007A
:10B670001547E37DA7FC03C737001305F0057D17C9
:10B680001377F70FE364E5FC03C35700E30003FC03
:10B6900083C86700E38C08FA03C777004945791728
:10B6A0001377F70FE364E5FA03C7A7001148130502
:10B6B000F7FF1375F50FE36BA8F803CE97000D485D
:10B6C0001305FEFF1375F50FE362A8F803C8B70072
:10B6D0006309080065181378F80F1305600DE36718
:10B6E00005F703C5C700794879151375F50FE36FA2
:10B6F000A8F403C8D7000D457D181378F80FE36749
:10B7000005F503D80701930E401751184208135846
:10B710000801E3ED0EF303C8E7007D181378F80F76
:10B72000E36605F303C827017D181378F80FE36F6C
:10B7300005F103C88700C54E75181378F80FE3E7C5
:10B740000EF103D86701856E938EBEE06D18420836
:10B7500013580801E3EC0EEF03D847016D184208B7
:10B7600013580801E3E40EEF03D887017918420863
:10B7700013580801E36C05ED03C8A7017D18137881
:10B78000F80FE36505ED03C5B7011D487D15137579
:10B79000F50FE36DA8EA03C5D70171487915137554
:10B7A000F50FE365A8EA03D5E7011308E00F7D155F
:10B7B00042054181E36CA8E803C5070249487915B1
:10B7C0001375F50FE364A8E8C85301C937C83400FE
:10B7D0005915130858BFE36BA8E603A8870237C5BD
:10B7E0003400130555BF5918E36205E717A5FF1F7D
:10B7F0002320C56E03C6050117A5FF1F232CF56C7A
:10B800000545E375C5E403D82501D0493376060321
:10B81000E31E06E203C61501E30A06E217A6FF1FB0
:10B820002326B66A83C5270001466387A50003C6A1
:10B830001700F1453306B60283C707039305C0021C
:10B8400072971A071307C70516031A9796084697A3
:10B85000B387B70241553E973297420741836362EF
:10B86000E8061773FFFFE70283863685978000009E
:10B87000E780A06897000100E78020482A8497A00D
:10B880000000E780805A2A9497F00000E780602645
:10B890002A9497900000E780A0812A9497F0FFFFF8
:10B8A000E780E06F2A9497400000E78060932A9435
:10B8B00097700000E780A09C22951773FFFF670038
:10B8C000438382801773FFFFE70263804111A30760
:10B8D000A10097A00000E780A0C59305F10017051F
:10B8E00000001305E5B597F0FFFFE780802F0145C5
:10B8F00041011763FFFF6700C37F1763FFFFE70284
:10B90000837A17A4FF1F1304E47F03288400795966
:10B910009368180097A4FF1F23AA147F13781800B8
:10B9200063100802BA84BE89368B328A2E89AA8AAD
:10B9300097F0FFFFE780E0A77D15269519E53159BF
:10B940004A851763FFFF6700837997F0FFFFE78061
:10B9500040A67D152695A167E353F5FE97B7FF1F17
:10B96000938747B198433E8C814B01CB014597F0BB
:10B970000000E7802044933B15004A85DA8656860E
:10B98000D28597900000E780C04D2A8911CD1C44D4
:10B99000F99B17A7FF1F232BF77683270C00CDD326
:10B9A000E3800BFA829769BF268597A7FF1F23AD17
:10B9B000077497F0FFFFE780809C4146CE8517A56E
:10B9C000FF1F1305A57D97300100E780C05697D073
:10B9D0000000E78040990325040B97D00000E78022
:10B9E000009D054597D00000E78000A4054597001D
:10B9F0000000E78060EDA9B797A7FF1F93878770C6
:10BA00009C47858BEDC71763FFFFE702436C17A5C3
:10BA1000FF1F1305E57697A7FF1F23A5076E97A7BE
:10BA2000FF1F23A3076E97A7FF1F23A1076E972071
:10BA30000100E780208197500000E780E0F5971033
:10BA40000100E780A04C97100100E780A05297A763
:10BA5000FF1F9387A7699C4391C705459780000006
:10BA6000E780402097A7FF1F938707529C4399C701
:10BA700041657D1597700000E78040A297F00000B7
:10BA8000E780E03D97D00000E780808F97A7FF1FF9
:10BA90009387477C9C43139717016356070097F0E1
:10BAA0000000E78000AD97A7FF1F23A9076E97A7A7
:10BAB000FF1F23A7076E97A7FF1F23A5076E97A752
:10BAC000FF1F23A3076E97000000E780008C9700FC
:10BAD0000000E780007297F0FFFFE780401897F0C2
:10BAE0000000E78040D61763FFFF67008360828015
:10BAF00097A7FF1F93870761884382801763FFFF23
:10BB0000E702E35C97800000E780607597800000A3
:10BB1000E780C0771763FFFF6700A35D1763FFFF30
:10BB2000E70243592A849304140201112E85B28935
:10BB3000A685214636C63A8997300100E780403D08
:10BB40000DE9B24638082686CE8513059404975031
:10BB50000000E780604121462C084A8597300100AB
:10BB6000E780003B1335150005611763FFFF670091
:10BB7000A3570145D5BF1763FFFFE7024355930560
:10BB8000450617A5FF1F1305253597100100E7800F
:10BB900020691763FFFF6700C3551763FFFFE702C4
:10BBA000035341112EC697F0FFFFE780601BB2459B
:10BBB00088C141011763FFFF6700A3531763FFFFAD
:10BBC000E702434FAA842E8497800000E780006C30
:10BBD000AA898545228597000000E780E07D83C71C
:10BBE000E4011389940899E313890403CE8522851F
:10BBF00097000000E780407C2146930519022285CA
:10BC000097000000E780607897A7FF1F9387874F12
:10BC10008C43228597100000E780C08221469385DF
:10BC20008402228597000000E78020761763FFFFDB
:10BC30006700834B1763FFFFE702E346397197F014
:10BC40000000E780E0B49305400661E997800000BA
:10BC5000E78000606302051497A7FF1F83C7872949
:10BC600013B7170097A6FF1F2386E628014499CF34
:10BC7000C16417A9FF1F1309E9489309400EFD1479
:10BC800097000000E780C0866342A40A97F0FFFF98
:10BC9000E780000D4169B7290900096AFD7A2A8BFE
:10BCA00081447D199389F97B130A0A71938A8AC7A3
:10BCB00097000000E780C08363D7A4041304400EFC
:10BCC000B387840217A7FF1F1307C7430324070B7B
:10BCD0003E948357C4016382270B18403307EB401F
:10BCE00063EAE900834744008507B3874703D69793
:10BCF0006365F70801468145094597F0FFFFE78036
:10BD0000604EAA8B29E597400000E7808083854735
:10BD10006317F50689659385057117A5FF1F130540
:10BD2000A51B97100100E780A04F95A0B30734032F
:10BD30000327090BBA9703D7C7016308970003C706
:10BD40005700A38207002382E700050415BF93056F
:10BD5000C500228597000000E78080E65E85228688
:10BD6000976501009385C57097F0FFFFE780E0526B
:10BD70005E8597100000E780608A850415BF97A74D
:10BD8000FF1F938727389C478D83858BC1F72161DF
:10BD90001763FFFF6700A33401468545094502D0BC
:10BDA00002D202D402D697F0FFFFE780A043AA8414
:10BDB00079DD97F00000E780E09C1389C4002A84B5
:10BDC00081454A8597000000E780005F0C404146AE
:10BDD0004A8597000000E780405B83294400638523
:10BDE000090C4E8502D802DA02DC02DE973001002F
:10BDF000E78000482ACE141005462C0808184ECCBF
:10BE000097500000E780E00A1375F50F51ED835558
:10BE1000840093E525004A8597000000E780E05EF6
:10BE200011460C104A8597000000E7800056014635
:10BE30009765010093854564268597F0FFFFE780AD
:10BE4000C045268597000000E780407D5C40A1D377
:10BE5000014685450D4597F0FFFFE780A038AA848D
:10BE60001DD548401389C40097300100E780404049
:10BE70002AC64A8597000000E780404C3246636F2F
:10BE8000C5004C404A8597000000E78000500146FD
:10BE90008145268597F0FFFFE780204026859700A3
:10BEA0000000E780A077E5B583558400ADB7176340
:10BEB000FFFFE702C32197A7FF1F9387A7249C4793
:10BEC0001DC193E7870017A5FF1F1305E50017A7FE
:10BED000FF1F232DF72297100100E78040321763E0
:10BEE000FFFF67000321DD9B17A7FF1F2320F72219
:10BEF00097300000E780E0647DF117A5FF1F130570
:10BF0000A5FD97100100E780E033D1BF1763FFFF65
:10BF1000E70263194169AA892E8AB28A368BBA8BE5
:10BF2000814417ACFF1F130CEC1D930C400E7D19C0
:10BF300097F0FFFFE780C05B63C4A40001443DA00D
:10BF40003384940383270C0B3E948357C401638688
:10BF500027055A87D6865286CE8513050403970097
:10BF60000000E780E0BB01C923800B002285176336
:10BF7000FFFF6700C3168347F40185C35A87D6863F
:10BF80005286CE851305940897000000E78040B9DB
:10BF900009C585472380FB00D1BF850451BF835766
:10BFA00045006380071E1763FFFFE702A31001111E
:10BFB0002A8497000000E780C04D09C985476309BE
:10BFC000F50605611763FFFF6700031297E00000A5
:10BFD000E780007C7DF5835744004947ED9BE39261
:10BFE000E7FEC145228597000000E7804033AA8420
:10BFF000228597000000E780204F0357440002CEBF
:10C0000091472A89631AF700228597000000E7808C
:10C01000A0513C082ACC3ECE97E00000E780807615
:10C020005C55C5D374084A86A6850545829751BFDD
:10C0300003574400D147E3F6E7F8032A0400C16937
:10C04000014997AAFF1F938AEA0B130B400EFD19B3
:10C0500097F0FFFFE780C049634FA90E2285032AAE
:10C06000040097000000E780C042A1452A8922858C
:10C0700097000000E780A02AAA842285970000008C
:10C08000E780804A14402A86AA8978082685CA85CE
:10C0900097000000E780C0E7AA8405D503C7F40134
:10C0A00089476315F7008347C10181DF5546D28573
:10C0B0001385640097300100E780E0E70145978031
:10C0C0000000E780C01901C583D7C401A5E797A781
:10C0D000FF1F938727039C4793551900858913D722
:10C0E0003700058B01CF8983858B6399B7000145A4
:10C0F0002EC697000000E780C0DBB2454E859780D2
:10C100000000E780601F0346C1012A84937519006F
:10C11000268597900000E780E03935C12685978015
:10C120000000E780E018268511C0014597800000D7
:10C13000E780004C97300000E780A0408547E3127D
:10C14000F5E883C754001307F00FE38CE7E6850793
:10C15000A382F400BDB5B304690383A70A0BBE94A0
:10C1600083D7C401638B37015546D285138564009C
:10C1700097300100E780C0D955DD0509D1BD5DD8F4
:10C180006DB782801763FFFFE702C3F2978000005C
:10C19000E780000C05C1C164014417A9FF1F130902
:10C1A00069F69309400EFD1497F0FFFFE7804034D5
:10C1B000634EA40017A5FF1F130505D297100100B9
:10C1C000E780E0031763FFFF670003F233053403E2
:10C1D0008327090B3E958357C50163889700231277
:10C1E000050097800000E780A00C050475BF97A7A5
:10C1F000FF1F938727F19C478D83858B8DE3176302
:10C20000FFFFE702C3EC17A5FF1F1305E5CC97104E
:10C210000100E78020031763FFFF670083ED828042
:10C220001763FFFFE702A3EA970500009385C5A007
:10C2300017A5FF1F130545CA97100100E78020EEE0
:10C240001763FFFF6700E3EA1763FFFFE70223E8D6
:10C250008841B7E70400BC5B050542054181829730
:10C2600009C585472300F50005051763FFFF670033
:10C2700043E883C7F5FF2E858507A38FF5FE8280EF
:10C2800083C7F5FFFD1793F7F70FA38FF5FE99EF1F
:10C290001763FFFFE702A3E3B7E70400BC5713856A
:10C2A000F5FF82971763FFFF6700A3E482801C41BC
:10C2B000035745008D8FBA951CC12312B5003E85EA
:10C2C000828093D78500A2051441DD8D83574500F8
:10C2D0001387E6FF18C189072312F50013D68500DE
:10C2E0004111238FB6FEA38FC6FE41018280184103
:10C2F0009307F7FF1CC18357450085072312F500FC
:10C30000A30FB7FE8280835745008D8F2312F5005F
:10C310001C41BE950CC12E858280AA8703D7470099
:10C3200008410D8FAA952392E7008CC382801841A3
:10C3300008453305A74082808357450003576500B1
:10C340001D8F1C4108453385A7403305A7408280D7
:10C350001763FFFFE702A3D741112EC62A84970077
:10C360000000E780A0FDB2456373B50001A08357CC
:10C3700044000840BE952312B4003E954101176366
:10C38000FFFF670003D71763FFFFE70243D44111A4
:10C390002E84B28532C697000000E780A0FB3246AB
:10C3A000A28597300100E78000B941011763FFFFC4
:10C3B000670023D41763FFFFE70263D12E8485450E
:10C3C00097000000E78000F9230085001763FFFF56
:10C3D000670023D21763FFFFE70263CF41112317E2
:10C3E000B100894597000000E780C0F68347E1006F
:10C3F0002300F5008347F100A300F5004101176316
:10C40000FFFF670003CF1763FFFFE70243CC93D71B
:10C410008500A2054111DD8D2317B10089459700E4
:10C420000000E78020F38347E1002300F500834705
:10C43000F100A300F50041011763FFFF670063CB24
:10C440001763FFFFE702A3C81397850193D7850100
:10C45000C166938606F0D98F13D78500758FD98F63
:10C46000A2053707FF00F98D4111DD8D2EC69145DC
:10C4700097000000E78000EE6C0011469730010045
:10C48000E78060AB41011763FFFF670083C6176356
:10C49000FFFFE702C3C31C41854503C407009700A3
:10C4A0000000E78080E622851763FFFF670063C412
:10C4B0001763FFFFE702A3C11C414111894503C770
:10C4C000070083C717002307E100A307F1009700C7
:10C4D0000000E78080E30355E10041011763FFFF9F
:10C4E000670023C11763FFFFE70263BE1C414111D0
:10C4F000894503C7070083C717002307E100A30787
:10C50000F10097000000E78040E08357E10041011F
:10C5100013D58700A2075D8D420541811763FFFF98
:10C52000670023BD1763FFFFE70263BA0C414111A7
:10C530002A841146680097300100E780C09F91452A
:10C54000228597000000E78040DCB247C1669386F1
:10C5500006F01397870113D58701598D13D78700EC
:10C56000758F598DA2073707FF00F98F5D8D410147
:10C570001763FFFF6700E3B71C45BE950CC18280BF
:10C58000AE87944391E6584101EF0CC15CC18280B3
:10C5900003C7570013671700A382E700B687D5B714
:10C5A0000CC3EDB7AA87084119CD1841D44398C3ED
:10C5B0006313D500D8C32A87034657009376160025
:10C5C00081E6232007008280944381CA8C4203A81D
:10C5D00047008CC363930601CCC3799A14C3A302AA
:10C5E000C7003687D1BF1C45DC471D8DB777DBB64A
:10C5F000938777DB09853305F50242054181828007
:10C60000F147B385F50248452E9582808347450062
:10C6100085072302F50082801763FFFFE70223AB43
:10C620002A8409E41763FFFF6700A3AC8347440033
:10C63000F5DBFD1793F7F70F2302F400E5F71C4431
:10C6400003D7270005072391E700DC4399C3228520
:10C6500082974C4889CD83475400898B99E71C44C5
:10C6600022859C479C439C478297232A04000040D4
:10C67000232004007DB71763FFFFE70243A583571C
:10C68000250041112EC681EB01442285410117632B
:10C69000FFFF670003A6035705008147F146E30546
:10C6A000F7FEB385D702404585072E9483454400A5
:10C6B00008C4F5F5B247AA8481E7232A040009A833
:10C6C0001C456C0022859C439C43829748C84DDDE5
:10C6D00085472312F400B2472320040023180400E6
:10C6E0002319F4005C485CC483D72400FD17239110
:10C6F000F40061BF1763FFFFE702639D9797FF1F79
:10C700009387877F8843232605002324050041055E
:10C7100097100100E78000B31763FFFF6700639D78
:10C720001763FFFFE702A39A1794FF1F1304C47C4B
:10C730001C40411199CF9C472300B5002AC65CC11B
:10C7400097000000E78040FB1C40DC4399C3324562
:10C75000829741011763FFFF6700A39903474500D4
:10C7600029E3584DAA877D551DCF1763FFFFE702C8
:10C7700003961CC3DC479796FF1F23AFE676F1565E
:10C78000130507012390D700970500009385050244
:10C7900097100100E780A09801451763FFFF67002D
:10C7A00043957D55828082801763FFFFE7022392C5
:10C7B00001116146814528009760FFFFE7802094C2
:10C7C0009797FF1F938747739C4328009305F00FAB
:10C7D000DC473EC697000000E780C0F405611763A0
:10C7E000FFFF670003919797FF1F9387E7709C43B4
:10C7F000D847A1679387C702631EF70A397106DE1F
:10C8000022DC26DA80004AD84ED652D456D232855F
:10C81000B28497000000E780C0C7AA8926859700E8
:10C820000000E78020C92318A4FC2685970000009B
:10C83000E78040C82319A4FC268597000000E78004
:10C8400060C783D744000A8A231AA4FC858393F720
:10C85000F70F230EF4FC8607BD0793F7073F33015C
:10C86000F1408A8A01498347C4FD6367F902CE8596
:10C87000130584FC232C54FD97000000E78080EA18
:10C880005281130104FCF2506254D2544259B259FD
:10C89000225A925A21618280268597000000E78003
:10C8A00060C193171900D69705092390A700137943
:10C8B000F90F55BF82809797FF1F9387E7639C43CB
:10C8C000D847A1679387A702631AF70A397106DE72
:10C8D00022DC26DA80004AD84ED652D456D232858F
:10C8E000B28497000000E780C0BAAA892685970025
:10C8F0000000E78020BCFD572318A4FC26852319DF
:10C90000F4FC97000000E780E0BA83D744000A8A6D
:10C91000231AA4FC858393F7F70F230EF4FC8607F4
:10C92000BD0793F7073F3301F1408A8A01498347E6
:10C93000C4FD6367F902CE85130584FC232C54FDE6
:10C9400097000000E78000DE5281130104FCF250E2
:10C950006254D2544259B259225A925A2161828069
:10C96000268597000000E780E0B493171900D6975A
:10C9700005092390A7001379F90F55BF8280979777
:10C98000FF1F938767579C43D847A16789076310A8
:10C99000F70A397106DE22DC26DA80004AD84ED644
:10C9A00052D456D23285328997000000E78060AEBB
:10C9B000AA894A8597000000E780C0AF83574900E5
:10C9C0000A8A2318A4FC858393F7F70F230CF4FC41
:10C9D0008607BD0793F7073F3301F1408A8A8144F8
:10C9E000834784FD63E7F402CE85130584FC232A84
:10C9F00054FD97000000E780E0D25281130104FC4F
:10CA0000F2506254D2544259B259225A925A216178
:10CA100082804A8597000000E780C0A993971400A0
:10CA2000D69785042390A70093F4F40F55BF828016
:10CA30009797FF1F9387474C9C43D847A1679387DD
:10CA4000E704631EF70A397106DE22DC26DA80006D
:10CA50004AD84ED652D456D23285B28497000000BE
:10CA6000E78020A3AA89268597000000E78080A49C
:10CA70002318A4FC268597000000E780A0A3231AB2
:10CA8000A4FC268597000000E780C0A283D744005D
:10CA90000A8A2319A4FC858393F7F70F230EF4FC6D
:10CAA0008607BD0793F7073F3301F1408A8A0149A2
:10CAB0008347C4FD6367F902CE85130584FC232CEC
:10CAC00054FD97000000E780E0C55281130104FC8B
:10CAD000F2506254D2544259B259225A925A2161A8
:10CAE0008280268597000000E780C09C931719007C
:10CAF000D69705092390A7001379F90F55BF8280B7
:10CB00009797FF1F9387473F9C43D847A167938719
:10CB1000C704631AF70A397106DE22DC26DA8000C0
:10CB20004AD84ED652D456D23285B28497000000ED
:10CB3000E7802096AA89268597000000E7808097E5
:10CB4000FD572318A4FC2685231AF4FC9700000047
:10CB5000E780409683D744000A8A2319A4FC858382
:10CB600093F7F70F230EF4FC8607BD0793F7073FF3
:10CB70003301F1408A8A01498347C4FD6367F902A2
:10CB8000CE85130584FC232C54FD97000000E7801C
:10CB900060B95281130104FCF2506254D2544259DC
:10CBA000B259225A925A216182802685970000004C
:10CBB000E780409093171900D69705092390A700A6
:10CBC0001379F90F55BF82809797FF1F9387C7325C
:10CBD0009C43D847A167DD076317F7041753FFFF8E
:10CBE000E702E34E79713285328497000000E780D6
:10CBF000408A2AC6228597000000E780A08B231177
:10CC0000A102228597000000E780A088B24523009A
:10CC1000A102280897000000E780C0B045611753C3
:10CC2000FFFF6700034D82809797FF1F9387C72CF4
:10CC30009C43D847A167938787046317F70417536A
:10CC4000FFFFE702C3487971328532849700000004
:10CC5000E78020842AC6228597000000E78080852F
:10CC60002311A102228597000000E7808082B2454F
:10CC70002300A102280897000000E780A0AA4561D0
:10CC80001753FFFF6700E34682809797FF1F938744
:10CC9000A7269C43D847A1679387A7046312F7028E
:10CCA0001753FFFFE702A3420111280081459700B7
:10CCB0000000E78020A705611753FFFF670063436B
:10CCC00082809797FF1F938727239C43D847A167AC
:10CCD000938757026319F7021753FFFFE702233FB9
:10CCE0000111328597F0FFFFE780A07A2308A100A9
:10CCF0008145280097000000E780C0A20561175316
:10CD0000FFFF6700033F82809797FF1F9387C71E2F
:10CD10009C43D847A1679387E702631BF704175327
:10CD2000FFFFE702C33A01113285328497F0FFFF1B
:10CD3000E7804078AA84228597F0FFFFE78080771C
:10CD4000854709E9228597F0FFFFE7808074420557
:10CD5000B337A00028008145231891003ECA9700F0
:10CD60000000E780209C05611753FFFF67006338D0
:10CD700082809797FF1F938727189C43D84799472E
:10CD80006313F7081753FFFFE702633479713285A5
:10CD9000328497F0FFFFE780C06F2AC6228597F0A4
:10CDA000FFFFE78020712310A102228597F0FFFF8B
:10CDB000E780206E2301A102228597F0FFFFE78024
:10CDC000406DA301A102228597F0FFFFE780606C10
:10CDD0002302A102228597F0FFFFE780806B2313D7
:10CDE000A102228597F0FFFFE780A06AB2452314D5
:10CDF000A102280897000000E780C0924561175300
:10CE0000FFFF6700032F82809797FF1F9387C70E4E
:10CE10009C43D847A1679387C7036313F708175349
:10CE2000FFFFE702C32A79713285328497F0FFFF52
:10CE3000E78020662AC6228597F0FFFFE78080679B
:10CE40002310A102228597F0FFFFE780A06623113F
:10CE5000A102228597F0FFFFE780A0632302A102D1
:10CE6000228597F0FFFFE780C062A302A10222851E
:10CE700097F0FFFFE780E0612303A102228597F08E
:10CE8000FFFFE7800061B245A303A10228089700D5
:10CE90000000E780208945611753FFFF6700632585
:10CEA00082801753FFFFE702832201112A8497F043
:10CEB000FFFFE780005EAA84228597F0FFFFE780EE
:10CEC000605F228597F0FFFFE780C05E0357440054
:10CED0008D4763F7E700228597F0FFFFE780805DCD
:10CEE000228597F0FFFFE780E05C2800A685970089
:10CEF0000000E780208305611753FFFF6700631F71
:10CF00009797FF1F938747FF9C43D847A167FD076B
:10CF1000631FF7001753FFFFE702631B328597007B
:10CF20000000E78040F81753FFFF6700831C8280F2
:10CF30009797FF1F938747FC9C43D847A167E50756
:10CF40006315F7081753FFFFE702631879713285FD
:10CF5000328497F0FFFFE780C0532AC6228597F0FE
:10CF6000FFFFE7802055228597F0FFFFE780805480
:10CF70002310A102228597F0FFFFE780A0535205FE
:10CF800051812311A10222852302010297F0FFFFA4
:10CF9000E7802050A302A102228597F0FFFFE780DF
:10CFA000404F2303A102228597F0FFFFE780604EE8
:10CFB000B245A303A102280897F0FFFFE78080761F
:10CFC00045611753FFFF6700C31282809797FF1FC9
:10CFD000938787F29C43D847A1679387E703631F32
:10CFE000F7001753FFFFE702830E3285970000001A
:10CFF000E78060EB1753FFFF6700A30F82809797CE
:10D00000FF1F938767EF9C43D847A1679387470427
:10D01000631EF7021753FFFFE702630B7971328536
:10D02000328497F0FFFFE780C0462AC6228597F03A
:10D03000FFFFE7802048B245280897F0FFFFE78010
:10D04000606E45611753FFFF6700A30A82809797C0
:10D05000FF1F938767EA9C43D847A167938787029E
:10D060006310F7041753FFFFE702630679713285F7
:10D07000328497F0FFFFE780C0412AC6228597F0EF
:10D08000FFFFE7800041B2452300A102280897F086
:10D09000FFFFE780206945611753FFFF67006305C5
:10D0A00082801753FFFFE7028302011197F0FFFF11
:10D0B000E780203EAA85280097F0FFFFE780806682
:10D0C00005611753FFFF6700C3029797FF1F938700
:10D0D000A7E29C43D847A167D107631FF700175306
:10D0E000FFFFE702C3FE328597000000E780A0FB48
:10D0F0001753FFFF6700E3FF82809797FF1F938717
:10D10000A7DF9C43D847A167C507631FF7001753E4
:10D11000FFFFE702C3FB328597000000E780A0F81D
:10D120001753FFFF6700E3FC82809797FF1F9387E9
:10D13000A7DC9C43D847A167B907631FF7001753C3
:10D14000FFFFE702C3F8328597000000E780A0F5F3
:10D150001753FFFF6700E3F982809797FF1F9387BC
:10D16000A7D99C43D847A167AD07631FF7001753A2
:10D17000FFFFE702C3F5328597000000E780A0F2C9
:10D180001753FFFF6700E3F682809797FF1F93878F
:10D19000A7D69C43D84789476318F7021753FFFF68
:10D1A000E702E3F20111328532C897F0FFFFE78012
:10D1B000402EAA85280097F0FFFFE780A056056162
:10D1C0001753FFFF6700E3F282809797FF1F938753
:10D1D000A7D29C43D847A1678D076311F704175363
:10D1E000FFFFE702C3EE01113285328497F0FFFFA3
:10D1F000E780202A13066100AA844C00228597301C
:10D200000000E780C0232800A68597F0FFFFE78095
:10D21000605105611753FFFF6700A3ED8280979768
:10D22000FF1F9387A7CD9C4381CFDC4391CB17533E
:10D23000FFFFE702C3E982971753FFFF670063EB25
:10D2400082801753FFFFE70283E879713C08AE84C0
:10D250003ED2A165B7070A002A843ED448103C0894
:10D26000DD053ED636C432C63AC297D0FFFFE7800E
:10D27000E02F12474810BA8597F0FFFFE780C013F0
:10D2800032464810B28597F0FFFFE780E014A246CF
:10D290004810B68597F0FFFFE78000125010014755
:10D2A0008146A685228597D0FFFFE78080514561A2
:10D2B0001753FFFF6700E3E31753FFFFE70223E184
:10D2C00001117C000329C501AE843ECAA165B707E0
:10D2D00007002A843ECC48087C00C5053ECE97D086
:10D2E000FFFFE780A0288345D900480897F0FFFF9B
:10D2F000E780800C500801478146A685228597D09B
:10D30000FFFFE780004C05611753FFFF670063DEF6
:10D310001753FFFFE702A3DB83C7950093F7F707D7
:10D32000A384F50097000000E78040F91753FFFF42
:10D33000670023DC1753FFFFE70263D979713C08CC
:10D34000AE843ED2A165B70709002A843ED44810B6
:10D350003C08938545043ED632C636C497D0FFFFBD
:10D36000E780C020A2464810B68597F0FFFFE7800F
:10D37000A00432464810B28597F0FFFFE780C00551
:10D38000501001478146A685228597D0FFFFE78090
:10D39000404345611753FFFF6700A3D51753FFFFB5
:10D3A000E702E3D283C7950041112A8493F7F70778
:10D3B000A384F50032852EC697F0FFFFE780800F2B
:10D3C00085672AC46370F50297700000E78020E942
:10D3D0002246B24509ED114781462285970000009B
:10D3E000E78060E641011753FFFF670083D00147E4
:10D3F0008346F501DDB71753FFFFE702A3CB011109
:10D400003C003ECAB7070A003ECC3C003ECE83C774
:10D410009500AA89328593F7F707A384F5002E8437
:10D4200097F0FFFFE78000098567637DF504A1653C
:10D43000AA8493858504480897D0FFFFE7800013EE
:10D44000268597700000E78080E12A8929E19145CF
:10D45000480897F0FFFFE78020F6A685480897F078
:10D46000FFFFE78060F7CA85480897F0FFFFE78075
:10D47000A0F4014781465008A2854E8597D0FFFF52
:10D48000E780203405611753FFFF6700E3C581453E
:10D49000480897F0FFFFE78020F20349090275BFB3
:10D4A0001753FFFFE70203C179711C103ECAB7078B
:10D4B0000F003ECC404D1C10AA84AE894808994507
:10D4C00032C636893ECE97D0FFFFE780200A32462B
:10D4D0004808B28597F0FFFFE78000EE630C090271
:10D4E000A545480897F0FFFFE780C0E62546CA85B6
:10D4F00097200100E78020A4500801478146CE858F
:10D50000268597D0FFFFE780C02B45611753FFFFAB
:10D51000670083BD8355C402480897F0FFFFE7808A
:10D52000A0EB0355E402814505C5854785456301A8
:10D53000F502C167FD179305F00F630BF5007D152C
:10D5400097700000E780208E9305150093F5F50F86
:10D55000480897F0FFFFE78020E68345040348086A
:10D5600097F0FFFFE78040E583451403480897F0F4
:10D57000FFFFE78060E483552403480897F0FFFF2E
:10D58000E78080E583554403480897F0FFFFE78074
:10D59000A0E49DB71753FFFFE70263B383C795006D
:10D5A0008146014693F7F707A384F5009700000032
:10D5B000E78040EF1753FFFF6700A3B31753FFFF48
:10D5C000E702E3B079713E841C103ECA2E89B7078A
:10D5D0000F00A1653ECCFD051C10AA84480842C07E
:10D5E0003AC23ECE36C432C697D0FFFFE78000F87D
:10D5F00032464808B28597F0FFFFE780E0DBA2469D
:10D600004808B68597F0FFFFE78000DD124748081D
:10D61000BA8597F0FFFFE78020DC0248630C080220
:10D620009145480897F0FFFFE780C0D21146A285D8
:10D6300097200100E7802090500801478146CA8565
:10D64000268597D0FFFFE780C01745611753FFFF7E
:10D65000670023AA8945480897F0FFFFE78080CF3D
:10D66000834704002300F50083471400A300F5005E
:10D67000E1B71753FFFFE702E3A383C7950001114A
:10D680002A8A93F7F707A384F5003285AE8432C661
:10D6900097F0FFFFE78000E232462A89328597F053
:10D6A000FFFFE78000DF85676373F902AA894A8577
:10D6B00097700000E780A0BA2A8419ED11478146CF
:10D6C0004A86A685528597000000E780C0B70561AD
:10D6D0001753FFFF670043A19387E9FF93F7F70F05
:10D6E0000547E366F7FE8347F50195EB8947E3803D
:10D6F000F9FE8346F401528501474A86A6859700C4
:10D700000000E78040B4A167D90748083ECC230A4F
:10D71000010002CE97000000E780A0B04DBF639EDD
:10D72000E7008947639EF90093071020231FF50047
:10D7300097700000E780C0B76DBF0947E39BE7FA29
:10D740008D47E398F9FA228597700000E78080DF23
:10D750009797FF1F938787999C4399E79797FF1F98
:10D76000938787829C4399C703D504009780000064
:10D77000E780A0CE231F040022855DBF1753FFFF63
:10D78000E702E39401113C003ECAB7070B003ECC10
:10D790003C003ECE83C795002A89328593F7F70770
:10D7A000A384F500AE8497F0FFFFE780A0D0931725
:10D7B0000501C187635AF006A1652A849385E502B5
:10D7C000480897D0FFFFE78060DAA285480897F005
:10D7D000FFFFE78060C09787FF1F9387E77A9C432E
:10D7E000A9EB01449375F40F480897F0FFFFE78019
:10D7F000A0BC9355844093F5F50F480897F0FFFFC0
:10D80000E78080BB9355044193F5F50F480897F0E6
:10D81000FFFFE78060BA014781465008A6854A8528
:10D8200097D0FFFFE780E0F905611753FFFF67001E
:10D83000438C416585460546A2857D1597500000BD
:10D84000E78060BD59DD510597000100E780808FBA
:10D85000130440063344850271B71753FFFFE702F4
:10D8600003870111B70706003EC683C795002164F0
:10D870002A8993F7F707A384F500AE84280093055F
:10D88000A4040AC40AC897D0FFFFE78020CE300066
:10D8900001478146A6854A8597D0FFFFE78060F261
:10D8A00097E0FFFFE780801513049404480822CC1A
:10D8B000230A010002CE97000000E78080960561F0
:10D8C0001753FFFF6700E3821743FFFFE702837EE2
:10D8D000C1642A8901449799FF1F9389A982130A79
:10D8E0008002FD1497E0FFFFE78080C16347A4003A
:10D8F00001451743FFFF6700237FB307440303A7D6
:10D90000C90ABA9703D707006306970083D7270091
:10D91000638427010504F9B70545E1BF1743FFFFFD
:10D92000E70243792A8A2E8999C123A005008149FB
:10D930008144978AFF1F938AAA5C614B97E0FFFF9F
:10D94000E78040C263C7A4004E851743FFFF67000E
:10D95000A3793384640383A70A003E9483570400A9
:10D9600099E763040900232089008504C1BF41466B
:10D97000D2851305440097100100E780605975F5C2
:10D98000A289E5B71743FFFFE702C37239717C082C
:10D990003ED4B7070A003ED67C083ED883C7950020
:10D9A0002A8A328593F7F707A384F5002E8932C6B9
:10D9B00097F0FFFFE78000B085676373F508324694
:10D9C000AA84328597F0FFFFE780A0AC8547AA893B
:10D9D00063E8A706A16593858504281097D0FFFF0B
:10D9E000E780C0B8268597700000E78040872A84CA
:10D9F00029ED9145281097F0FFFFE780E09BA68571
:10DA0000281097F0FFFFE780209DCE85281097F023
:10DA1000FFFFE780609A014781463010CA85528532
:10DA200097D0FFFFE780E0D9A16793877704481874
:10DA30003EDC230A010202DE97F0FFFFE780607EF2
:10DA400021611743FFFF6700236A8145281097F083
:10DA5000FFFFE7806096A685281097F0FFFFE7801C
:10DA6000A0979797FF1F9387A7A09C4381CB228500
:10DA70006389090097D00000E780402483450402B1
:10DA800071B797D00000E780C022CDBF1743FFFFDA
:10DA9000E702436283C795004111AA8993F7F7070C
:10DAA000A384F5003285AE84328A97F0FFFFE780C9
:10DAB00060A08567637FF5022A8997600000E78090
:10DAC000007A2A84914631C58347F501054763876B
:10DAD000E70291C70D476366F704AD461DA893059D
:10DAE000050303250A00414697100100E7804042E4
:10DAF0000DE941011743FFFF6700035F9305950898
:10DB000003250A00414697100100E78060408146E6
:10DB100069F54A86A6854E8597000000E780C0819A
:10DB2000C9BF83250A001305940897700000E78099
:10DB3000A02919C1C146F1BF9787FF1F9387075BD3
:10DB40009C4399E79787FF1F938707449C4399C796
:10DB5000228597800000E780208A69FD8547A30F12
:10DB6000F400228597B00000E780608422859760EA
:10DB70000000E780E0734E8581464A86A68597F0CF
:10DB8000FFFFE780607BA1679387570448003EC48E
:10DB90002302010002C697F0FFFFE780806891BF73
:10DBA0001743FFFFE702235083C795004111AA895D
:10DBB00093F7F707A384F50032852E89B28A97F090
:10DBC000FFFFE780208F85676374F50EAA84976056
:10DBD0000000E780C0682A840DED416B014A978BF5
:10DBE000FF1F938B2B52130C400E7D1B19A833047F
:10DBF0008A0383A70B0B3E948357C4016383670595
:10DC0000050A97E0FFFFE780A08EE342AAFE954653
:10DC10000DA08357C501639697029305050303A5DD
:10DC20000A00414697100100E780802E994611E1D5
:10DC300081462686CA854E8597F0FFFFE780C06F34
:10DC400085A883A50A001305040397700000E780E8
:10DC5000A017C14679FD2285231E940097A00000DD
:10DC6000E780E074228597600000E7806064978712
:10DC7000FF1F9387E77F9C43A9C3230004022285EB
:10DC800097D00000E78040F04E8581462686CA8501
:10DC900097F0FFFFE780406AA16793870704480079
:10DCA0003EC42302010002C697F0FFFFE7806057E1
:10DCB00041011743FFFF6700834289472300F402B5
:10DCC000E1B7397106DE22DC4AD8800052D456D240
:10DCD0005AD026DA4ED65ECE2E8A32892A8B97D03B
:10DCE000FFFFE780E07D0605710541998A8A3301CF
:10DCF000A140232224FC231404FC97D0FFFFE780DB
:10DD0000207C83479A000605350593F7F70723150E
:10DD1000A4FCA304FA004A85232624FC97E0FFFF15
:10DD2000E780407993170501C1876340F00256816F
:10DD3000130104FCF2506254D2544259B259225A8F
:10DD4000925A025BF24B21618280AA844A8597E055
:10DD5000FFFFE7802076AA894A8597E0FFFFE780EA
:10DD60006075A1659385C5022A89130544FC97C097
:10DD7000FFFFE780A07F268597C0FFFFE780E07365
:10DD8000854511C94A86CE8597C0FFFFE780606D43
:10DD9000AA8B21E98945130544FC97E0FFFFE78042
:10DDA000A061A685130544FC97E0FFFFE780C062F1
:10DDB000CE85130544FC97E0FFFFE780E061CA854C
:10DDC000130544FC97E0FFFFE780006101478146AF
:10DDD000130644FCD2855A8597D0FFFFE780609EEA
:10DDE000B9B78145130544FC97E0FFFFE780C05CAD
:10DDF000A685130544FC97E0FFFFE780E05DCE8534
:10DE0000130544FC97E0FFFFE780005DCA8513051A
:10DE100044FC97E0FFFFE780205C814497D0FFFF40
:10DE2000E780006AE3D4A4FA83A70B0113971400D8
:10DE3000BA9783D5070099C5130544FC97E0FFFF07
:10DE4000E78080598504D9BF797106D622D44AD09B
:10DE500000184ECE52CC56CA26D25AC8AE89328944
:10DE6000AA8A97D0FFFFE780A0650605690541995A
:10DE70000A8A3301A140232A24FC231C04FC97D0E6
:10DE8000FFFFE780E06383C7990006052D0593F740
:10DE9000F707231DA4FCA384F9004A85232E24FC44
:10DEA00097E0FFFFE780006193170501C187634F8B
:10DEB000F0005281130104FDB250225492540259D1
:10DEC000F249624AD24A424B45618280AA844A851D
:10DED00097E0FFFFE780005EA1659385A5022A8990
:10DEE000130544FD97C0FFFFE7804068268597C073
:10DEF000FFFFE780805C854509C9CA8597C0FFFFA1
:10DF0000E78020592A8B29E18945130544FD97E0D4
:10DF1000FFFFE780604AA685130544FD97E0FFFFF9
:10DF2000E780804BCA85130544FD97E0FFFFE7803B
:10DF3000A04A01478146130644FDCE85568597D0F9
:10DF4000FFFFE7800088B5B78145130544FD97E0E2
:10DF5000FFFFE7806046A685130544FD97E0FFFFBD
:10DF6000E7808047CA85130544FD97E0FFFFE780FF
:10DF7000A046814497D0FFFFE7808054E3DBA4FAFA
:10DF800083270B0113971400BA9783D5070099C50F
:10DF9000130544FD97E0FFFFE78000448504D9BFE7
:10DFA0001743FFFFE702A31283474500404DD5EF1B
:10DFB000FD575DC48346940009476363D70A03464F
:10DFC000B400854663EEC6088306E40063CA06080B
:10DFD0005C45F9562390D7009787FF1F83C787F2C8
:10DFE00099E3A304E4009787FF1F9387E7F99C4315
:10DFF00081E78947A306F4009787FF1F9387474768
:10E000009C4381E789472306F40097050000938528
:10E010004506AA841305040197F00000E78020104C
:10E02000FD57231AF40281471CDC01489787FF1F24
:10E0300023A687EC9787FF1F938787EC232E040383
:10E0400004C0804397D0FFFFE780C051614633068C
:10E05000C502814522859740FFFFE780400A81473E
:10E060003E851743FFFF6700C308FD57D5BF174321
:10E07000FFFFE702C3052A840355450297600000AD
:10E08000E780E01D19E5231E04001743FFFF67002A
:10E0900043068357E401F5DB930504FF17450100B0
:10E0A0001305457797E00000E780E014F9BF1743B8
:10E0B000FFFFE702C3012E89A16541119385E503A6
:10E0C0002A8436C432C6BE843AC297C0FFFFE780B6
:10E0D000E04912472285BA8597E0FFFFE780C02D0F
:10E0E00032462285B28597E0FFFFE780E02EA24608
:10E0F0002285B68597E0FFFFE780002E63030902C3
:10E100009145228597E0FFFFE780C0241146A68550
:10E1100097100100E78020E241011743FFFF6700ED
:10E1200043FD8945228597E0FFFFE780A02283C752
:10E1300004002300F50083C71400A300F500E9BF25
:10E140001743FFFFE702A3F883C79500444D054737
:10E1500093F7F707A384F5001C42411183C707001A
:10E160006367F7062E842A89B1C003C7D400630F02
:10E17000F7021787FF1F130727E1184305C3A3867C
:10E18000F40097A00000E780404A83C7D40099E7D5
:10E1900041657D1597400000E780403083D7240318
:10E1A000918B89C797E00000E780C0134A85A2855C
:10E1B00097F0FFFFE7808010A167C10748003EC4C9
:10E1C0002302010002C697F0FFFFE78080054101AE
:10E1D0001743FFFF6700E3F11743FFFFE70223EF59
:10E1E00003D745008D47AA8441112E8432892E859C
:10E1F00063E3E70297E0FFFFE780C02BAA852300D7
:10E200000900268597C0FFFFE780A028410117433A
:10E21000FFFF670003EE97E0FFFFE780A0292AC613
:10E22000228597E0FFFFE780E028B24585472A86F0
:10E230002300F900268597C0FFFFE7808022F9B709
:10E24000397106DE22DC26DA80004ED652D456D250
:10E250004AD85AD05ECEAE89B284AA8A97D0FFFF40
:10E26000E780002506051305250241990A8A330136
:10E27000A140232224FC231404FC97D0FFFFE78055
:10E28000202383C7990006054D0593F7F70723154B
:10E29000A4FCA384F9002685232624FC97E0FFFF35
:10E2A000E780402193170501C1876340F002528146
:10E2B000130104FCF2506254D2544259B259225A0A
:10E2C000925A025BF24B21618280AA8B03AB04005D
:10E2D00097C0FFFFE780601E51E583D744000149E6
:10E2E0008544F11793B71700A301F4FC834734FC6E
:10E2F000A165C9C79385E504130544FC97C0FFFFDA
:10E30000E780C026A685130544FC97E0FFFFE78061
:10E31000A00ADE85130544FC97E0FFFFE780C00BF1
:10E32000834734FC114691E30946DA85130544FC22
:10E3300097E0FFFFE78060058144630A0900416BB5
:10E340007D1B97D0FFFFE780A01663CCA402014796
:10E350008146130644FCCE85568597C0FFFFE780B3
:10E360004046B1B7A685130634FC97000000E7804D
:10E37000E0E6933415002A8986048DBF9385C50491
:10E38000A5BF8327C90013971400BA9783D5070048
:10E3900063886501130544FC97E0FFFFE780C00335
:10E3A000850445B71743FFFFE702E3CF79711C10DF
:10E3B0003EC4B7070F003EC61C103EC883C7950079
:10E3C000AA8A328593F7F707A384F500AE893284D1
:10E3D00097E0FFFFE780000E93170501C187635A9E
:10E3E000F0062A8A228597E0FFFFE780A00C2A89A1
:10E3F0005285032B040097C0FFFFE780000C39ED26
:10E400008357440081440544F11793B71700A303D1
:10E41000F10083457100DA872287CA865286280078
:10E4200097000000E780E0C8014781463000CE85B4
:10E43000568597C0FFFFE780C038A1679387D70351
:10E4400048083ECC230A810026CE97F0FFFFE780E4
:10E4500040DD45611743FFFF670063C8A2851306CF
:10E46000710097000000E78060D7AA84094455D165
:10E470003544E30055FB4A8597F0FFFFE7800045F0
:10E480000D4441D9014497D0FFFFE7806002634DFE
:10E49000A400C16B0144FD1B97D0FFFFE780400142
:10E4A000634EA4001544B5B7DC4413171400BA97A3
:10E4B00083D70700638327030504F1B7D844931774
:10E4C0001400BA9703D70700631B77012390270135
:10E4D000268597A00000E78080DB01441DBF05046E
:10E4E00065BF1743FFFFE702E3BC83C795004111F7
:10E4F0002A8A93F7F707A384F50032852E893284A0
:10E5000097E0FFFFE78000FB93170501C187635386
:10E51000F006AA89228597E0FFFFE780A0F9231182
:10E52000A1004E85832A040097C0FFFFE780E0F832
:10E5300039E58357440085440144F11793B7170028
:10E54000A300F1000348110003572100D68752852C
:10E55000CE862686CA8597F0FFFFE7806006A16712
:10E56000F10748003EC42302910022C697F0FFFF46
:10E57000E78020CB41011743FFFF6700E3B6A28588
:10E580001306110097000000E78040C52A848944E3
:10E5900055D98357210011678544BA97C20711677F
:10E5A000C1831307F7EFE36FF7F89787FF1F938790
:10E5B000E7B39C4381CB85451305210097500000AC
:10E5C000E7802075835521002285814497C0FFFF95
:10E5D000E78040E525D923100500228597A000009B
:10E5E000E78040CD85B71743FFFFE702C3AB83C782
:10E5F000950041112A8B93F7F707A384F500328524
:10E600002E8A328497E0FFFFE780C0EA9317050166
:10E61000C1876351F006AA8A228597E0FFFFE78051
:10E6200060E92A895685832B040097C0FFFFE780A5
:10E63000C0E831E58357440081440544F11793B79E
:10E640001700A301F10003483100DE875A854A878D
:10E65000D6862286D28597F0FFFFE78060F6A16715
:10E66000ED0748003EC42302810026C697F0FFFF55
:10E67000E78020BB41011743FFFF670043A6A28547
:10E680001306310097000000E78040B5AA840944D2
:10E690005DD99167CA97C2071167C1831307F7EF66
:10E6A0000544E362F7FACA8597C0FFFFE78080D789
:10E6B000014451F9814997D0FFFFE78060E063DBB7
:10E6C000A900984893971900BA9703D7070005EF58
:10E6D0002390270197D0FFFFE78080DE1544E38475
:10E6E000A9F6268597A00000E780C0BC9787FF1F8A
:10E6F0009387C79F9C430144B9D74A859750000030
:10E70000E780C05889B785097DB71743FFFFE70247
:10E71000639A79713E847C083EC82E8AB70714003C
:10E72000A1653ECAE5057C08AA89080836C4428965
:10E7300032C6BA8AC6843ECC97C0FFFFE78000E3AA
:10E74000CA85080897E0FFFFE78000C7324608083F
:10E75000B28597E0FFFFE78020C8A246630A09045C
:10E760009D45080897E0FFFFE780C0BE1D46814534
:10E770009740FFFFE780A09863890A089145080841
:10E7800097E0FFFFE78000BD1146A68597000100D6
:10E79000E780607A100801478146D2854E8597C090
:10E7A000FFFFE780000245611743FFFF6700C39347
:10E7B000B685080897E0FFFFE78000C21C40080804
:10E7C000D8439355C701858912075183B205D98D66
:10E7D00097E0FFFFE78040C01C40080883C5870022
:10E7E00097E0FFFFE78040BD1C40080883C5A700F5
:10E7F00097E0FFFFE78040BC1C40080883C59700F6
:10E8000097E0FFFFE78040BB85BF8945080897E098
:10E81000FFFFE78020B483C704002300F50083C70F
:10E820001400A300F500BDB71743FFFFE70283887C
:10E8300083C795004111AA8993F7F707A384F500D0
:10E840003285AE84328497E0FFFFE780A0C693173D
:10E850000501C187635DF0042A89032A040097C07B
:10E86000FFFFE78080C519E9835744000548F11789
:10E8700093B71700A307F100814631A81306F100F2
:10E88000A28597000000E78060951DC51C459DC7C7
:10E8900083D6470001480347F10093078500D288DB
:10E8A0004A86A6854E8597000000E78040E6410134
:10E8B0001743FFFF6700438309487DBF1D486DBFB5
:10E8C0001733FFFFE702037F65715C083EC4B7079B
:10E8D0007B013EC65C083EC883C795002A8A328504
:10E8E00093F7F707A384F500AE8997E0FFFFE78071
:10E8F00040BA8357E100E1C78945280097C0FFFF70
:10E90000E780C0C68145280097E0FFFFE780C0AAE6
:10E9100097C0FFFFE780A0CC9787FF1F938747B57D
:10E920009C431774FF1F0344E45DAA8433348000C2
:10E9300099C3136424009777FF1F9387E7649C4370
:10E9400099C3136444009777FF1F9387277A9C43EA
:10E9500099C31364840083D504002800014997E01B
:10E96000FFFFE78060A783D52400280097E0FFFF22
:10E97000E78080A683D54400280097E0FFFFE7806A
:10E98000A0A597D0FFFFE780A0AE93150501C18138
:10E99000280097E0FFFFE78020A4A285280097E0E9
:10E9A000FFFFE78060A39C446360F9020147814652
:10E9B0003000CE85528597C0FFFFE78080E0596127
:10E9C0001733FFFF67004372DC441314490028002B
:10E9D0003E9497E0FFFFE78060968347440003473B
:10E9E000540089070607BA978607E36AF5FC835542
:10E9F00024002800814A97E0FFFFE780E09D8345DF
:10EA00004400280097E0FFFFE780009B8345540007
:10EA1000280097E0FFFFE780209A8347440063C9FE
:10EA2000FA00814A8347540063C1FA020509A5BF71
:10EA30001C4413975A002800BA9783D50700850A0B
:10EA400097E0FFFFE7804099C9BF032BC40093976D
:10EA50005A0028003E9B83552B00850A97E0FFFF54
:10EA6000E780809783550B00280097E0FFFFE78041
:10EA7000A0964DBF1733FFFFE70263655C4993E73C
:10EA800017005CC997A00000E78020B61733FFFF8E
:10EA9000670023661733FFFFE70263632E84814517
:10EAA00097F0FFFFE780C0E705C583570500FD1716
:10EAB0002310F50009C4835725002310F4009700A4
:10EAC0000000E78060FB01451733FFFF67006362CA
:10EAD00031457DD823100400C5BF1733FFFFE7027F
:10EAE000635D83C7950041112A8A93F7F707A384D2
:10EAF000F50032852E89328497E0FFFFE780809B06
:10EB000093170501C1876356F006AA89C14522857E
:10EB100097E0FFFFE780A0802A8B4E85832A0400C0
:10EB200097C0FFFFE780609931E9835744002311C4
:10EB300001000544F11793B71700A300F1008144C9
:10EB40000348110003572100D6875285CE862286BE
:10EB5000CA8597F0FFFFE780A0A6A16793871702F9
:10EB600048003EC42302810026C697E0FFFFE780ED
:10EB7000406B41011733FFFF670003571306110075
:10EB8000A28597F0FFFFE7806065AA8409E523115D
:10EB90000100094475B7930521005A8597000000CC
:10EBA000E78080EF835721002A84D9DB9777FF1F06
:10EBB0009387C7539C4381CB85451305210097500C
:10EBC0000000E7800015835521002685314497C059
:10EBD000FFFFE78020852DD523100500268597901F
:10EBE0000000E780206D0144A1BF1733FFFFE7025B
:10EBF000034E41112E896C00AA8402C697F0FFFFD4
:10EC0000E78000D20DC10357050005072310E5007A
:10EC100097000000E78040E681473E8541011733B9
:10EC2000FFFF6700034D3247954765DBCA852685A0
:10EC300097300000E780400DC147E34005FE3244B5
:10EC4000854741462310F40083570900A685130524
:10EC500044002311F40097000100E780C02D2285B5
:10EC600045BF1733FFFFE702E34483C79500411117
:10EC7000AA8A93F7F707A384F5003285AE89328418
:10EC800097E0FFFFE780008393170501C187635674
:10EC9000F0062A8AC145228597D0FFFFE7802068C9
:10ECA000AA845285032B040097C0FFFFE780E08011
:10ECB00031E983574400231101008544F11793B7CC
:10ECC0001700A300F100014403481100035721007D
:10ECD000DA875685D2862686CE8597F0FFFFE780B5
:10ECE000208EA1679387070248003EC4230291004B
:10ECF00022C697E0FFFFE780C05241011733FFFFB4
:10ED00006700833EA2851306110097F0FFFFE7809E
:10ED1000E04C2A8409E523110100894475B7268552
:10ED20009305210097000000E78060ECAA8449FD6C
:10ED300083552100228597B0FFFFE780A06E49F53B
:10ED4000014997C0FFFFE780A077635DA9001848DD
:10ED500093171900BA9703D707000DEF0357210047
:10ED60002390E70097C0FFFFE780807563062503C7
:10ED70009777FF1F938787379C4399C703552100D7
:10ED800097500000E78080F0228597900000E78090
:10ED900060521DBF050975B795443DB705C193077E
:10EDA000F00F630FF500C547630CF5009307F5FFFF
:10EDB00005453315F5004205418182800145828079
:10EDC00041657D158280B9E91733FFFFE7022330E3
:10EDD00003450603328497000000E78060FC93053A
:10EDE000803EB305B502C205C18181CD0357E4025F
:10EDF000854763F8E7001305040197E00000E7800A
:10EE000020428357E40241677D176385E700FD17C1
:10EE10002317F4021733FFFF6700A32D82801733F7
:10EE2000FFFFE7024328004283C79500444D034992
:10EE3000140093F7F707A384F50083470400220921
:10EE400011673369F900A167B347F90041112A8BB3
:10EE5000AE8A63ECE70E834724001307C00EB91790
:10EE600093F7F70F6373F71003473400C14763EE5E
:10EE7000E70E834744001307E00793C70708637151
:10EE8000F70C8349840083477400A209B3E9F900B1
:10EE9000856763F7F90A034A6400834754004E8587
:10EEA000220A336AFA0097500000E780403B61C1B4
:10EEB00023962403834B3400137AFA00239A3403F5
:10EEC000238874032399440393890401631C090074
:10EED00023A60402239804024E8597E00000E780F1
:10EEE00060363DA0034924004A8597000000E78072
:10EEF00020EB2397A402834744004E85A388F402A5
:10EF0000E38D0BFCE30B09FC97E00000E780202F6A
:10EF100097900000E780007381460146D6855A85A8
:10EF200097E0FFFFE7800058A167938797033EC4EF
:10EF300023020100480002C697E0FFFFE780602E31
:10EF400041011733FFFF670083198544A286268697
:10EF5000D6855A8597E0FFFFE780C054A167938765
:10EF600097033EC423029100F1B7BD44C5B7914455
:10EF7000F1BF1733FFFFE702E31301111C08404DF7
:10EF80003EC2B7070F003EC41C083EC62A89AE89A0
:10EF900097C0FFFFE780A0DA585C1C5C6346B70EA1
:10EFA0006394E50063E2A70E3385A740B3B7A700DB
:10EFB000B305B7401306803E81469D8D9700010042
:10EFC000E78080B793140501C180A1659385C503CF
:10EFD000480097B0FFFFE78060598145480097D00F
:10EFE000FFFFE780603D83550404480097D0FFFF92
:10EFF000E780803E83552404480097D0FFFFE780D8
:10F00000A03D814589CCC167FD179305F00F63884A
:10F01000F400268597500000E780E0E0AA854800CC
:10F0200097D0FFFFE780403903554404814501CD67
:10F03000C167FD179305F00F6307F50097500000B7
:10F04000E78060DEAA85480097D0FFFFE780C036E2
:10F0500083456404480097D0FFFFE780E03583458F
:10F060007404480097D0FFFFE78000355000014747
:10F070008146CE854A8597B0FFFFE78080740561A1
:10F080001733FFFF67004306814481B71733FFFF43
:10F09000E702E30383C7950093F7F707A384F5001E
:10F0A00097000000E78020ED1733FFFF670063043F
:10F0B0001733FFFFE702030083C795004111404D5E
:10F0C00093F7F707A384F5002A8A3285B284AE89C4
:10F0D00097D0FFFFE780003E2A8B268597D0FFFF61
:10F0E000E780403D2A89268597D0FFFFE780603A78
:10F0F00093170B0163CA0702E177CA97C207C1835E
:10F10000116763E3E70293070910C207C18313077E
:10F11000B00F637BF70093170901C187AA8A634A7E
:10F12000F000C54763FE570141011733FFFF670039
:10F13000A3FB97B0FFFFE780C028E31725FFD5B7F3
:10F1400063080B0263060902814463890A02B70758
:10F150007F0023106405231124057CC05685970089
:10F160000000E780E0C39304803EB304950239A019
:10F17000B7077F00232004047CC081440355240486
:10F1800097E00000E780A0A3A1C497C0FFFFE7803D
:10F1900000BB269593D7F44133379500AE97BA97C5
:10F1A00008DC5CDCCE85528597000000E780A0DC9F
:10F1B00099E023220404A1679387B70348003EC463
:10F1C0002302010002C697E0FFFFE7808005A9BF88
:10F1D000814701481CDC232E0403E9B71733FFFFE6
:10F1E000E702E3EE97C0FFFFE780C037E147330552
:10F1F000F502914597500000E78000C5E55711C51D
:10F200009777FF1F23AEA7CE81473E851733FFFFB9
:10F21000670023EE85471777FF1F2305F7CE82800F
:10F220001733FFFFE702A3EA9777FF1F938707CD06
:10F2300080433DC0835704046390A706835724048A
:10F24000639CB7043689B28497C0FFFFE78020AF84
:10F250005C5C63C3B7046395B7001C5C63EEA702F4
:10F260008347640463F3F400A6872303F40483470D
:10F27000740463F39700A687A303F404835744043C
:10F2800041677D176385E70085072312F4043C443A
:10F2900081C7CA85268582971733FFFF670063E51C
:10F2A0009777FF1F938787C59C43014599C303C583
:10F2B000870082801733FFFFE70263E10111B70780
:10F2C00007003EC683C79500584D0AC493F7F70759
:10F2D0000AC8A384F5002A89AE8411CB1C4283C7D7
:10F2E00007002304F70097900000E78000342164B2
:10F2F00093055402280097B0FFFFE780202797006E
:10F300000000E78020FAAA85280097D0FFFFE78059
:10F31000A00A300001478146A6854A8597B0FFFFC5
:10F32000E780204A13044402480822CC230A010043
:10F3300002CE97E0FFFFE780C0EE05611733FFFFC5
:10F34000670023DB1733FFFFE70263D801117C005E
:10F350003ECAB70707003ECC7C003ECE83C795006F
:10F360002E84AA8493F7F707A384F500A1659385FB
:10F370005502480897B0FFFFE780401F9700000044
:10F38000E78040F2AA85480897D0FFFFE780C002D7
:10F39000500801478146A285268597B0FFFFE78088
:10F3A000404205611733FFFF6700A3D49777FF1F23
:10F3B0009387C7B49C43094599C303C597008280CE
:10F3C0009777FF1F938787B39C43094599C303C56C
:10F3D000D70082809777FF1F938747B29C430145F0
:10F3E00099C303C5A70082801733FFFFE70283CCD0
:10F3F0000111B70708003EC683C79500404D0AC4F7
:10F4000093F7F7070AC8A384F5002A89AE8429C4B4
:10F410001442854703C7060063E0E70A8347940068
:10F42000094681496380C702B307F740A304E4009B
:10F43000B339F00083C716002305F400979000004D
:10F44000E780A01E03572403058B19C763860900B4
:10F4500097D00000E78000E921649305840228002A
:10F4600097B0FFFFE780801097000000E78040F42E
:10F47000AA85280097D0FFFFE78000F497000000DE
:10F48000E78080F5AA85280097D0FFFFE780C0F2CB
:10F49000014781463000A6854A8597B0FFFFE78087
:10F4A000403213047402480822CC230A010002CE21
:10F4B00097E0FFFFE780E0D605611733FFFF6700A5
:10F4C000A3C21733FFFFE70283C001117C003ECACD
:10F4D000B70708003ECC7C003ECE83C795002E8443
:10F4E000AA8493F7F707A384F500A16593858502A5
:10F4F000480897B0FFFFE780600797000000E780AB
:10F5000020EBAA85480897D0FFFFE780E0EA970044
:10F510000000E78060ECAA85480897D0FFFFE780ED
:10F52000A0E9500801478146A285268597B0FFFFD4
:10F53000E780202905611733FFFF670083BB9777BA
:10F54000FF1F9387A79B9C43014599C303C5B70041
:10F5500082801733FFFFE70283B70111B707070067
:10F560003EC683C79500404D0AC493F7F7070AC803
:10F57000A384F5002A89AE8405C81C42054783C7C9
:10F5800007006368F7060347B400630FF700A3059D
:10F59000F40097900000E78040098347B400B9CF9A
:10F5A00097D0FFFFE78040BE21649305B400280098
:10F5B00097B0FFFFE78080FB97000000E78060F8CE
:10F5C000AA85280097D0FFFFE78000DF014781462A
:10F5D0003000A6854A8597B0FFFFE780801E29048A
:10F5E000480822CC230A010002CE97E0FFFFE78003
:10F5F00040C305611733FFFF6700A3AF97D0FFFF3C
:10F60000E78020BF55B71733FFFFE70243AC011176
:10F610007C003ECAB70707003ECC7C003ECE83C7C5
:10F6200095002E84AA8493F7F707A384F500A165BB
:10F63000AD05480897B0FFFFE78040F39700000052
:10F64000E78020F0AA85480897D0FFFFE780C0D662
:10F65000500801478146A285268597B0FFFFE780C5
:10F66000401605611733FFFF6700A3A89777FF1FB8
:10F670009387C7889C43094599C303C5C700828007
:10F680001733FFFFE702A3A401117C00AE843ECA3A
:10F69000A165B70707002A843ECCD1057C00480845
:10F6A0003ECE97B0FFFFE78060EC97000000E78058
:10F6B00020FCAA85480897D0FFFFE780E0CF5008DC
:10F6C00001478146A685228597B0FFFFE780600F3E
:10F6D00005611733FFFF6700C3A11733FFFFE70280
:10F6E000039F83C7950093F7F707A384F50097005E
:10F6F0000000E78020F91733FFFF6700839F17336F
:10F70000FFFFE702239B83C795000329C501411131
:10F7100093F7F707A384F5001C4283C907008547C8
:10F7200063E637079777FF1F938787D49C432E8420
:10F73000AA8485CF97000000E78080F3894763069D
:10F74000F502630409028347C90063803703230677
:10F75000390197900000E78040ED83572903898B9A
:10F7600089C797D00000E780E0B72685A28597007B
:10F770000000E78020F1A167CD0748003EC42302C6
:10F78000010002C697E0FFFFE780A0A941011733FF
:10F79000FFFF670063959767FF1F938727769C435A
:10F7A0001D4599C303C5E70082801733FFFFE702B9
:10F7B00003920111B70707003EC683C79500584D55
:10F7C0000AC493F7F7070AC8A384F5002A89AE8410
:10F7D00015C71C4283C7070093968701E18663C45F
:10F7E000060685466381D7068346E7006388F600F0
:10F7F0002307F70097900000E78020E3216493053A
:10F80000E400280097B0FFFFE78040D69700000093
:10F81000E780A0F8AA85280097D0FFFFE780C0B94D
:10F82000014781463000A6854A8597B0FFFFE780F3
:10F8300040F93504480822CC230A010002CE97E0A3
:10F84000FFFFE780009E05611733FFFF6700638AB3
:10F850001733FFFFE702A38701117C003ECAB707F9
:10F8600007003ECC7C003ECE83C795002E84AA8440
:10F8700093F7F707A384F500A165B905480897B089
:10F88000FFFFE780A0CE97000000E78000F1AA8587
:10F89000480897D0FFFFE78020B250080147814613
:10F8A000A285268597B0FFFFE780A0F10561173399
:10F8B000FFFF670003841723FFFFE702A37FAA84EB
:10F8C00001441769FF1F1309A963E14997C0FFFFAE
:10F8D000E78040C96344A400014519A833053403F7
:10F8E000832709003E9583572500639797001105EC
:10F8F0001723FFFF6700437F0504C9BF032E850060
:10F90000630A0E121763FF1F1303437E03230300D2
:10F910006315030029436390061203234E01631508
:10F9200003001D43639907101723FFFFE702A37726
:10F93000C689428A3E89BA8AB684328BAE8B2A84C3
:10F94000B5E103554E0019E501431A851723FFFF62
:10F950006700E378A167A98F116763FBE700970051
:10F960000000E78080F5814597F0FFFFE780C01237
:10F970000844B70700E05841F98F18455CC1B70744
:10F98000001FF98F1CC55C4991C7610597E0000015
:10F99000E780408BE38A09FA228597900000E78090
:10F9A00060C65DB7328597C00000E78040430D43D5
:10F9B00049DD1C44116703D54700A167A98F63FB8C
:10F9C000E70097000000E78040EF814597F0FFFFD8
:10F9D000E780800C0323840093164B01D182834778
:10F9E000B300035663008588FD8BA305F300FD7704
:10F9F0007D8E558EFD76FD16B204F18E8327430170
:10FA0000C58E231273012313D3002304530123054E
:10FA10002301A3044301BDDF228597B0FFFFE780E8
:10FA200020CDAA850844B5D1610597D00000E780B4
:10FA3000207F8DB71D431A8582801723FFFFE702C1
:10FA400063670569AA84AE89328A0144FD5A7D192B
:10FA500097C0FFFFE780C0A56347A40001451723B7
:10FA6000FFFF67006368D84493171400BA9703D761
:10FA70000700631F37032390570163070A00268599
:10FA800097900000E780A0809C449DC383D76700C7
:10FA9000B3F72701639E3701D288014881470147A8
:10FAA000814601468145268597000000E78040E5B4
:10FAB000050479BF1723FFFFE702C35F79711C10AC
:10FAC0003EC4B7070F003EC61C103EC883C7950052
:10FAD000AA8A328593F7F707A384F5002E8932842A
:10FAE00097D0FFFFE780009D93170501C187635AF8
:10FAF000F006AA89228597D0FFFFE780A09B2A8A7B
:10FB00004E85032B040097B0FFFFE780009B39ED83
:10FB10008357440081440544F11793B71700A303AA
:10FB2000F10083457100DA872287D2864E8628004D
:10FB300097E0FFFFE780E057014781463000CA8524
:10FB4000568597B0FFFFE780C0C7A1679387F7038B
:10FB500048083ECC230A810026CE97D0FFFFE780DD
:10FB6000406C45611723FFFF67000358A285130609
:10FB7000710097E0FFFFE7806066AA84094455D1D1
:10FB8000528597E0FFFFE78060D40D4459D90546C0
:10FB9000D285268597000000E78060EA2A8451B765
:10FBA0001723FFFFE702A3528355070003462700F0
:10FBB00041112A842E8532C62EC497E0FFFFE780CC
:10FBC000E0D001C93246A245228597000000E780B7
:10FBD00000E741011723FFFF6700A3511723FFFF31
:10FBE000E702634C83C795004111AA8A93F7F70790
:10FBF000A384F5003285AE89328497D0FFFFE78079
:10FC0000608B93170501C1876357F00AC1452A8AA3
:10FC1000228597C0FFFFE78080702A8D228597D0CC
:10FC2000FFFFE78020892A89228597D0FFFFE780A0
:10FC30004086930705F893F7F70F1307E007AA8BA1
:10FC4000637BF706228597D0FFFFE78080842A8CAC
:10FC5000228597D0FFFFE780C083AA8C5285032BB3
:10FC6000040097B0FFFFE780408539E983574400DF
:10FC7000231101008144F11793B71700A300F1008D
:10FC8000054403471100835621009387840056855D
:10FC9000DA8822885286CE8597F0FFFFE78020A77A
:10FCA000A167E90748003EC42302810026C697D019
:10FCB000FFFFE780005741011723FFFF6700234242
:10FCC00013061100A28597E0FFFFE7802051AA8468
:10FCD00009E52311010009446DB7930521006A85E8
:10FCE00097F0FFFFE780A0F02A8441FD83552100B3
:10FCF0009356C9001316490185486688E2875E87D6
:10FD0000858A5182268597000000E78060BF2A849B
:10FD10008DBF1723FFFFE702033983C79500411109
:10FD20002A8B93F7F707A384F5003285AE893284D6
:10FD300097C0FFFFE780007893170501C1876352E2
:10FD4000F00A2A8A228597C0FFFFE780A076AA8A58
:10FD5000228597C0FFFFE780E0752A89228597C03A
:10FD6000FFFFE7800073930705F893F7F70F13077A
:10FD7000E0072A8C6377F706228597C0FFFFE780AC
:10FD80004071AA8C228597C0FFFFE78080702A8D82
:10FD90005285832B040097A0FFFFE780007239E5AE
:10FDA0008357440085440144F11793B71700A3011A
:10FDB000F10003473100930784005A85DE882688C6
:10FDC000D6865286CE8597F0FFFFE78040948D4718
:10FDD00048003EC42302910022C697D0FFFFE7806F
:10FDE000404441011723FFFF6700632FA2851306DC
:10FDF000310097E0FFFFE780603E2A84894455D9AF
:10FE00009356C9001316490185486A88E6876287B8
:10FE1000858A5182D68597000000E78060AEAA846B
:10FE200049BF1723FFFFE702E3282A8981440144E1
:10FE3000617A916A176BFF1F130B4B2B97B0FFFF73
:10FE4000E780006863C7A40022851723FFFF6700CF
:10FE5000A3298327090093991400CE9703D507009F
:10FE600033074501420741836364570305C10327F4
:10FE70000B0019C785453E8597400000E78060E983
:10FE8000832709000504CE972390070085047DB7DA
:10FE900097000000E78060A2832709000504CE9741
:10FEA0002390070065D5814597F0FFFFE780C0BE2E
:10FEB000F1BF1723FFFFE702E31F83C7950041113E
:10FEC0002A8A93F7F707A384F50032852E893284B6
:10FED00097C0FFFFE780005E93170501C187635A53
:10FEE000F004AA89832A040097A0FFFFE780E05C62
:10FEF00031E58357440085440144F11793B7170057
:10FF0000A301F10003483100D68752850147CE8610
:10FF10002686CA8597D0FFFFE780806AA167F5072C
:10FF200048003EC42302910022C697D0FFFFE7801D
:10FF3000402F41011723FFFF6700031BA285130613
:10FF4000310097E0FFFFE78060292A8489445DD96A
:10FF50009767FF1F938787199C4381CF044997B008
:10FF6000FFFFE780E055AA85268597400000E780DF
:10FF700040DA1305040197000000E780C0EA2285FB
:10FF800097800000E78000338144ADBF1723FFFF57
:10FF9000E702631183C795004111AA8A93F7F70717
:10FFA000A384F5003285AE8932842311010097C005
:10FFB000FFFFE780205093170501C1876354F006C7
:10FFC0002A8AC145228597C0FFFFE7804035AA8B6A
:10FFD0005285032B040097A0FFFFE780004E21E924
:10FFE0008357440085440144F11793B71700A300D9
:10FFF000F1000348110003572100DA875685D286A5
:020000040001F9
:100000002686CE8597D0FFFFE780805BA167938728
:10001000270248003EC42302910022C697D0FFFF6A
:10002000E780202041011723FFFF6700430BA285D3
:100030001306110097E0FFFFE780401A2A848944E5
:100040004DD99767FF1F9387670A98433E8901CF71
:10005000044997B0FFFFE780A046AA852685974010
:100060000000E78000CB1305040197000000E78043
:1000700080DB97B0FFFFE780A04495443DD993050E
:1000800021005E8597F0FFFFE78060B6AA8435F116
:100090001C480357210022852390E7009780000029
:1000A000E780402183270900A9D703552100974005
:1000B0000000E780A0BD35BF1723FFFFE702A3FEC6
:1000C00083C795004111AA8A93F7F707A384F50027
:1000D0003285AE89328497C0FFFFE780A03D931739
:1000E0000501C1876351F0062A8A228597C0FFFF68
:1000F000E780403C2A895285032B040097A0FFFF2C
:10010000E780A03B31E58357440085440144F11763
:1001100093B71700A301F10003483100DA87568531
:100120004A87D2862686CE8597D0FFFFE780404952
:10013000A167F90748003EC42302910022C697D068
:10014000FFFFE780000E41011723FFFF670023F93F
:10015000A2851306310097E0FFFFE78020082A847C
:1001600089445DD99167CA97C2071167C183130794
:10017000F7EF8544E362F7FA9767FF1F938707F766
:100180009843BE8B01CF044997B0FFFFE78040330F
:10019000AA85268597400000E780A0B713050401D3
:1001A00097000000E78020C897B0FFFFE78040314C
:1001B00095443DD11C482285814423902701978096
:1001C0000000E780200F83A70B00B9D74A8597402E
:1001D0000000E780A0AB89B71723FFFFE70223EFFA
:1001E0002A844105B28497000000E780C0C311C58E
:1001F000228597800000E780E00B81460146A685B6
:10020000228597800000E780C04E1C4C89C7DC47E0
:1002100099C3228582971723FFFF670083ED9767B5
:10022000FF1F9387A7CD9C43014599C31385070101
:1002300082809767FF1F938767CC8843828017234C
:10024000FFFFE702C3E89317C600DD8DC205411129
:10025000C1812A8432C697C0FFFFE780E01732468B
:10026000228511829375F60F97C0FFFFE780C014B7
:1002700041011723FFFF6700C3E71723FFFFE702D2
:1002800063E379713C083ED2B7070C003ED43C08CA
:100290003ED683C79500AE842A8993F7F707A384D7
:1002A000F500A16593853504481097A0FFFFE7800E
:1002B000E02BC165FD150144176AFF1F130A8AE48C
:1002C000930A400EAE892E8B2EC697B0FFFFE780B3
:1002D00020224205931704014181C183B24563E99D
:1002E000A702C167FD176387F500481097C0FFFF9D
:1002F000E780800E501001478146A6854A8597A069
:10030000FFFFE780004C45611723FFFF6700C3DD57
:100310003307540383270A0BBA9703D6C701630A2E
:100320003601638A3501481097000000E78060F1CC
:10033000DA85050451BFB285EDBF1723FFFFE70241
:1003400083D679717C083EC8B70711003ECA7C0885
:100350003ECC83C79500AA89328593F7F707A3841B
:10036000F5002E8997C0FFFFE780C014856763788A
:10037000F504A165AA848905080897A0FFFFE78016
:10038000E01E268597400000E78060ED13341500DD
:100390000A04A285080897C0FFFFE780E001A68550
:1003A000080897C0FFFFE780200325CC014781465E
:1003B0001008CA854E8597A0FFFFE7808040456101
:1003C0001723FFFF6700A3D1B30754030327CA0A0B
:1003D000BA9703D70700631C970003D627006380F2
:1003E0006505080897000000E780A0E5DE850504A4
:1003F0002EC697B0FFFFE780A010420593170401B7
:100400004181C183B245E3E1A7FCC167FD17E38FDA
:10041000F5F8080897C0FFFFE78000FC41BFB285F0
:10042000F9B7C165FD150144176AFF1F130A8ACD8C
:10043000930A80022E8BAE8B65BF1723FFFFE70266
:1004400003C918418347170083460700A207D58FC9
:10045000D207D1832390F500834727000347170075
:100460008D45A207D98F91832310F60097C0FFFF17
:10047000E780A0E91723FFFF6700A3C71723FFFF4B
:10048000E70243C3C16401441769FF1F130989C709
:1004900093098002FD1497B0FFFFE7806006634771
:1004A000A40001451723FFFF670003C4330534038D
:1004B0008327C90A3E9583570500E38597FE050407
:1004C000D9BF1723FFFFE702E3BE2A8AAE89B284B1
:1004D000B68A97400000E78080D819E591473E85AD
:1004E0001723FFFF670043C02A894E8597C000008D
:1004F000E780E08E2A84638E0A048D476DD103570E
:100500000500C547E31D47FD0347F9018546AD4793
:10051000E317D7FC8347450081CF4146A6855D059B
:1005200097F00000E780C09E814755D9AD4745BF91
:10053000130965012302E500CA852685971000008E
:10054000E780606231C1A547E38B0AF8230204000B
:1005500079B705C183570500E39247F94146A6855F
:10056000190597F00000E780A09A81472DD9994797
:10057000BDB74E8597000000E78080F02A8495473C
:1005800039DD130955004DBF4146A68523104401AE
:10059000231134011305190097F00000E780A0999A
:1005A000228597800000E780A0EA81470DBF1723CE
:1005B000FFFFE702C3B179717C003ECCB7070A00A8
:1005C0003ECE7C003ED083C79500B2842E8493F744
:1005D000F707A384F5001306A1002A892C002685BD
:1005E00097000000E780A0E5A16528088D0597A089
:1005F000FFFFE780A0F790408355A10003558100DD
:10060000854697000000E78000ECAA84AA852808A8
:1006100097C0FFFFE78040DA0356A10083558100B1
:10062000280897000000E780C0C1300801478146D4
:10063000A2854A8597A0FFFFE780A018854748104C
:100640003ED42302910202D697D0FFFFE78060BD1F
:1006500045611723FFFF6700C3A91723FFFFE702C8
:1006600003A779717C003ECCB7070A003ECE7C0020
:100670003ED083C79500B2842E8493F7F707A384F6
:10068000F5001306A1002A892C002685970000009A
:10069000E780E0DAA16528088D0597A0FFFFE780D5
:1006A000E0EC90408355A1000355810081469700FE
:1006B0000000E78040E1AA84AA85280897C0FFFFD0
:1006C000E78080CF0356A10083558100280897005A
:1006D0000000E78000B7300801478146A2854A85BF
:1006E00097A0FFFFE780E00D48102302910202D49B
:1006F00002D697D0FFFFE780C0B245611723FFFF06
:100700006700239F1723FFFFE702639C9700000009
:10071000E78060DB1723FFFF6700A39D9757FF1F4C
:100720009387077E884382801723FFFFE702239A7F
:10073000835725004111AE842A842307B10017F5A1
:10074000FFFF130525466C002316F10097A0FFFF5D
:10075000E780204991C4228597800000E780E0D699
:10076000FD572310F40013062002814513055400A1
:100770009720FFFFE780A09841011723FFFF670044
:1007800043971723FFFFE702E39279717C003ECC89
:10079000B7070A003ECE7C003ED083C79500AA89E9
:1007A000AE8493F7F7073285A384F5001306A10002
:1007B0002C0097000000E78080C803558100114499
:1007C00097400000E780A0A915C50355A10001448A
:1007D00097B00000E780A06011CD03570500835754
:1007E000810045446318F700854597000000E780C5
:1007F000E0F30144216993053900280897A0FFFF21
:10080000E780C0D6A285280897C0FFFFE780C0BA5E
:100810000356A10083558100280897000000E78057
:1008200040A2300801478146A6854E8597A0FFFF6C
:10083000E78020F948104AD42302810202D697D0DB
:10084000FFFFE780009E45611723FFFF6700C38914
:100850001723FFFFE70203869757FF1F9387076A57
:100860002A8488432E8915C5035745038357C4013D
:100870006311F7022326050223180502410597D0CC
:100880000000E780209C6306090097800000E78055
:1008900060DB81449769FF1F9389C986130A800230
:1008A00097B0FFFFE780C0C563C4A4049757FF1F3C
:1008B0009387876D9C4399C70355C4019720000017
:1008C000E780C0BD63070900228597800000E780AC
:1008D000C0A01306400E814522859720FFFFE780C8
:1008E0000082FD57231EF4001713FFFF6700C37F2C
:1008F0003385440383A7C90A3E95035705008357F0
:10090000C4016317F700CA8597000000E78000E282
:10091000850479B71713FFFFE702C37983C79500F2
:100920004111AA8993F7F707A384F5003285AE84B5
:1009300097C0FFFFE78000B885676378F5042A89D0
:1009400097400000E780A091014401CD83D70400C7
:10095000314463882701854597000000E78080EFD8
:1009600001444E85A2864A86A68597D0FFFFE78080
:10097000A09CA1679387170448003EC4230281000E
:1009800002C697D0FFFFE780C08941011713FFFF20
:10099000670083751713FFFFE702C3719757FF1FA7
:1009A0009387C755804329C4014597C00000E7805D
:1009B000002181470148C1641CDC232E040323204D
:1009C00004041759FF1F1309E97301449309400EEA
:1009D000FD1497B0FFFFE780A0B1634FA4008145ED
:1009E00017F5FFFF1305857F97A0FFFFE780601FC6
:1009F0001713FFFF6700436F330534038327090B89
:100A00003E958357C5016387970085459700000091
:100A1000E78040E4050475BF9357050113D78700AD
:100A2000A380F50093170501C183A1832380E5000E
:100A30002381F500A381A50082801713FFFFE70241
:100A400003692300050083C71500A300F50083C7D1
:100A500025002301F50083C73500A301F50083C7F6
:100A600045002302F50083C75500A302F50083C7A4
:100A7000650093059500A30305002303F5002304F7
:100A80000500328597000000E78040F91713FFFF4B
:100A9000670023661713FFFFE702C3614111E954A2
:100AA0000DCD85CD93F9C5FF2E842A89AA84338A7A
:100AB000A900B7EA040063189A020D88854411CC96
:100AC000B7E704009C5F82972AC622866C00330534
:100AD000390197E00000E7800046268541011713A1
:100AE000FFFF6700636083A78A03910482979317CF
:100AF0000501C183A183A38EF4FE93570501238FC3
:100B0000F4FEA183238EA4FEA38FF4FE6DB763E6EB
:100B1000D5021713FFFFE702835BB28741113686C8
:100B2000BE8536C697E00000E780E040B24641014E
:100B300036851713FFFF6700C35B814636858280C9
:100B4000838705001387F5003D05FD8793F7770838
:100B5000834607007D158606B58FA300F500630761
:100B6000B7007D17834717009D83DDB78280171379
:100B7000FFFFE702C355B7E7040083A707093287E1
:100B80002A863A858297133515001713FFFF6700F1
:100B9000435615C181478DC11713FFFFE702235349
:100BA000414697E00000E780003985473E851713EE
:100BB000FFFF6700035481473E8582801DCD1713D8
:100BC000FFFFE702C350414681452A849710FFFF8B
:100BD000E780E05241468145130504039710FFFF6B
:100BE000E780E0510147C1672322040438C87CC86C
:100BF00005451713FFFF6700C34F014582808147FA
:100C00003DCDB5CD1713FFFFE702634CB2842E89AB
:100C10001306800581452A849710FFFFE780204E48
:100C2000CA8524C4268597000000E780C0F64146A7
:100C3000814522859710FFFFE780604C3044A285F4
:100C4000228597000000E780C0F293040401A2858A
:100C5000268597000000E780E0EEA68513050402D4
:100C600097000000E78000EE228597000000E780F3
:100C700020F585473E851713FFFF670083473E85B4
:100C800082801713FFFFE702E3424111E9540DCDC3
:100C900085CD93F9C5FF2E842A89AA84338AA900B9
:100CA000B7EA0400639844030D88814411CCB7E788
:100CB00004009C5F82972AC622866C0033053901A6
:100CC00097E00000E7802027268541011713FFFFEA
:100CD0006700834183A78A039104829793170501D4
:100CE000C183A183A38EF4FE93570501238FF4FEE5
:100CF000A183238EA4FEA38FF4FE6DB765CD1713D9
:100D0000FFFFE702233BB28411E605451713FFFFFF
:100D10006700833D2A842E890145EDD93C487848F7
:100D2000B3E6E700E5D69386F7FFB3B7F6007D1785
:100D3000032A4404BA9734C87CC863050A06C1492B
:100D400013050A03B38949412295637D3601B286B2
:100D50002E86A68597000000E780A0DB7C40BE942D
:100D600064C065B7CE862E86CE8597000000E780EA
:100D700040DAC114D2944E9923220404A287930628
:100D8000040103C7070003C607038507318FA38F3C
:100D9000E7FEE398F6FE3044A28522859700000026
:100DA000E78020DD2699C1493306994063EC99001C
:100DB000A9DCA686A6851305040397000000E7803A
:100DC00040D579BF8147B306F4003307F6000347E7
:100DD000070083C5060085072D8F2380E600E39476
:100DE00037FF3044A285228597000000E78060D855
:100DF000C1145DBF014582800DC11713FFFFE702DB
:100E0000032D1306800581459710FFFFE780202FF3
:100E100005451713FFFF6700C32D014582808147F9
:100E200049C5C1C51713FFFFE702632AFC414146CC
:100E30002E84AA846399C70413860501A28781467C
:100E4000C14503C7070003C507038507298F33057D
:100E5000D600034505008506298FA38FE7FEE392A0
:100E6000B6FE3044A285268597000000E78060D05A
:100E7000228597000000E78060F885473E851713BC
:100E8000FFFF67000327138507031D8E8145229509
:100E90009710FFFFE780A0267C40130700F8130699
:100EA0000402A2972388E70251BF3E858280171370
:100EB000FFFFE702C3216D712E84B284AA859010D2
:100EC0002800368997000000E780A0D309EDD557A8
:100ED00025A050400C40280097000000E78040E229
:100EE0007DD5FD142104F5F42C004A8597000000FF
:100EF000E78020F3814761DD3E8551611713FFFFD5
:100F00006700231F1713FFFFE702631C41112EC464
:100F100032C62C00054697000000E78080F94101A9
:100F20001713FFFF6700E31C1713FFFFE702231AE5
:100F300001112A842EC602C802CA02CC02CE97E052
:100F40000000E780E032B2462A86A28508089700B2
:100F50000000E78060FB1375F50F05611713FFFFB5
:100F6000670023191713FFFFE70263167971B28731
:100F70002A8421462308B10013051101BE853AC415
:100F800036C697E00000E78000FBB246930591016A
:100F9000368597000000E78060A82285141035464A
:100FA0000C0897000000E78020F62A84224701E918
:100FB00021460C103A8597E00000E780C0F72285B3
:100FC00045611713FFFF6700C3121713FFFFE70206
:100FD00003107171AE84AA850A85328497000000DF
:100FE000E78060BB11C90A86A685228597000000AC
:100FF000E78020B8814711E1C5473E854D61171351
:10100000FFFF6700030F1713FFFFE70243091D717E
:101010002A8AB289BE8435468547130511012E8C74
:10102000B68A3A8BC28C468D2308F10097E0000007
:10103000E78060F010100C085285231F0100970014
:101040000000E780C0F82A843DEDA1476313FD0846
:101050009307900591E0E5473546E28513051101B8
:1010600013990A012308F1001359090197E00000C0
:10107000E78060EC1357890093978A00D98F900816
:101080000C085285231FF10097000000E78020F430
:101090002A8415E9A1E49387FA0091831379F90072
:1010A0003EC6631309004149668B8144C14B854D9F
:1010B000B247639F970C6A868C0033855C0197E08A
:1010C0000000E78040E7228525611713FFFF6700D6
:1010D000C30093079004C9F0A547BDBF834701052E
:1010E0000947C14B2308F10083471105A58FA308C9
:1010F000F10093872400814463E1FB040147140855
:101100003386E6008C08B386E400BA95DA9683C687
:10111000060083C505000507AD8E2300D600E390C9
:10112000E7FE4147639CE70490080C08528597004E
:101130000000E780C0E925D181A0B3069B00BA87F3
:101140001008B305F60090083E9603C50600034656
:10115000060085078506298E2380C500E39277FF68
:10116000998F90080C085285BE9497000000E78084
:1011700000E68947014749D12A84B1B790083E96D5
:10118000034606001408BE962380C600850759BF93
:10119000B24785046387971481471808B306F700A0
:1011A00098083E973386F900034707000346060078
:1011B0008507318F2380E600E39177FF90080C08C4
:1011C000528597000000E78080E05DF53546E285B6
:1011D000130511012308B10197E00000E780A0D5B5
:1011E000139704014183939784002183D98F1018AA
:1011F0000C085285231FF10097000000E78020DDD6
:1012000025FD814710183387F9003E9603470700F4
:1012100003460600B306FB008507318F2380E600F6
:10122000E39277FF65A81808B306F70098083E9781
:101230003386F90003470700034606008507318F10
:101240002380E600E3E127FFCA87639E77099008C1
:101250000C08528597000000E78060D711FD814798
:101260009800B306F700900818103E973E96034783
:101270000700034606008507318F2380E600E391CF
:1012800077FF3546E285130511012308B10197E088
:101290000000E78040CA13970401418393978400BC
:1012A0002183D98F10180C085285231FF100970055
:1012B0000000E780C0D1E31105EC814710183387A7
:1012C000F9003E960347070003460600B306FB00FD
:1012D0008507318F2380E600E3E227FFC109410B38
:1012E000C1BB814785B79408BE9683C6060018081F
:1012F0003E972300D700850789BF63800632171306
:10130000FFFFE702C3D959712A84BE89B28B854792
:101310003546130511022E8B468C4289BA8A368ACD
:101320002300F10297E00000E780E0C010180C10E5
:1013300022852317010297000000E78040C9631847
:101340000512A147631FFC069307900563930900EC
:10135000E5473546DA851305110293140A01230087
:10136000F102C18097E00000E780E0BC93178A009B
:1013700013D78400D98F90080C1022852317F1020F
:1013800097000000E780A0C47DE163920904930701
:10139000FA00BD88918391E0C144C207C183DE8C0D
:1013A000814A3EC6414DB24763E2FA0E6286B3857A
:1013B0004B01881097E00000E78080B54DC93D558E
:1013C0007DA093079004E39609F8A54759B7834792
:1013D00001050947C14C2300F10283471105B3C73A
:1013E000F900A300F10293872900814963E1FC041D
:1013F000814618103306D7008C083387D900B6957C
:1014000056970347070083C5050085062D8F2300E7
:10141000E600E390D7FE41476390E70690080C1082
:10142000228597000000E78080BA35D189A0B38675
:101430003A01BA871010B305F60090083E9603C52E
:1014400006000346060085078506298E2380C50011
:10145000E39297FF3387EC4090080C102285BA99ED
:1014600097000000E780A0B68947014741D1656138
:101470001713FFFF670063C690083E9603460600F9
:101480001410BE962380C600850779B7B247850A37
:1014900093990A01939D8A0093D909016391570F8B
:1014A00085473546DA85130511022300F10293D9E9
:1014B000890097E00000E78000A8B3ED3D019000AF
:1014C0000C1022852317B10397000000E78020B09D
:1014D00059FD8147A68963EA970626860C084A8546
:1014E00097E00000E78020A581471810B306F700B9
:1014F000100898083E973E960347070003460600EB
:101500008507318F2380E600E3E197FE639FA905FD
:1015100090080C10228597000000E78040AB21F96D
:1015200081479810B306F700900818183E973E962A
:1015300003470700034606008507318F2380E60036
:10154000E391A7FF4109C10CB9BD18089000B3068B
:10155000F7003E963387FC0003470700034606006A
:101560008507318F2380E600B5B798084E9703476B
:1015700007001C10CE972380E700850941BF8547EF
:101580003546DA85130511022300F10293D989004B
:1015900097E00000E780209AB3ED3D0190000C1029
:1015A00022852317B10397000000E78040A2E310D3
:1015B00005EC814718089000B306F7003E96338784
:1015C000FC0003470700034606008507318F238090
:1015D000E600E391A7FF41460C084A8597E000002A
:1015E000E780609581471810B306F7001008980847
:1015F0003E973E9603470700034606008507318F56
:101600002380E600E391A7FF90080C102285970045
:101610000000E780C09B1DD599BD7D5582801713C2
:10162000FFFFE702C3AA01112A842E85930551000A
:10163000328902C002C202C402C69304740097F049
:10164000FFFFE780A03D1D46A6851305910097E0AA
:101650000000E780408E10088A854A8597000000C8
:10166000E780E09619ED93071400180883C6070079
:101670000346070085070507B18EA38FD7FEE397C2
:10168000F4FE05611713FFFF6700A3A61713FFFF02
:10169000E70243A22E848C414111AA898387150059
:1016A0003289914463D30700A1449757FF1F938762
:1016B00027DC9C43A1C7C1CA8D472310F10083C713
:1016C00025004A852301F10083C73500A301F100FD
:1016D00083C745002302F10083C75500A302F10030
:1016E00083C7650093059100A30301002303F10064
:1016F0002304010097F0FFFFE78040320C404A8648
:101700000A8597F0FFFFE7808033032804008356A3
:101710004400A6881D0881470147E51642868A8550
:101720004E8597000000E780408E2A8919E5A6853E
:10173000228597B0FFFFE780E0C14A85410117137A
:10174000FFFF6700639A4A860A8597F0FFFFE780EC
:10175000002F6DB71713FFFFE702C3952E848C414E
:101760004111AA89838715003289914463D3070008
:10177000A1449757FF1F9387A7CF9C43A1C7C1C61A
:101780008D472310F10083C725004A852301F1000E
:1017900083C73500A301F10083C745002302F10090
:1017A00083C75500A302F10083C76500930591002C
:1017B000A30301002303F1002304010097F0FFFFBE
:1017C000E780C0250C404A860A8597F0FFFFE78036
:1017D000002783564400032804008A85858EC206AC
:1017E0001D08C1822312D400A68881470147E5164F
:1017F00042864E8597000000E78060B041011713D4
:10180000FFFF6700638E4A860A8597F0FFFFE78037
:1018100000234DBF1713FFFFE702638BB335B00002
:10182000011185052A891315F60133651501230871
:10183000B1009305110136843AC632C03EC442C29B
:1018400097F0FFFFE780801DA2471248425593D6CC
:101850008700230BF1009305910193578800A30A99
:10186000D100A30BF100230C010197F0FFFFE780EB
:10187000E01A3247024603280400B337E0008356DB
:1018800044009207914411C2A1444A85A688428629
:101890000C0897F0FFFFE78040772A8919E5A685B5
:1018A000228597B0FFFFE780E0AA4A8505611713FC
:1018B000FFFF670003841703FFFFE702A37F011107
:1018C0003EC68647B335B0008505AA891315F601D3
:1018D0005D8D2308B1009305110136843A89B284E5
:1018E00042C446C297F0FFFFE78040132248924867
:1018F000164593578800A30AF1009305910193D7E9
:101900008800230B0101A30BF100230C110197F0B8
:10191000FFFFE780A0103247104083564400B337E2
:10192000E000920703280900914891C0A1480C08E3
:101930004E8597000000E780809CAA8401E98355CA
:1019400044004A8597B0FFFFE780C0A02685056167
:101950001703FFFF67004379AA959307F00F171746
:1019600001001307A7EE6317B50013C5F7FF137542
:10197000F50F828005058346F5FFB58FBA9783C7BB
:101980000700D5B70357450014419307F00F17160A
:1019900001001306A6EB3697420741831395060113
:1019A0004181631BE500AD8FB29703C507001305A6
:1019B00015F3133515008280850603C5F6FFA98F40
:1019C000B29783C70700D9BF1703FFFFE702237051
:1019D000B28736842E86BA86AA853E85BA8497F069
:1019E000FFFFE7806052634F0500228597E000000B
:1019F000E78000882A86A686A285268597F0FFFFC5
:101A0000E78080501703FFFF6700A36E1703FFFFF7
:101A1000E702436A5D712A8BAE8A17150100130530
:101A200065E02C00B284368ABA893E8997F0FFFFC0
:101A3000E780C04F2A845DE134104146DA852800F2
:101A400097F0FFFFE780404C2A8449E98547A303CC
:101A5000F100A6C2930771002408BEC4A68685477C
:101A60000D462C18281002DC02DED6C0BEC697F048
:101A7000FFFFE78000442A8435E183477102A68690
:101A80000D4693F7F7072300FA00C1473EDE2C18F6
:101A90008947281026DCA303F10097F0FFFFE780B9
:101AA00040412A8405ED4146A6854E8597D0000029
:101AB000E78060488D47A6860D462C182810A303A2
:101AC000F10097F0FFFFE780C03E2A8401E941461C
:101AD000A6854A8597D00000E780E04522856161B0
:101AE0001703FFFF670043601703FFFFE702235E52
:101AF00097F7000093870713984383C747007971CE
:101B00002A89AE8417150100130545D20C083AC482
:101B10002306F10097F0FFFFE78040412A8405ED9E
:101B200014104146CA85080897F0FFFFE780C03DC2
:101B30002A8415E1140815462C00081097F0FFFFC1
:101B4000E780803C2A8401E921462C08268597D02D
:101B50000000E780403E228545611703FFFF6700D4
:101B600043591703FFFFE702835697F70000938757
:101B7000670B9C477971AA842E8417150100130501
:101B800065CB0C083EC697F0FFFFE780203A0DE9D1
:101B900014104146A685080897F0FFFFE780C0367D
:101BA00005E1140811466C00081097F0FFFFE7806C
:101BB000A03519E58347F10193F7F7032300F400FB
:101BC00045611703FFFF6700C3521703FFFFE702DA
:101BD00003503688A14881470147E54697F0FFFF4B
:101BE000E780A0421703FFFF6700A3501703FFFF22
:101BF000E702E34D3688A14881470147E54697F063
:101C0000FFFFE780C06F1703FFFF6700834E1703D6
:101C1000FFFFE702C34B01112A842E850C0832C650
:101C200097F0FFFFE780803009ED324797160100FB
:101C30009386C6BE1008C145228597000000E78044
:101C4000E0D805611703FFFF6700A34A1703FFFFF2
:101C5000E702E3474111C1472EC032C48A850946D5
:101C60003EC23EC697F0FFFFE780A0244101170364
:101C7000FFFF670003481703FFFFE70243454111D9
:101C8000AE8613061009AA850A8502C002C202C4E4
:101C900002C697F0FFFFE780202741011703FFFFEF
:101CA000670023451703FFFFE70263423287971659
:101CB00001009386A6B82E869305000297000000C7
:101CC000E780C0D01703FFFF6700A3421703FFFFA1
:101CD000E702E33F7971C1472ACC2ED032D42C08D9
:101CE0000D4628003ECE3ED23ED602C402C602C8F1
:101CF00002CA97F0FFFFE780C01B45611703FFFF93
:101D00006700233F1703FFFFE702633C0111AA842A
:101D10002E84171501001305E5B28A8597F0FFFFA1
:101D2000E780C02015E514084146A6850A8597F08E
:101D3000FFFFE780601D09ED8347E1010347F101E3
:101D4000A207D98FCA07C9836177D98F2310F400FE
:101D500005611703FFFF6700C33915CD1703FFFFA8
:101D6000E702E3369747FF1F9387071E9043974587
:101D7000FF1F9385A51D1745FF1F1305E51897D075
:101D80000000E78000C51745FF1F1305E51717037F
:101D9000FFFF670003361745FF1F1305E516828016
:101DA0008DCD1703FFFFE70283329747FF1F93870D
:101DB000A719944301112E840A869745FF1F938526
:101DC000E51897D00000E78040C60A8502940145D7
:101DD00005611703FFFF6700C3317D55828017033C
:101DE000FFFFE702C32E97D00000E78080D197471E
:101DF000FF1F23ABA71417F5FFFF1305E5C997B025
:101E00000000E780C0741703FFFF6700832E1747A9
:101E1000FF1F1307A7159317150008433E95FD579D
:101E20002310F50082801703FFFFE702432A2A846C
:101E3000084009E51703FFFF6700A32B1C4158402A
:101E40001CC06313E5005CC08347550023200500D8
:101E5000F99BA302F50097A0FFFFE780207CC9BF94
:101E60001703FFFFE70203259747FF1F938707121A
:101E700098432A8411CB8347350093F7070289C71B
:101E800003550500894502971305440197B00000EA
:101E9000E780403B835504000355E4009730000081
:101EA000E780A00C485819C597A0FFFFE78000778E
:101EB000232A04021305840397000000E780E0F65C
:101EC0008144B1499790FFFFE780C06D63CBA402C6
:101ED000834734002320040493F727FCA301F40074
:101EE00000489790FFFFE780E06C131615008145CE
:101EF00022859700FFFFE78080201703FFFF670020
:101F0000A31EB38734030329040385043E994A853D
:101F100097000000E78060F12304090065B783475C
:101F2000350093F7070299E3014582808357E50066
:101F3000E39CB7FEC167FD176316F6000545828076
:101F4000054599A81703FFFFE702631893170601D9
:101F5000C187B2842A8401496359F002835705007E
:101F60009DCB01456367F600034584003E9533250C
:101F7000A6001375F50F0DA01C4813171900BA978A
:101F800083D70700E38E97FA05099790FFFFE78054
:101F90006062E343A9FE01451703FFFF6700631575
:101FA0001703FFFFE7020311AE89AA849790FFFF92
:101FB000E78000562A8497D0FFFFE780A02EAA86EC
:101FC00001471306840197050000938585E41745B2
:101FD000FF1F1305E5F99790FFFFE780801C2A8912
:101FE00025C98C441304C50022859E0593F5050878
:101FF00097A0FFFFE780403CCC4083877400E181DD
:1020000063DD070493E50508228597A0FFFFE780BD
:10201000A03A0D4693854400228597A0FFFFE780F4
:10202000C03683D50400228597A0FFFFE780E03DFE
:1020300083D52400228597A0FFFFE780003D03D6CB
:10204000490083A50900228597A0FFFFE780E033C0
:102050004A851703FFFF6700230993F5F5076DB75E
:102060001703FFFFE702A30601112A84328532C657
:1020700097A0FFFFE780E0279780FFFFE7806034AD
:10208000835704001747FF1F1307C7073246231B58
:10209000F100930700F8A30DF1001C471843231A21
:1020A000A1008983858BB307F740B28548083ECEEF
:1020B000231C0100230D010097000000E78080EE43
:1020C00005611703FFFF6700C3021703FFFFE70265
:1020D00063FE004101453DC49304C4002685328956
:1020E000AE8997A0FFFFE780C02495452A8A268500
:1020F000035B040197A0FFFFE7802021268597A0BE
:10210000FFFFE780603E8D45AA8A268597A0FFFFE6
:10211000E780A01F268597A0FFFFE780E03C5C4892
:10212000420A135A0A01D2975CC4231864018147FA
:1021300063983A0146054D813306254193371600D1
:1021400013F5F70F1703FFFF670003FA1703FFFFED
:10215000E70263F589692A8BAE8B328AB68A81449D
:102160000144314CFD199790FFFFE780A04363CDF8
:10217000A4009790FFFFE780E045018D33B5AA00EA
:102180001703FFFF6700A3F53389840383270B0040
:102190003E9963170A008347890085043E94E1B79E
:1021A00003560A00DE854A8533F6C9009700000011
:1021B000E780E0F16DD10545E1B71703FFFFE702C6
:1021C00003F101112A847C000355E5003ECAB707DC
:1021D00007003ECC7C003ECE97200000E780200820
:1021E0002A898545480897A0FFFFE780203999454F
:1021F000480897A0FFFFE780E015AA844A8597204A
:102200000000E780A0082380A4009747FF1F938762
:1022100067EF9C434166130606F09396870113D738
:102220008701558F93D68700F18E558FA207B70689
:10223000FF00F58FD98F11462C00138514003EC482
:1022400097D00000E78020CF5008A3820400894582
:10225000228597000000E780E0E019C9AA851305F0
:10226000840397A0FFFFE780E0313C4085073CC036
:1022700005611703FFFF6700C3E71703FFFFE702CE
:1022800003E59790FFFFE780E0342A8405049790E8
:10229000FFFFE78020333305A402F1479145330562
:1022A000F50297200000E78020BA11E56555170375
:1022B000FFFF670003E49747FF1F23A1A7CC979078
:1022C000FFFFE78020312A8405049790FFFFE78015
:1022D000602F3305A4028945060597200000E7809A
:1022E000A0B669D59747FF1F23A2A7C89790FFFF05
:1022F000E780402E2A8405049790FFFFE780802C1A
:102300003304A4029747FF1F239487C69790FFFFCB
:10231000E780402C2A849790FFFFE780A02A93074C
:1023200014003385A7029747FF1F2394A7C497077C
:1023300001009387E7141747FF1F232FF7C20145BA
:10234000BDB71703FFFFE702E3D6AA842E89014435
:102350009749FF1F938909DB130A80069790FFFFB7
:10236000E78040266347A40001451703FFFF67008D
:10237000A3D73305440383A709024A86A6853E9561
:1023800097000000E780E0B919E10504C1BF0545E9
:10239000E9BF1703FFFFE70203D1AA8A2E8BB28B96
:1023A000368C3A8A814401448149974CFF1F938CB3
:1023B0006CD5130D80069790FFFFE780A02063C9BE
:1023C000A40011E085494E851703FFFF670023D164
:1023D0003389A40383A70C025E86D6853E994A857D
:1023E00097000000E780E0B31DC19790FFFFE780F2
:1023F000601E0544636D4501D2866286DA85130549
:10240000090397000000E780A0D411C18549850425
:102410005DB71703FFFFE702E3C9C16441112A89D1
:1024200001449749FF1F9389E9CD130A8006FD14E3
:1024300036C632C42EC29790FFFFE780A01892459F
:102440002246B2466348A400014541011703FFFF3D
:10245000670083C93305440383A709023E9509C673
:1024600083473500C18B9DC791C68347350093F7DD
:1024700007028DC3630699008357E500639C27011B
:102480000357050001CB63E7E50083478500BA9752
:10249000E3CDF5FA050469BF1703FFFFE70283C127
:1024A000C1642A8901449749FF1F9389A9C5130A6A
:1024B0008006FD149790FFFFE780C0106346A400DC
:1024C0001703FFFF670043C23305440383A70902D4
:1024D0003E958357E500638A9700630499006396ED
:1024E000270197000000E780E0970504E1B7170394
:1024F000FFFFE702C3BA89692A8AAE8A328BB68B9C
:102500008144174CFF1F130CECBF930C8006314D18
:10251000FD199790FFFFE780E00A63C6A400170348
:10252000FFFF670083BB3389940383270C02835525
:10253000CA015A863E994A8597000000E780609E4E
:1025400031C1814D15A03384AD038327090303D620
:102550000B00D68533F6C9003E9422859700000013
:10256000E780E0B609E9850D9790FFFFE7808003DB
:10257000E3CBADFC01A8228597000000E780E08A4C
:1025800023040400850471B71703FFFFE702A3B11A
:102590004169AA8A014A174BFF1F130BABB67D197D
:1025A000C14B054C9790FFFFE780C0016346AA002E
:1025B0001703FFFF6700A3B293098006B3073A032E
:1025C00083290B02BE9983D7E900638E27016384B8
:1025D0002A01639A570103A4890301E84E859700F5
:1025E0000000E780C0BD050A75BF835704016399E9
:1025F00077099304C400268597A0FFFFE78060D386
:1026000085452A8D2685835C040197A0FFFFE7801E
:10261000C0CF268597A0FFFFE780A0E76205618510
:10262000635905048D45268597A0FFFFE780E0CD1F
:102630008945268597A0FFFFE78020CD894526851F
:1026400097A0FFFFE78060CC8545268597A0FFFF18
:10265000E780E0CC83470500094793F7F707639AC3
:10266000E7009945268597A0FFFFE78040CBA302AE
:1026700085014848337D2D01231894016A9548C48B
:102680000040A1BF1703FFFFE70263A437E4040083
:102690008327041D82979747FF1F83C7A7931715AA
:1026A000FF1F130565E7A300F5008327441C8297ED
:1026B0008327841C81461306F00F814501458297CC
:1026C0001703FFFF6700E3A21747FF1F1307878069
:1026D00018439745FF1F83C5E58F9747FF1F9387D3
:1026E000E78D83468703034697036397D500974793
:1026F000FF1F2381C78E828083C587010347A703FD
:102700006317B6009747FF1F2386E78C828003C6B6
:1027100087016317C7009747FF1F238DD78A8280E1
:1027200083C68701130750026319D700930760021D
:102730001747FF1F2300F78A828083C6870113068D
:1027400060026315D60093077002DDB783C7870167
:1027500055BF9747FF1F93876786D44B0947638D03
:10276000E6081703FFFFE70283961749FF1F1309C7
:1027700029823E8483470900918B9DCFB7E40400F2
:1027800083A7041D829783A7441C1745FF1F1305C9
:10279000A580829783A7841C81461746FF1F0346A6
:1027A000A68181450145829721C583470900ED9B9C
:1027B0001737FF1F230EF77C8347040093F7F70FAB
:1027C00085CB91471747FF1F2324F7809700000010
:1027D000E78080EB97000000E78040EFB7E7040058
:1027E000BC4F414691451735FF1F0345A57D829794
:1027F0001703FFFF6700E38F82801703FFFFE702E5
:10280000038D8D4741116306F504C5476308F50242
:1028100085476310F5029737FF1F238FA77AB7E725
:102820000400BC4B930500101735FF1F0345857945
:10283000829741011703FFFF6700A38B8547173776
:10284000FF1F230BF778B7E70400BC4B930500206C
:10285000E1BF9737FF1F93876776D44B1147638D8E
:10286000E600B7E7040083A7071D8297B7E70400D7
:10287000BC4B930500044DBF05491737FF1F2329A3
:10288000277583C7070032C62E8493F7F70FD5D379
:10289000B7E4040083A7041D7D141374F40F82971A
:1028A000E37689FCB245994703C61500E3F0C7FCFF
:1028B000FC4409061735FF1F130545728297BC4873
:1028C000930500081735FF1F0345C56F829779BF31
:1028D00017F3FEFFE702A37F1737FF1F1307076EEB
:1028E0004047184B1C409736FF1F23AFF66C63160A
:1028F000E4001737FF1F232BF76C130584FE979016
:10290000FFFFE78000AA035564FF9780FFFFE78081
:10291000807297A0FFFFE78060D017F3FEFF67008B
:10292000437D17F3FEFFE702837A9737FF1F9387F4
:10293000E768D84BDC4789C797000000E78080F93B
:1029400085471737FF1F2325F7689737FF1F9387A2
:1029500067589C43930500021735FF1F03458566A2
:1029600083C787031737FF1F2306F766B7E70400FF
:10297000BC4B829717F3FEFF6700A3779737FF1FC3
:1029800023A0A764828017F3FEFFE702A37237E457
:1029900004007C4CA1451735FF1F0345A5628297B3
:1029A0007C48A1451735FF1F0345C5619734FF1FBC
:1029B0009384C4608297DC4489EB97000000E78031
:1029C00080D917F3FEFF6700237203D567FF978056
:1029D000FFFFE7804066AA896DD1D8489147631010
:1029E000F7027C4C91451735FF1F0345A55D829783
:1029F0007C4891451735FF1F0345C55C829703A9A5
:102A0000490103D409018947B7E904001737FF1FBB
:102A10002320F75C83A7091D21044204829783C702
:102A200084011715FF1F130525AF61191717FF1F25
:102A3000A304F7AE83A7491C418082979737FF1FF5
:102A4000238C075883A7C91C814609469375F40F48
:102A50004A85829711E99737FF1F83C7276889C77F
:102A60009700FF1FE780E017B7E70400BC4F21463F
:102A7000A1451735FF1F0345E554829799B717F312
:102A8000FEFFE702C36493F7052001112E8481CF76
:102A900097000000E78020E913450420056117F343
:102AA000FEFF6700036593F70510A9CF9734FF1F5A
:102AB0009384C450DC4897000000E78020C117379A
:102AC000FF1F13072741184383C784010347870368
:102AD0006318F700DC4489C797000000E78080DFB7
:102AE00085471737FF1F2325F74EB7E70400BC4B78
:102AF000930500021735FF1F0345C54C8297134508
:102B0000041069BF93F70508BDC79737FF1F83C738
:102B1000F74CE91719469735FF1F9385454C130568
:102B2000D10093F4F70F1739FF1F0349294B97C0C2
:102B30000000E780404093970401C1831737FF1FCF
:102B40001307474A231DF100231CF1009737FF1F8D
:102B50009387C7463ACE3ACAD8432306010009CB29
:102B6000DC439315890154080D46E185680082977E
:102B70001345040825B793F72500A5C39737FF1F12
:102B80009387C743D84B89476306F7029737FF1FE0
:102B900083C7074013F7270011EF918B99CFB7E751
:102BA0000400BC4F1306000A89451735FF1F034573
:102BB0006541829713452400D5B59737FF1F93874A
:102BC00067319C4383C787031737FF1F2304F740F0
:102BD00097000000E78060DBF1BF93F7050281CB2F
:102BE00097000000E78060DA1345040245BD93F7C3
:102BF000850081CB97000000E780E0D21345840078
